:020000022000DC
:1060000000000120756302005D6302005F6302000F
:106010006163020063630200656302000000000028
:1060200000000000000000000000000067630200A4
:1060300069630200000000006B6302006D630200F0
:10604000C99D02006F630200CDA102006F630200D0
:106050006F6302006F63020081A002006F630200A1
:106060006F6302006F6302006F6302006F630200E0
:106070006F6302006F6302006F6302006F630200D0
:106080006F630200FD7B02006F6302006F6302001A
:106090006F6302006F630200650203006F6302001A
:1060A0006F6302006F6302006F6302006F630200A0
:1060B0006F6302006F630200000000000000000038
:1060C0006F6302006F6302006F6302006F63020080
:1060D0006F6302006F6302006F6302000000000044
:1060E00000000000000000000000000000000000B0
:1060F00000000000000000000000000000000000A0
:10610000000000000000000000000000000000008F
:10611000000000000000000000000000000000007F
:10612000000000000000000000000000000000006F
:10613000000000000000000000000000000000005F
:10614000000000000000000000000000000000004F
:10615000000000000000000000000000000000003F
:10616000000000000000000000000000000000002F
:10617000000000000000000000000000000000001F
:10618000000000000000000000000000000000000F
:1061900000000000000000000000000000000000FF
:1061A00000000000000000000000000000000000EF
:1061B00000000000000000000000000000000000DF
:1061C00000000000000000000000000000000000CF
:1061D00000000000000000000000000000000000BF
:1061E00000000000000000000000000000000000AF
:1061F000000000000000000000000000000000009F
:10620000354936480A1A02D0072291438D4634494F
:1062100034480A1A06D00722914381F309880222E2
:1062200082F3148830483149314A00F044F831484B
:106230003149324A00F03FF831483249324A00F0E1
:106240003AF832483249334A00F035F83248334997
:10625000334A00F030F833483349344A00F02BF821
:1062600033483449344A00F026F83448344900228F
:1062700000F02CF833483449002200F027F8334866
:106280003349091A082902DB002202604160314AC1
:1062900090471F481F49884205D00268043003B464
:1062A000904703BCF7E700208646EC46002000211B
:1062B000294A9047FEE7884207D0521A05D0037852
:1062C00001300B700131013AF9D17047884202D098
:1062D00002700130FAE770470000012000E0002062
:1062E00000000120000001202C3103007422002056
:1062F00074230020D0630200D0630200F80703007B
:106300002C31030074220020742200208C09030029
:106310008C0903008C0903008C0903008C0903001D
:106320008C0903008C0903008C0903002C31030045
:106330002C320300742300207423002074230020D7
:106340008C3500208C3500208C3500208C350020C9
:106350008C5500209D63020079B30200FEE7FEE742
:10636000FEE7FEE7FEE7FEE7FEE7FEE7FEE7FEE705
:1063700000F002B8FFF7FCBF0F484FF00701884359
:1063800085460E4880470E48016841F4700101605F
:10639000BFF34F8FBFF36F8FFFF732BF09480A4932
:1063A0000A4A884207D0521A05D0037801300B7090
:1063B0000131013AF9D1704700000120ED6E020071
:1063C00088ED00E07809030060220020742200209C
:1063D000F0B595B01D46164608460C4603F05EFA29
:1063E0001A9B0D93CDE9086500252B46082205A9C7
:1063F00020460A958DF82C500C9503F06BFA079BFC
:106400000293069B03939DF814308DF8115003F00E
:106410000302012A1DD1BDF81420059DC3F3C20358
:10642000C2F383168DF81030B20008230EA920465F
:1064300003F050FAC5F3952508AB0093324602AB42
:106440000EA9284600F0C8FB204603F02BFA15B031
:10645000F0BD022AF8D1BDF81650C3F3C203C5F34C
:1064600089158DF810300827082D2E4628BF0826DC
:106470003B4632460EA9204603F02CFAAD1B08AB72
:1064800002AA31460EA8374400F00AFC002DEBD1D9
:10649000DAE70000014B01221A707047B523002093
:1064A0007047000070B50E4D06460FCD88B06C46A3
:1064B0000FC495E80F00002E84E80F00094A0A482F
:1064C0004FF0060308BF00226946009303F004FC66
:1064D00008B100F0C9FF054B1E7008B070BD00BFC9
:1064E0008C090300956402007422002074230020AC
:1064F00007B5044B0093044A4023FFF769FF03B03C
:106500005DF804FB0D6502007523002038B50D48C9
:106510000D4C0E4D002323700378EB5CD2B263B1B7
:10652000043004F0E1FA08B100F09EFF084B1A783D
:1065300012B12378002BFBD038BD0C3004F082F868
:10654000F1E700BF74220020B5230020082C0020B2
:106550007423002008B50848084A0378D35C3BB18F
:10656000043004F025FABDE808400020FFF79ABF88
:106570000C3003F0F1FFF6E774220020082C002015
:106580000120FFF78FBF000008B5FFF7F9FF0448AF
:10659000042100F08BFA034B01225A7108BD00BFA1
:1065A0005409030088220020037813F0040216D057
:1065B00003F00303012B03D0022B09D00120704705
:1065C0000A6800880232C0F3831002440A60F5E7CB
:1065D0000B684288023303EB92130B60EEE7104620
:1065E000704700002DE9F04FDFF81CA187B00F467F
:1065F00000230446861C0DF1070015468DF8073070
:1066000001F08EF9DAF804203A60DAF8083003F580
:1066100080739B1A0AF21C470AF583690AF2144830
:10662000B3421AD30020002D69D004F00F039B0160
:1066300043F0050363F30F00DAF80430DAB20332F3
:1066400033444AF822009DF80700CAF8043001F0EC
:106650008BF9012007B0BDE8F08F0121384602F028
:1066600089FB484602F0A1FB404602F09EFBDAF8A7
:1066700008000290C0B203300AEB800002A9FFF7C5
:1066800093FF029B30BBDAB20AEB8202D16803911E
:106690009A1C0133DBB20AEB83030292D3F80CB0ED
:1066A00001F00303012B22D0022B15D08346404674
:1066B00002F07EFB10B1029BCAF8083059463846FA
:1066C00002F058FBDAF80830DAF8042003F580739A
:1066D0009B1AA5E7D8B2CEE7BDF80E30C3F38913F5
:1066E00003334FEA1B4B02EB93030293DFE7BDF842
:1066F0000C30C3F383134FEA1B4B1344F5E7A40597
:1067000044F0060098E700BF88240020064B0748A5
:1067100010B500221A7003F07AF8044610B9044844
:1067200003F098F9204610BD882400206409030076
:10673000E009030030B50A4C71B10A4A0A49121B3C
:10674000D20800239A4201D1002030BD31F82350F5
:10675000854202D00133F5E7034654F83300F4E7ED
:106760005C0803002409030060220020094B013962
:1067700003EBC000032909D8DFE801F00A02040690
:1067800004207047007970474079704700207047B7
:10679000022070475C08030070470000034BD3E9F8
:1067A0000130C31A58425841704700BF8824002066
:1067B0002DE9F04186B0FFF7F1FF0546002840F0D3
:1067C000ED80774CC4F81804BFF34F8FA368029391
:1067D000DBB2033304EB830002A9FFF7E5FE029B63
:1067E00018B1D4F81824002A5AD0DAB2991C01330F
:1067F00004EB8202DBB204EB8303D268DB68049310
:1068000002F00303022B0392029154D1BDF80E3023
:106810006448C3F38917502F3E4628BF502606F11F
:10682000080166F38F13C1F30901ADF80E3003F0D0
:1068300006F80546002800F09C8003F02FF800239E
:10684000082203A9284603F03BF80299CB43DBB2A8
:106850000133C9B20331B6EB830F4FEA830204EB75
:10686000810125D95FFA82F80823A6EB080628469D
:1068700003F026F8F6B208F108034B4903F0FC03D5
:106880003246284603F01CF8029B033703EB9707B8
:106890000297D4F81834002B43D1D4F8106453E095
:1068A00062689A4294D8A260284606B0BDE8F0819A
:1068B00008233246E5E7012B5BD1BDF80C3039489F
:1068C000C3F38311062928BF062161F3891302311E
:1068D00001F00F018900ADF80C3002F0B0FF054661
:1068E000002846D002F0DAFF0023082203A9284638
:1068F00002F0E6FF0026BDF80C20C2F38312B300BD
:10690000964203F10803C4D202994A1CC9B203316A
:10691000029204EB81010422284602F0D1FF0136E5
:10692000E9E7284602F0BEFFFFF738FF80F00100DC
:10693000C5B2B9E7F3685B7923B1336829461B68B0
:1069400030469847F3681E68002EF3D1284602F0BF
:10695000A9FF0DF107008DF8076000F0E1FFD4F802
:1069600018340BB9029BA3609DF8070000F0FCFFF0
:10697000DAE7D4F8104454B90C4B0D480D49C01A4D
:10698000C008000440F0020000F05EF8CCE7236885
:1069900020469B689847E3681C68ECE7002583E77E
:1069A0008824002064090300942400205C0803006C
:1069B00084080300C90903002DE9F34704460E4685
:1069C000924601A9012218469946FFF70BFE1C4F7B
:1069D00010B3019D4FF00008AA1CC84508EB020146
:1069E00025D11848002102F07EF980F31000000440
:1069F00040EA1440E4006B1C04F03804DBB2EDB252
:106A000044F0010407EB8303033544EA881444EAA5
:106A10008624D86047F825403B781BB1FFF7C8FEB5
:106A20000028FBD1FFF7B8FE02B0BDE8F087C9B27D
:106A300007EB81015AF82830CB6008F10108CCE758
:106A400088240020A428002000231A46FFF7B4BFA2
:106A500007B50123019201AAFFF7AEFF03B05DF86D
:106A600004FB07B5CDE9002302236A46FFF7A4FF24
:106A700003B05DF804FB1FB5CDE90123069B03932A
:106A800001AA0323FFF798FF05B05DF804FB1FB5CB
:106A9000CDE90023069B0293079B03936A460423D8
:106AA000FFF78AFF05B05DF804FB000030B50F4C1E
:106AB000D4F8102403460020114631B9D968087172
:106AC0004AB9C4F810340A6030BDC9680D798542EE
:106AD00006D00968F1E7D26814680C601360F3E728
:106AE00001300A28E8D14FF0FF30EDE7882400207C
:106AF00038B5084B0125D3F810441D7004B938BDD2
:106B0000E3685D71236820465B689847E3681C680A
:106B1000F4E700BF8824002030B5C38885B0044660
:106B20000D4633B1144A00921449154A284602F022
:106B3000A2F9217A05291DD0637A4BB1A088FFF70D
:106B400015FE104B104953F82020284602F093F907
:106B5000227A0E4BA08853F8222003920021FFF7DF
:106B6000E9FD039A0A490346284605B0BDE83040CE
:106B700002F081B905B030BD0C0A0300F40903002E
:106B8000EC090300780A0300732303009C0A030046
:106B9000110A030007B503460846197A052911D0E2
:106BA0005B7A2BB1094A0A49019002F064F9019815
:106BB0000849019002F05FF9019803B05DF804EB19
:106BC00002F04EB9002AF8D0F2E700BF0C0A030029
:106BD00073230300090A03002DE9F04385B01F4623
:106BE0000C9D002395F80C902B7306460C4690469E
:106BF00029463846FFF790FFB8F1060F09D8DFE8BD
:106C000008F00412181F283340003146284602F0CD
:106C100032F9002229463846FFF7BCFF85F80C9070
:106C200005B0BDE8F08322683146284602F023F91A
:106C3000EFE7D4E900233146284602F01CF9E8E7E3
:106C4000A36800933146D4E90023284602F013F9E3
:106C5000DFE7E3680193A36800933146D4E900239A
:106C6000284602F008F9D4E723690293E368019308
:106C7000A36800933146D4E90023284602F0FBF8CC
:106C8000C7E76369039323690293E3680193A368E9
:106C900000933146D4E90023284602F0ECF8B8E727
:106CA00008292DE9F74F80460E4617461C463DD869
:106CB00000251B7B2573214610460193FFF72CFF0F
:106CC000DFF88CA0DFF88CB0AE4232D918F805207E
:106CD0005946204602F0CFF80135082DF4D11B4962
:106CE000DFF874A0DFF874B0204602F0C4F84FF06B
:106CF00000094E4524D918F809507E2D1ED8284683
:106D000009F0ACFC002814BF2A462E225946204622
:106D100002F0B1F809F10109B9F1080FE9D1012236
:106D200021463846FFF736FF019B237303B0BDE8C9
:106D3000F08F5146204602F09EF8CDE72E22E5E77F
:106D40005146204602F097F8E4E700BF250A030009
:106D5000210A03001B0A0300230A0300270A030079
:106D6000054A4FF0A043105CD3F8043523FA00F035
:106D7000C04300F001007047B40A0300044B1A5CE2
:106D8000012393404FF0A042C2F80C35704700BF7A
:106D9000B40A0300044B1A5C012393404FF0A04255
:106DA000C2F80835704700BFB40A030008B50020D8
:106DB000FFF7F0FF0120FFF7EDFF0220FFF7EAFFEA
:106DC000BDE808400320FFF7E5BF08B50020FFF746
:106DD000D5FF0120FFF7D2FF0220FFF7CFFFBDE86C
:106DE00008400320FFF7CABF074A4FF0A041105CDC
:106DF000D1F804350122824022EA03001340C1F891
:106E00000805C1F80C357047B40A0300054A4FF075
:106E1000A043105CD3F8103523FA00F0C04300F013
:106E200001007047B00A03000D2809D00E2809D0D0
:106E30000F2809D010280CBF03204FF0FF307047F7
:106E4000002070470120704702207047014B185CFA
:106E5000704700BFB00A0300C20708B501460CD551
:106E60004FF0A0430322C3F84427C3F84827C3F8D0
:106E70004C27C3F85027FFF799FF8B070AD54FF02F
:106E8000A0430C22C3F83427C3F83827C3F83C27A3
:106E9000C3F8402708BD4FF08053D3F83001421C9F
:106EA00004BF4FF0704393F8E00F831F58425841DE
:106EB000704700004FF0704393F8E02F062A09D185
:106EC000D3F8E83FC3F30313033B042B02D8024A71
:106ED000D05C704700207047C70A0300024AD2F80E
:106EE0000034002BFBD0704700E0014010B5FFF7E5
:106EF000D2FF40B14FF08053944AD3F82433C3F308
:106F00000423C2F84035FFF7D5FF10B1904B914AEA
:106F10005A67FFF7C0FF48B14FF080534FF08042EF
:106F2000D3F84432C3F34233C2F83C35FFF7C2FF13
:106F300030B1894AD2F8FC3023F08073C2F8FC30BB
:106F4000FFF7A9FF40B14FF080430022C3F80C21A6
:106F5000C3F81021C3F83825FFF7ACFF20B14FF07C
:106F600080430322C3F8A025FFF7A4FF60B17B4B49
:106F70000522C3F810260122C3F888260022C3F890
:106F800018263F22C3F814264FF08053D3F830213F
:106F9000511C09BF4FF07043D3F8343193F8E02F00
:106FA000D3F8E83F08BFC3F30313062A4DD1033BD0
:106FB000042B03D86A4AD35C002B46D04FF0805292
:106FC000684BD2F80414C3F82015D2F80814C3F89B
:106FD0002415D2F80C14C3F82815D2F81014C3F8ED
:106FE0002C15D2F81414C3F83015D2F81814C3F8BD
:106FF0003415D2F81C14C3F84015D2F82014C3F885
:107000004415D2F82414C3F84815D2F82814C3F84C
:107010004C15D2F82C14C3F85015D2F83014C3F81C
:107020005415D2F83414C3F86015D2F83814C3F8E4
:107030006415D2F83C14C3F86815D2F84014C3F8AC
:107040006C15D2F84424C3F87025FFF724FF48B12B
:107050004FF080534FF08042D3F8583203F04F0383
:10706000C2F8E43EFFF717FF48B14FF08043D3F872
:107070000024D20744BF6FF00102C3F800244FF090
:107080008053D3F83021062A0ED1D3F83431033B94
:10709000042B02D8344AD35C33B1344AD2F83C379B
:1070A00043F48063C2F83C372B4AD2F8883043F46B
:1070B0007003C2F88830BFF34F8FBFF36F8F4FF06C
:1070C0008053D3F83021062A0FD1D3F83431033B53
:1070D000042B02D8264AD35C3BB14FF01023D3F8DF
:1070E00008224FF08043C3F858254FF01023D3F8FF
:1070F0000022002A03DBD3F80432002B22DA1D49D8
:1071000001234FF01020C1F804351524FFF7E6FEE7
:10711000C0F80042FFF7E2FEC0F80442FFF7DEFECF
:107120000023C1F80435FFF7D9FEBFF34F8F0A499A
:10713000114BCA6802F4E0621343CB60BFF34F8F78
:1071400000BFFDE70D4B0E4A1A6010BD0030014034
:1071500000C007400DF0ADBA00ED00E00050004067
:10716000B80A030000C00040BD0A03000010004040
:10717000C20A030000E001400400FA05902200204A
:107180000090D003C30710B507D4F023054A400888
:10719000145C23401943115410BD0901C9B20F23D7
:1071A000F4E700BF5029002030B5094B1C78094B8B
:1071B000196800239C4202DC0022104630BD11F801
:1071C0003350854201EBC302F7D00133F2E700BF31
:1071D000402900206029002013B504460191FFF7E3
:1071E000E3FF38B143682BB10199204602B0BDE8F6
:1071F0001040184702B010BD034B04481968002224
:10720000490800F055BA00BF442900209822002008
:1072100010B5C0B2FFF7C8FF0446007802F026FFA1
:1072200063785A1E53425341834208D1044BD3E939
:107230000023134303D1BDE81040FFF7DDBF10BDAD
:107240004829002037B54308374AD35CC2074CBFF2
:107250001B0903F00F0304460D46042B25D8DFE875
:1072600003F003262F3C4000F9B10121FFF78AFF0C
:1072700000230DF107008DF8073000F051FB0120CD
:10728000A4F12003C4F12001284A20FA01F100FAF8
:1072900003F30B43A040D2E9004120430B43C2E972
:1072A00000039DF8070000F05FFB03B030BD00292C
:1072B00018BF0221204603B0BDE83040FFF762BF8F
:1072C00049B10321FFF75EFF0121204603B0BDE86D
:1072D0003040FFF781BF0121ECE70029E5D104210F
:1072E000E8E709B10321E5E7FFF74CFF294620460F
:1072F000FFF772FF0DF107008DF8075000F010FB4B
:107300000120A4F12003C4F12001084A20FA01F170
:1073100000FA03F30B43A040D2E9004124EA000045
:1073200021EA0303BBE700BF5029002048290020C1
:107330002DE9F041124E134F00243378A34208DCAC
:10734000114BD3E90023134318D0BDE8F041FFF7F8
:1073500053BF3D6805EBC40815F8340002F086FE03
:1073600098F801305A1E53425341181A4142414184
:1073700015F83400FFF766FF0134DEE7BDE8F08161
:10738000402900206029002048290020092AF7B55B
:1073900005460C4616463ED902F0A0FDE8B11F4B4B
:1073A0001F481D601F4B204F1C70204B00211022D6
:1073B0001E6009F0BEF91E4B00200021C3E9000148
:1073C000013CE4B20326FF2C0DD11A4A1A480021D1
:1073D00003B0BDE8F04000F059B902F047FD0028C5
:1073E000DDD003B0F0BD9DF8063015F834008DF8FF
:1073F000046005EBC40223F007038DF8063001A9F1
:1074000093788DF805303A4602F072FD013CE4B203
:107410000028D8D0E5E70720E3E700BF6029002077
:107420005029002040290020117202004429002028
:107430004829002031730200D80A030070B5084DB6
:10744000084E00242B789C4201D3002070BD336885
:10745000012113F8340002F0C3FD0134F2E700BF4C
:1074600040290020602900201FB50021039001AAB7
:1074700044F20100CDE9011100F004F805B05DF817
:1074800004FB000038B572B6FFF732FBFFF790F946
:107490000028FBD1104B114C114D1249E41AE4089D
:1074A000240444F00100FFF7CFFAD5F8F030DB07F1
:1074B00000D500BE0C4944F00200FFF7C5FABFF347
:1074C0004F8FEA68094B02F4E0621343EB60BFF3AD
:1074D0004F8F00BFFDE700BF5C0803008408030076
:1074E00000ED00E0DC0A0300E80A03000400FA05EE
:1074F00010B5D0E90243D1E90202A04272EB0303C6
:107500002CBF0120002010BD08B50A4800F05FFB29
:10751000094AD2E90031C018084BD3E9002341F1F0
:107520000001904271EB030303D210F1807041F12E
:10753000000108BDB822002068290020E0290020B1
:1075400037B505460C460A4801A901F000FB60B1B9
:107550000570446001A9064801F023FB18B10548F5
:1075600000F03AFB002003B030BD0420FBE700BF71
:10757000CC290020B8220020294B73B51E78044680
:107580001EB90026304602B070BD0028F9D0FFF7C2
:10759000BBFFD4E902239042994139D300230DF176
:1075A00007008DF8073000F0BBF923692BB94FF0C5
:1075B000FF324FF0FF33C4E902239DF8070000F0CB
:1075C000D3F9D4E90530984700250DF107008DF86F
:1075D000075000F0A5F92369C3B1D4E90212B2F152
:1075E000FF3F08BFB1F1FF3F05D05B1842F1000239
:1075F000C4E9023235469DF8070000F0B5F9002DC8
:10760000BFD00848214602F044FABBE71D46F2E726
:10761000B3F1FF3F08BFB2F1FF3FB2D0F1E700BFC7
:1076200070290020040B030013B5114B1149186891
:10763000019008231048582201F054FA044698B9E2
:107640000E4A0F4801A900F0B3F9044660B90C488E
:10765000012100F09FFA01230A4A0948194600F067
:1076600001FA094B01221A70204602B010BD00BF7A
:10767000000B030074290020CC2900206977020048
:10768000B8220020FFFF7F007029002030B56AB1CA
:1076900003684FF0FF344FF0FF355A614A1E5142E4
:1076A000C3E9024551411961002030BD0720FCE7C4
:1076B000F7B5044600250DF1070017460E468DF874
:1076C000075000F02DF9D4E90223B3F1FF3F08BFC2
:1076D000B2F1FF3F07D1FFF717FF301841F100016A
:1076E000C4E9020101259DF8070000F03DF955B1FC
:1076F0002369A76103B126612146002003B0BDE8DC
:10770000F040FFF71DBF284603B0F0BD37B5054672
:1077100000240DF107008DF8074000F001F9D5E9CC
:107720000223B3F1FF3F08BFB2F1FF3F1FBF4FF08D
:10773000FF324FF0FF33C5E9022301249DF8070013
:1077400000F012F934B12946012003B0BDE8304001
:10775000FFF7F6BE204603B030BD0000014800F040
:1077600036BA00BFB82200202DE9F743064600F0E4
:1077700019FA40B1624AD2E9003113F1807341F144
:107780000001C2E900310021304600F01AFA38B198
:107790005C4C236823B12068FFF7EEFE00232360D2
:1077A0000121304600F00DFA20B1FFF7ADFE564B37
:1077B000C3E900015548534C01A901F002FA4FF00A
:1077C000FF384FF0FF39A0B9DFF844814D4D4046F6
:1077D00002F075F9002800F08580D0E90223B3F1AA
:1077E000FF3F08BFB2F1FF3F32D1404602F061F9DE
:1077F000EDE70378012B20D0022B08D1444D284619
:1078000002F057F9002877D0C0E90289F7E75BB9A1
:107810004168D1E90223B3F1FF3F08BFB2F1FF3F56
:1078200002D03B4802F035F901A9384801F0F4F9DB
:1078300001A9364801F0C5F9C5E7416823689942B6
:1078400002D100232360EFE7314802F03BF9EBE778
:10785000296891B12968D1E9020182428B412FD276
:107860002B68D3E90223B3F1FF3F08BFB2F1FF3F1A
:1078700003D02968404602F00CF9404602F019F99D
:10788000D0E902490746FFF73FFE201A69EB0109DC
:10789000012879F1000318DBB0F5350F13D3FFF79A
:1078A0005DFF1C4A02441C484FF49603002100F07F
:1078B000F9F890B92B6813B9304600F0CBF82F6077
:1078C00003B0BDE8F0832246EDE71348002100F045
:1078D0006EF93846FFF750FE01E00D28F9D000237D
:1078E0002B6074E7074B1B68002BE9D1304603B0CF
:1078F000BDE8F04300F0B2B8084B01221A7093E7DC
:1079000068290020E8290020E0290020CC29002057
:10791000040B0300FFFFB400B822002070290020F0
:1079200070B5EFF3108672B60C4A946801239CB9C7
:1079300093600B4B0B4DD3F8801029401160C3F8B6
:107940008050D3F8841051604FF0FF32C3F8842088
:10795000047006B962B670BD0370FAE7EC29002026
:1079600000E100E0FC06FFBD084B9A6810B55AB173
:1079700050B9EFF3108172B6054A1C6814605C6858
:107980005460986001B962B610BD00BFEC290020B8
:1079900000E100E0435882B03BB10023435043581C
:1079A0000193019B012002B070471846FBE70000DD
:1079B000F8B5204B4479204E43F824201F4A204B31
:1079C00006EBC4049B1A2279DB081B0432B143F096
:1079D00002001C49FFF738F80820F8BD02680C883F
:1079E000C2F8084590F904508A7804795201002DB4
:1079F000D2B219DB14494F1987F8002301226D090F
:107A000004F01F0402FA04F441F82540427906EB21
:107A1000C201012446F832000C7143F003000B4907
:107A2000FFF712F80020D8E7094904F00F040A55BF
:107A3000ECE700BF002A0020F82900205C080300C2
:107A400094080300100B030000E100E0320B030078
:107A500014ED00E0036801221A60704703680122F8
:107A60005A60704773B501F15005AD000068ADB2C2
:107A70004FF480348C400026C0F80843C0F84843D7
:107A8000465101F5A8714559019522F07F42019DAB
:107A900040F82120C0F844430BB1C0F8044302B0C1
:107AA00070BD00002DE9F74F0D4622F07F440268BB
:107AB0004FF4803705F150068F408046B60002EB48
:107AC0008500C2F84873B6B2C2F80873D2F804153C
:107AD00099464FF0000BD0F84035C0F8401542F8F9
:107AE00006B05B1A9259009223F07F43012B009A53
:107AF0004FEA850A0CD1264B4FF4806043F0010316
:107B00009847D8F8003043F806B09B590193019B81
:107B1000D8F80010D1F80465C1F84473A31B23F012
:107B20007F43012B1CD11A4B05F5A875013443F096
:107B3000010341F825404FF480609847D8F80030A1
:107B4000D3F804359E4209D1D8F800300020C3F89C
:107B50004473C3F8047303B0BDE8F08F0D20FAE757
:107B60008A44C9F1FF13CAF84045D1F80405221A26
:107B7000013A22F07F4203F57F439342EED3002A7D
:107B8000E2D10134CAF84045D1F804359842DAE729
:107B9000500B030003680222C3F8442309B1C3F861
:107BA0000423704700684FF48271FFF7F3BE4FF46F
:107BB000803303FA01F10368C3F84813C3F80813CC
:107BC000704750318900006889B2FFF7E3BE03684F
:107BD000D3F804057047000090F90430002B09DB4E
:107BE0005A09012103F01F0301FA03F3403202494D
:107BF00041F82230704700BF00E100E0024B034A29
:107C00001B681068184700BF002A0020F8290020D0
:107C100070B5064D0646002455F8043B0BB13046BE
:107C200098470134042CF7D170BD00BF102A002002
:107C30004388033300EB830399420BD382884FF6CA
:107C4000FF739A4208D0038833B18068431C5842BE
:107C5000584170470220704701207047033080B2BE
:107C600040F2FE33984230B51FD8134B1A783AB918
:107C70001C895D892C440444A4B2B4F5806F0AD9F0
:107C80001A7DAAB99A8BDC8B2244024492B2B2F5D7
:107C9000806F0DD801220A801446142202FB04339F
:107CA0005A8910445881002030BD48F20860FBE733
:107CB00048F20660F8E700BF442A00200B4A0C494E
:107CC0005388142000FB0311CB6833B904204968A2
:107CD00010700122074801F063BB074905231370A8
:107CE00002238B80012209680023F3E7282A002061
:107CF000442A0020602200200C2B002007B500231E
:107D000005490093054A09680548082301F0AEFAC1
:107D100003B05DF804FB00BF0C2B0020640B0300D4
:107D20006022002007B5002301460093034A04485F
:107D3000082301F09BFA03B05DF804FB5C0B030021
:107D40006022002013B500230C4600930146084A28
:107D50000848042301F08AFA38B9074B142101FBC3
:107D6000043101230B7402B010BD48F20D60FAE734
:107D7000580B030060220020442A002037B50A482F
:107D80000A4B42689C8819685388032503330570A1
:107D90009BB2002000909B0001EB8401044801F09D
:107DA00065FA03B030BD00BF282A00200C2B00204C
:107DB0006022002010B50146044800F0C8FE1C22D5
:107DC0000446002108F0B5FC204610BDF82A00202A
:107DD00068B10268084B9A4209D14068074B984243
:107DE00007D00133984214BF0320012070470320BD
:107DF00070470020704700BFDEC0ADDEFE011EF1FF
:107E00002DE9F0410D460223154F2B80164600F553
:107E1000805100F108044FF001088C420ED2236813
:107E200001330BD02046FFF703FF48B10EB186F8AF
:107E30000080022809D14FF480632B80BDE8F081D7
:107E4000A3683A68934200D93B602B886288033369
:107E500013442B806388033304EB8304DDE700BF06
:107E60003C2A002038B5144B14220D4602FB00308A
:107E70002B68446804F58051A3B15C88033403EB9C
:107E800084048C4215D22368013312D02046FFF7B8
:107E9000CFFE012808D002280BD00028F1D12C6099
:107EA000012038BD0834ECE76388033304EB830416
:107EB000E7E70020F5E700BF442A0020426873B5D9
:107EC00004460D466AB3234BD9688A4229D31B69FD
:107ED0009A4226D812F0030323D11F490089098949
:107EE00088421ED12068916888421AD11B48416897
:107EF0008A4203D901F580518A420DD381698A42B1
:107F00000CD901F580518A4208D201222A80B3FAA5
:107F100083F0400902B070BD1A46F7E748F20963E2
:107F2000F5E700262E800196288801A9FFF79AFF21
:107F300030B92B8801339BB2012B2B80F3D9E9E7B1
:107F4000019B226899689142EED16360024B1B89C4
:107F50002381DFE760220020282A0020442A002015
:107F60002DE9F8431C461D4B1B7806460F46154667
:107F700073B382B37CB3DFF86C804FF01409A3882D
:107F8000012B02D948F2096020E009FB03F318F83D
:107F900003302BB9A0882146FFF764FF20B9206089
:107FA000A3880133A380EAE723681EB19988328849
:107FB0009142EFD11FB119883A889142EAD19A686B
:107FC000C5E90023064B1B892B810020BDE8F883FF
:107FD00048F20160FAE748F20460F7E7202A00203F
:107FE000282A0020442A002008B5074B5888191D6C
:107FF000FFF738FF18B1BDE80840FFF7BFBEBDE886
:108000000840FFF75BBE00BF282A00202DE9F0479B
:108010009F4FDFF8A08288B006463B6823B99D4891
:10802000414600F0CEFD38603D6829784B1E052B97
:1080300007D8DFE813F02000740074000601060181
:108040005D0148F20E641422002103A808F071FBC0
:1080500041F61D539C4208BF00243B6804941A78E3
:10806000023A042A00F2FC81DFE812F0DD01E901A6
:108070000B0213021A022EB1874B00225A604FF4F2
:108080000644E0E72B79032B1CD8DFE803F0140249
:108090002A35824A1378022B1AD0137D022B4FF017
:1080A000010317D114214B43D1180020D054486844
:1080B000FFF738FE03E001232B71FFF71FFE0028B6
:1080C00000F0B980744B00225A6048F20D64BAE7A0
:1080D0000023E7E7704A13700023536041F61D54F4
:1080E000B1E76F496F48002302222B718A8009682B
:1080F000012201F055F9E2E76B4B684C5B88684A56
:1081000014214B43E11800262E714D68106815604C
:10811000958848600D810221E6549180C8E7B5F842
:1081200014A0AA7DDFF87491AEB1022AEB8806D9BB
:10813000142101FB0A91DA1C088902440A811422E5
:1081400002FB0A99C3F57F43B9F80A20FD331344B3
:10815000A9F80A3093E7142303FB0A9318895C6893
:1081600004EB8004062A69D8DFE802F0274E364483
:108170001D5A040041F61D54AA7DEB88022A06D937
:10818000142101FB0A91DA1C088902440A81142295
:1081900002FB0A99C3F57F43B9F80A20FD33134463
:1081A000A9F80A304FE74148414900234360AB69D1
:1081B0000360FFF783FE00285BD00223AB7500232A
:1081C00000930423EA182146364801F04FF80028AE
:1081D00031D048F20D64CFE72B69002B14BF032385
:1081E0000123AB750023009305F10C02042304F175
:1081F0000801E9E70123AB750022EB8800922A69A8
:108200009B0004F10C01DFE703290CBF05230623C3
:10821000AB7500230093042305F10802E118D3E7AE
:108220000623AB75224B1988204B5868FFF78AFD4F
:1082300004460028A0D108B0BDE8F08748F20E64DB
:108240009AE7002E7FF41BAF2B79012B34D0022B41
:108250003FF444AF002B7FF4F4AE02232B710DF1F9
:108260000A01EB68039303A8CDE90466FFF726FE35
:1082700010B948F20964E6E60498BDF80A1083884C
:10828000EB8003882B81FFF75DFD044629E000BFEA
:10829000402A0020F82A0020202A0020442A00201A
:1082A0000C2B002060220020282A0020042A002015
:1082B000182B0020382A0020DFF8009203AA4B4632
:1082C0003146A81DFFF74CFE044670B9B9F80410FA
:1082D0000498FFF737FD044648F209639C423FF4D7
:1082E000FDAE002C7FF4AFAEA5E7C9E90066F3E769
:1082F000002E7FF4C4AE6C4B1A7BBAB11E731A7891
:10830000013A062A3FF69DAE01A151F822F000BFC6
:10831000BB830200E1830200FF83020005840200A8
:10832000438002000B8402001D8402001A78072A91
:10833000E5D801A151F822F059830200FF82020022
:10834000FF8202007F83020093830200B783020052
:10835000B78302007B8302001A89544901321A81D3
:1083600000225A801A730A78B2FA82F252099A727B
:108370000A7DB2FA82F25209DA72012207E04C4910
:1083800058688A884088033202448A8002221A7020
:10839000B5E75C88454A4649142505FB0422086870
:1083A000546850608888108102200C608880002109
:1083B00011740622EBE70722E9E79A7A32B9DA7AF2
:1083C0008AB900221A705A805A6087E6374900221B
:1083D0009A72CA68002AF2D1097C0029EFD05A802B
:1083E000FFF702FE51E70022DA72304A116A0029D3
:1083F000E7D192F82420002AE3D00122EFE7FFF72B
:10840000BDFC42E7FFF75AFC3FE75A88274B14218F
:1084100001FB02335868FFF785FC36E700225A60FB
:10842000FFF76CFC31E701228DF80C201A89ADF8BA
:1084300018209A88DB68ADF81A20059310E0022214
:108440008DF80C201A89ADF818209A88ADF81A20FA
:10845000DA689B7D05929A1F534253418DF81C3078
:1084600003A8FFF7D5FB0026414612483E6000F006
:10847000D3FB1148012100F089FC00287FF4CDAD29
:10848000D9E603228DF80C20DA88ADF818201A8975
:10849000D0E704228DF80C20DB88ADF81830DFE738
:1084A00005238DF80C30DBE7282A0020442A002021
:1084B0000C2B0020F82A0020082B00201C2B002069
:1084C0004068FFF7A3BD000008B50548012100F092
:1084D00045FC18B9BDE80840FFF798BD08BD00BFCE
:1084E000082B00202DE9F3419846374B1B780646B0
:1084F0000D46002B5CD000295DD009884FF6FF7334
:1085000099425BD06B88002B58D06B689B0758D181
:108510004AB92F890DF102013846FFF79FFB30B1B0
:1085200002B0BDE8F08113885788ADF8023001A889
:10853000FFF740FC044660B9BDF80220234B14212C
:1085400001FB023358890338C01B588148F2076089
:10855000E6E780F8008000238375BDF8023083824F
:108560006B68036101211A4800F004FC2B88238109
:10857000B8F1030F6B88A38004BF0423A3754FF0E9
:10858000000508BF3368E06008BFA3611148E780B9
:10859000658101A900F005FB36B1E36833600E4B3D
:1085A00075601B89B5723381FFF78EFF0020B7E736
:1085B00048F20160B4E748F20460B1E748F20360B2
:1085C000AEE748F20260ABE7202A0020442A0020F0
:1085D0003C2A0020F82A0020282A002008B503465B
:1085E00007480268042A08D00168064A42F8213088
:1085F000012100F0BFFB002008BD48F20B60FBE743
:10860000142B0020102A00202DE9F04FDFF82082E3
:1086100089B01422002103A808F08BF898F80030E4
:1086200003F0FF0200923BB103A8FFF7F1FA002725
:10863000384609B0BDE8F08F08F1040000F0B2FB45
:108640000028F4D1009BDFF8ECA1D3F8F83F5C1CC4
:1086500008BF4FF010234FF0805208BF5B691169CB
:108660005269581C08BF02FB01F3CAF8103069496F
:10867000A3F5405300225046CAF80C3000F0C4FD68
:1086800007460028D4D11C2363496448DFF8A8B109
:108690008C2200F027FA0323B9463D4601933C465D
:1086A000DAF80C604E443046FFF792FB012867D0A1
:1086B000032817D000283DD159494FF0140C0CFB6A
:1086C00004FC01EB0C0201F80C0056600CF11002E6
:1086D0000CF1080C0A4430466144FFF791FB45F069
:1086E00002054AE03268531C02D04E4B9A4239D1FF
:1086F000321D06F580511068013033D104329142A9
:10870000F9D1DBF800203AB902220123CBF800604E
:10871000ABF8042000930BE014226243404B02208C
:1087200099189854404A4E60548001340881A4B28C
:1087300045F0010509F58059B9F5405FB0D1019BBD
:10874000012B98BF0025EDB2022D03D0062D36D0A7
:10875000002D3ED1002388F8003048F20A67C8F89F
:10876000043065E7019B2E495A1E93B214226243DE
:10877000881801934660032088540134A4B2D9E7D5
:10878000009B6BB1264B1422624399180220985427
:10879000DBF800204A60244A088154800134A4B2E6
:1087A00000222249CBF800603046FFF729FBBBF8D6
:1087B0000420022A0CBF042208221543BAE7012331
:1087C00088F8003003A80023C8F80430FFF720FA27
:1087D0002EE702A8FFF7EEFAC8B10123013D0370AE
:1087E0000A2D09D8DFE805F006080608070807087B
:1087F0000F110F000023037102A9084800F0D1F9FE
:10880000FFF762FE14E70323F5E70223F3E748F2DC
:1088100007670DE7580D03006C2A0020F82A002096
:10882000442A0020DEC0ADDE282A0020102B0020C4
:10883000202A0020602200200C2B002073B50D465A
:108840000446C8B1C1B10DF10601FFF737FBB0B165
:10885000BDF806300B486668142202FB03000121B4
:108860000C3000F087FA63682E600C336B600123D4
:10887000A372002002B070BD48F20460FAE748F22B
:108880000960F7E7442A002013B50446A8B10DF1AA
:108890000601FFF713FB98B1BDF806200B4B14211E
:1088A00001FB0233DA6872B1A27A62B1DA680020A1
:1088B000013ADA60A07202B010BD48F20460FAE733
:1088C00048F20960F7E748F20560F4E7442A00201F
:1088D00002230022FFF706BE18B103230022FFF790
:1088E00001BE48F204607047114B1B7813B5044673
:1088F000ABB14FF6FF73984214D001A8FFF75AFAB4
:1089000098B10523037001230371C48001A90948AC
:1089100000F047F9FFF7D8FD002002B010BD48F283
:108920000160FAE748F20360F7E748F20760F4E70E
:10893000202A0020F82A00200F4B1B7807B5A3B18E
:1089400001A8FFF737FA98B10623037001A90B4875
:1089500000F027F90A4B1A780AB101221A73FFF7BF
:10896000B3FD002003B05DF804FB48F20160F9E7B5
:1089700048F20760F6E700BF202A0020F82A00200E
:10898000282A002007B5ADF80600ADF804100DF157
:10899000060001A9FFF7E4FA03B05DF804FB07B590
:1089A0001346ADF806000A4600200DF10601FFF758
:1089B000D7FA03B05DF804FB07B51346ADF806001F
:1089C0000A460DF106000021FFF7CAFA03B05DF870
:1089D00004FB20B119B103680B600020704748F216
:1089E000046070472DE9F84F3C4B1B780446002B80
:1089F0006DD000286ED0DFF8E8901222002107F039
:108A000098FE032323804FF0000A4F4614264FF0B0
:108A10000108D9F80410B9F80AB0B9F808500846A6
:108A2000FFF7D6F9032808BF2388628804BF03F143
:108A3000FF33238006FB0A735D44DB6813446380C5
:108A400023899B446389A4F808B0ADB22B446381A9
:108A5000C5F58065A389ADB2AB4238BFA58101F1F0
:108A6000080501F58051A94229D92B68013326D088
:108A70002846FFF7DDF801280AD0022815D0002883
:108A8000F1D1A3880133A3800AE04FF0010AC0E7C7
:108A9000E3880133E380E3896A8803331344E38185
:108AA0006B88033305EB8305DDE7E38884F81080EA
:108AB0004D1BE189013301EBA501E380E18109F15F
:108AC0001409BAF1000FE0D00020BDE8F88F48F299
:108AD0000160FAE748F20460F7E700BF202A0020AF
:108AE000442A002010B561B1B2FBF3F403FB142457
:108AF000A4B244B9C0E9001484608281C3812046D5
:108B000010BD0E20FCE70920FAE782B050E8022FE2
:108B1000C188B2EB324F4FF0000317BF92B241EA67
:108B2000014142EA014104E04268B2EB324F08BF22
:108B3000012340E80212002AE8D18DF807309DF8A1
:108B40000730002B0CBF1120002002B0704737B552
:108B500050E8013F9DB2C48925448489A54228BFBD
:108B60002D1B0489A54202BFBFF32F8F002207E00F
:108B7000C5EA030540E80154002CE9D14FF0010299
:108B80008DF803200193019A0A609DF8031001F00B
:108B9000FF0321B1006810FA82F003B030BD18461F
:108BA000FBE70A884B889A4209D150E8012FC2EAB4
:108BB000024240E80123002BF7D10120704700203A
:108BC000704737B550E8023F1FFAA3F5C488A542A5
:108BD00002BFBFF32F8F00220DE0C4892544848992
:108BE000A54228BF2D1BC3EA054540E80254002CCE
:108BF000E8D14FF001028DF803200193019A0A6039
:108C00009DF8031001F0FF0321B1006800EB124052
:108C100003B030BD1846FBE70A884B889A4209D159
:108C200050E8022FC2EA224240E80223002BF7D18B
:108C3000012070470020704701F01F024B090121FD
:108C4000914000EB830000F065B84B0910B501F0CE
:108C50001F040121A14000EB830000F04FF8E04029
:108C600000F0010010BD01F01F0301229A404B09E2
:108C700000EB8300D14300F065B84B0901F01F0100
:108C800050F82300C84000F0010070472DE9F0477C
:108C90004F1E7F0980460E460137002558F82540B3
:108CA00008EB8509E44394FAA4F4B4FA84F44FEA97
:108CB000451A202C06D10135AF42EFD83446204664
:108CC000BDE8F0875444A642F5D921464046FFF757
:108CD000BCFF0028F3D0D9F80040E44394FAA4F490
:108CE000B4FA84F4E5E710B5034653E8000F0A46EA
:108CF00043E8002494F0000FF7D110BD10B50346EF
:108D000053E8000F40EA010243E8002494F0000F0A
:108D1000F6D110BD10B5034653E8002F42EA01001A
:108D200043E8000494F0000FF6D110BD10B50346DF
:108D300053E8000F00EA010243E8002494F0000F1A
:108D4000F6D110BD10B5034653E8002F02EA01002A
:108D500043E8000494F0000FF6D110BD10B50346AF
:108D600053E8000F00EB010243E8002494F0000FE9
:108D7000F6D110BD10B5034653E8002F02EB0100F9
:108D800043E8000494F0000FF6D110BD10B503467F
:108D900053E8002FA2EB010043E8000494F0000F19
:108DA000F6D110BD0121FFF7A9BF0121FFF7B2BF26
:108DB0000021FFF7BBBF10B590B1D0E901230168D6
:108DC0009B1ADBB20A60013BDBB2FF2B026802D1C7
:108DD0000020107110BD11684C1C14600B70F2E77C
:108DE0000E20F7E737B5054600240DF107008DF892
:108DF0000740FEF795FD2A686B68116899420ED905
:108E0000481E106011F8013CEC68298A01FB0344FC
:108E1000AB6811791B1ADBB2994238BF13719DF808
:108E20000700FEF7A1FD204603B030BD37B505466B
:108E300000230DF107000C468DF80730FEF770FD9A
:108E40002A681368591C1160E968641A298AB4FBFE
:108E5000F1F41C709DF80700FEF786FD03B030BDED
:108E6000826810B504462AB14369016800699847D1
:108E70000023A36010BD0EB403B5039921B104AB68
:108E800001AA019300F076F802B05DF804EB03B09C
:108E900070470A2938B504460D4602D10D21FFF767
:108EA000F8FFA3682268591CA160D554D4E90132A7
:108EB0009A4204D32046BDE83840FFF7D1BF38BD01
:108EC0002DE9F84F9846DDE90A43154682460F46DC
:108ED0000A464FF00109AA420FD2C14538BFC14628
:108EE00013F0010B01D16CB900240126B8F1010F78
:108EF0001BD908F1FF386E43F8E709F10109B2FB0D
:108F0000F5F2E8E79B070ED5B8F1000F0CBF30264D
:108F10002026A145E9D2013C31465046FFF7B9FF72
:108F2000002CF6D1E0E72026F3E7B7FBF6F39D42ED
:108F3000E1D9DFF83C80B7FBF6F3504618F8031090
:108F400006FB1377FFF7A5FF3346AB42B6FBF5F6FA
:108F5000F1D2BBF1000F02D00CB1A14501D3BDE8A5
:108F6000F88F20215046013CFFF793FFF4E700BF44
:108F70006C0B03002DE9F74F05461746884600297C
:108F800000F03E8118F8011B49B92B7B002B00F043
:108F90003781284603B0BDE8F04FFFF761BF2529B0
:108FA00040F0B780002698F800302D2B424608F19B
:108FB000010823D0302B24D02B2B25D000242A2BA2
:108FC00002F1010123D13B681A1D1B683A601C4461
:108FD0000A4613782E2B26D101324FF0000A104694
:108FE00010F8011BA1F1300CBCF1090F1DD80A23A8
:108FF00003FB0A13A3F1300A0246F0E746F001062C
:10900000D1E746F00206CEE746F00406CBE711F8BA
:10901000013CA3F130000928DBD80A2202FB04340A
:10902000303C0A46CBE74FF0000A12F8011B01F072
:10903000FB0068289046F8D0782909D86F290CD809
:10904000632962D022D8252963D0582900F088806E
:1090500098F80030002B95D197E770390829F7D898
:1090600001A353F821F000BFDB91020051900200F0
:109070005190020071910200519002004F91020044
:10908000519002005190020061910200642901D0C8
:109090006929DDD13A68D2F80090111D89EAE97298
:1090A0003960A2EBE9724FF0010B092A35DCD34598
:1090B00038BFD3462CB1B9F1000F01DB720700D5E0
:1090C000013CB30702D5BAF1000F03D0F00701D479
:1090D0004CBB0024B9F1000F2DDAC9F100092D2194
:1090E0002846FFF7D6FE06F00302022A04D1BAF1A1
:1090F000000F01D11CBB0024CDE9004653460A22D3
:1091000049462846FFF7DCFEA2E73B681A1D19789E
:109110003A602846FFF7BDFE9AE70A230BF1010BE0
:10912000B2FBF3F2C1E7A345D4D220212846013C8B
:10913000FFF7AFFECCE77107D5D52B21D0E7A345CC
:10914000DAD230212846013CFFF7A3FED2E7396886
:10915000CDE900460A1D3A6053460A220968D0E765
:1091600039680A1D3A60CDE9004653461022F5E7FA
:109170003B681A1D3A6016F00106D3F8009024D11E
:10918000B9F1000F03D0484607F006FB0646B4428B
:109190001DD809F1FF3919F8011F00293FF458AF14
:1091A0002846FFF776FEF6E728460136FFF771FE00
:1091B00019F806100029F7D1A642BFF449AF2021C3
:1091C0002846013CFFF765FEF6E70026F0E7202180
:1091D0002846013CFFF75DFED9E73B681A1D3A605F
:1091E000302128461C68FFF754FE78212846FFF7F7
:1091F00050FE00220823CDE900322146102280E7EC
:1092000003B0BDE8F08F00BF13B50B46114680B91F
:10921000104B1148114AC01A0E23C0080093104B7E
:109220000004104940F00100FDF725FC0E2002B0BB
:1092300010BD4BB9074B08480B4AC01AC0080E2393
:1092400000930004064BECE703601B6802B0BDE826
:10925000104018475C080300AC0803007C0B0300B7
:10926000380D0300810B0300B00B03002DE9F74319
:10927000DDF8288088B93E4B3E483F4AC01AC008F6
:109280000E243E4B009400043D4940F00100FDF7E0
:10929000F2FB204603B0BDE8F0834AB9344B3548B1
:1092A000384AC01AC0080E24344B00940004EBE77F
:1092B000D0F800E0BEF1000F09D12D4B2D48324A05
:1092C000C01AC00808242D4B00940004DCE74BB9F9
:1092D000274B28482D4AC01AC0080924274B009460
:1092E0000004D1E74568D5F80490B3FBF9F509FB14
:1092F00015354DB11E4B1F48254AC01AC008092418
:109300001E4B00940004BFE78D0709D0184B194885
:10931000204AC01AC0081024184B00940004B3E778
:1093200012F0030F09D0124B12481B4AC01AC00892
:109330001024124B00940004A6E7C568A9420DD37F
:109340004D1EEC180569AC4208D8CDF82880DEF82F
:109350000C40A44603B0BDE8F0436047044B054809
:109360000E4AC01AC0081024044B009400048BE776
:109370005C080300AC0803007C0B0300250D030010
:10938000810B0300FE0B0300AA0B0300BD0B0300BF
:10939000040C03002E0C0300460C0300690C0300B0
:1093A000F7B580B92A4B2B482B4AC01AC0080E24A7
:1093B0002A4B009400042A4940F00100FDF75BFBB2
:1093C000204603B0F0BDD0F800C0BCF1000F09D1B9
:1093D0001F4B2048234AC01AC00808241F4B009482
:1093E0000004E8E74AB91A4B1A481F4AC01AC008D5
:1093F00009241A4B00940004DDE74568D5F800E025
:109400000EF1FF350D4209D0114B1248174AC01A10
:10941000C0081024114B00940004CCE7C568A94291
:109420000CD34D1E0EFB02540569AC4206D8DCF885
:109430001040A44603B0BDE8F0406047044B054827
:109440000B4AC01AC0081024044B00940004B2E771
:109450005C080300AC0803007C0B0300120D030042
:10946000810B0300AA0B0300BD0B0300900C03004B
:10947000B60C030029DF704728DF704770B503681A
:109480009E6886B004460D466EB1142200216846DF
:1094900007F04FF9A3680593237901952BB1012BB0
:1094A0000DD06846B04706B070BD01238DF800307E
:1094B00023690293E368039363690493F1E702234A
:1094C0008DF80030E3681B030293F5E70846704708
:1094D00000207047024B187A003818BF01207047EF
:1094E000C02B0020034B187A0122B0FA80F05A7486
:1094F00040097047C02B002008B510461A4607F0F7
:10950000EFF8002008BD000008B51422002104482F
:1095100007F00FF90348FFF7F8FA002008BD00BF75
:10952000C02B0020B02B002010B5094C094B436024
:109530002046FFF737FC40B906F07AFE0649207452
:109540001C2306488C22FFF7CDFA002010BD00BF77
:10955000C02B00204C0D0300242B0020B02B00203A
:1095600038B5234D234C2B7A3BB923492348FFF7C9
:1095700028FB206008B9686038BD022324682B727C
:10958000237973B1012B24D020460321FFF776FF06
:1095900000232B726B6018491848BDE83840FFF76C
:1095A0003BBBD4E90523D21AB2F5805FD4E903109E
:1095B00028BF4FF480529208012A38BF0122194473
:1095C0001844FFF757FF50B11128DDD101232B724A
:1095D000D2E7D4E903031844FFF74EFFF3E72B7CEF
:1095E000002BC9D1BDE83840022000F009B800BF07
:1095F000C02B0020D82B0020D42B0020B02B002023
:1096000038B5234C237A002B41D0022B09D10328F3
:1096100030D0204B00221B68E2601A793AB1012A4F
:1096200022D0637C7BBBBDE83840FFF799BFD3E90C
:1096300005128D1AB5F5805F94BF521902F580525C
:109640009A619142EDD102284FF0000308BF1946FC
:109650002372104B18BF0D211868FFF70FFF0E493A
:109660000E48FFF7D9FADCE71A6901321A615B6923
:109670009A42E7E7E3680133082B01D8E360D0E7BB
:109680000023E360DFE7BDE8384006F0C1BD38BD28
:10969000C02B0020D82B0020D42B0020B02B002082
:1096A000831E012B01D8FFF7ABBF704700F0FD030D
:1096B000012B08D1044B00225A74421E50425041E3
:1096C0001874FFF74DBF7047C02B002010B5064C33
:1096D000201DFFF767FB28B9637C1BB9BDE810406C
:1096E000FFF73EBF10BD00BFC02B00202DE9F341A6
:1096F00080460D46104801A916461F46FFF727FA77
:109700000446B0B118220021043007F012F82D0BE6
:109710000123237101A90848C4F80080A760E5600F
:109720006661FFF73EFAFFF7D1FF002002B0BDE807
:10973000F0810420FAE700BFB02B00202DE9F341AF
:1097400080460F460F4801A916461D46FFF7FFF950
:109750000446A8B118220021043006F0EAFF089B55
:10976000A36001A9C4E903670648C4F800806561E5
:10977000FFF717FAFFF7AAFF002002B0BDE8F0815B
:109780000420FAE7B02B00202DE9F84FB0F806A02E
:109790004579D2F800B09DF828900AFB05F5043D04
:1097A00088460BEB0301A94203F1040488BFA5EB33
:1097B000030BB4FBFAF607460AFB1644C2F800B0E6
:1097C0004EB9AAEB04055D4528BF5D46BBF1000F0D
:1097D00004D1BDE8F88F3F68013EF1E7043408EB9F
:1097E00006003C442A46B9F1000F0DD02146ABEBF0
:1097F000050B06F075FFDA452E443F6855464FF0DD
:10980000000428BF5D46E1E701462046EFE7FFF789
:10981000D2BAF8B546790146721E05460023934236
:109820002D6803D30024A64202D8F8BD0133F6E721
:109830000F682846FFF7FAFA01343946F3E72DE9B5
:10984000F843068ACD1C0746FFF7CCFA043E3544A0
:109850000446B5FBF6F5F0B14FF48073EDB28380AA
:10986000C680013D076081464FF00008A84512D22E
:109870003846FFF7B7FA064648B16379013363719A
:1098800008F10108C9F8000007608146EEE72046AC
:10989000FFF7BFFF34462046BDE8F88301210430BE
:1098A000FFF768BA10B5012104460430FFF76EFADD
:1098B000C0B220B92046BDE81040FFF7AABF10BDD6
:1098C0001FB503920022009203AAFFF75DFF05B0C7
:1098D0005DF804FB1FB503920122009203AAFFF773
:1098E00053FF05B05DF804FB33DF704741DF70477D
:1098F0000D4A08B5002313700C4A1360BFF35F8F45
:109900000B490C4800F0AFF80B4A0C480121FDF759
:10991000BDFE024630B9BDE8084009484FF4804119
:10992000FDF7C6BE08BD00BFE52B0020E82B0020D8
:10993000880D0300DC2B0020419A0200840D0300F7
:10994000C022002007B500230DF107008DF8073075
:10995000FDF7E6FFF1EE103A23F09F03E1EE103A37
:10996000BFF35F8F0A4B4022C3F884219DF80700A4
:10997000FDF7FAFF06F05CFC20B103B05DF804EBE4
:10998000FFF7B4BF20BF40BF20BF03B05DF804FBAA
:1099900000E100E070B5244D044601212846FFF7A0
:1099A000A2F9BFF35F8F38B9042C0AD01F4B1A7885
:1099B0001AB1BFF35F8F286070BD1D4A1470012279
:1099C0001A701C4C1A4E6368BBB9FDF791F8FCF78E
:1099D000EFFE0028FBD1164B1B78023B012B15D85C
:1099E000BFF34F8F1449154BCA6802F4E06213436A
:1099F000CB60BFF34F8F00BFFDE71B6830789847FF
:109A00000028D6D0204600F038F8DCE706F010FC3D
:109A100008B1FFF769FF4FF080430122C3F800252A
:109A2000BFF34F8F20BFFDE7E82B0020E52B002080
:109A3000E42B0020DC2B002000ED00E00400FA0500
:109A4000034B1B7813B10420FFF7A4BF704700BF7E
:109A5000E52B0020836800225A60C3E904229A6043
:109A6000DA601A6070470B684A684360934208BF27
:109A70000023016008BF43607047436843B1026838
:109A8000916852680B449342436004BF00234360D3
:109A9000704770B5446806460D46206818B1B36833
:109AA0002946984718B923682B60256070BD246843
:109AB000F3E74368186808B102681A6070474368A2
:109AC000186870474368186800B97047884203D126
:109AD00002681A600120704703460068F4E700003E
:109AE00010B50D49A1F59472914201D800200FE004
:109AF0008C1AE30F03EBE4035B1002EBC30452F890
:109B00003330834205D802D204F10802ECE76068E2
:109B100010BD2146E8E700BF9412030008B5FFF727
:109B2000DFFF024B002808BF184608BD571103008D
:109B300038B5074C051E04F1080318BF1C462368FE
:109B40002BB11A6822605B6828469847F7E738BD52
:109B5000F42B002020B9054B01225A70FFF7E8BF13
:109B6000012802D1014A9070F8E77047EC2B0020E1
:109B700020B9034B01225A70FFF7DABF704700BFCC
:109B8000EC2B002038B50E4C2378B3B90D48636038
:109B9000A3602361E36000F0E7F8054606F048FBA8
:109BA00008B900F0EDF801232370074BD3F8003417
:109BB0000BB10123A370284638BD8525F5E700BF0A
:109BC000EC2B0020559B02000000014037B50D4CE6
:109BD00000230DF107008DF80730FDF7A1FEE368C3
:109BE000013BE360E36833B9074BD3F8005415B980
:109BF00000F0D8F8A5709DF80700FDF7B5FE03B09A
:109C000030BD00BFEC2B002000000140012813B53F
:109C10000CD0032820D038B9134B0122C3F8802080
:109C2000BFF34F8FBFF36F8F02B010BD0F4C0023F7
:109C30000DF107008DF80730FDF772FE23780BB9A0
:109C4000FFF7A0FFE3689DF807000133E3600123FD
:109C5000A370FDF789FEE7E700F092F802B0BDE8D7
:109C60001040FFF7B3BF00BF00E100E0EC2B002085
:109C70001FB503788DF800304368019383688DF831
:109C80000830C368054A0393054B684653F82130F2
:109C900052F82110984705B05DF804FB002C002015
:109CA000042C00201FB503788DF800304368019321
:109CB00083688DF80830C368054A0393054B6846EE
:109CC00053F8213052F82110984705B05DF804FB95
:109CD000002C0020042C0020F0B5194B90F800C097
:109CE00091F81DE043F82C20164B16460A6943F8FC
:109CF0002C20154B03F80CE00C4607460FCC89B01E
:109D00006D460FC594E80F0085E80F00CDF810C030
:109D1000BEF1000F09D0002E0C4A694608BF32463A
:109D2000381D00F083FD09B0F0BD002E084A6946D9
:109D300008BF324607F10C0000F05AFBF3E700BF02
:109D4000042C0020002C0020082C0020719C020014
:109D5000A59C020000F18040002382B003600368EC
:109D60000193019B02B07047044A137923B9012182
:109D70001060918018467047852070470C2C002099
:109D8000074B1A68D20704D4C02283F800230122AB
:109D90001A604FF080430122C3F81825704700BFB6
:109DA00000E100E04FF0804208B50223C2F808331A
:109DB0004FF48270FFF7CEFF0123D360D2F818343E
:109DC000DB03FBD408BD00004FF0804110B5D1F893
:109DD000003163B14FF48070FFF7BCFF0D4B587931
:109DE0000122C1F8082310B95A711B6898474FF037
:109DF0008042D2F8043163B14FF48270FFF7AAFFBA
:109E00000223C2F80833034BBDE810401B68012051
:109E1000184710BD0C2C002000F1804000F5C04018
:109E2000002382B0036003680193019B02B0704776
:109E3000800000F1A040D0F8002722F44032C0F8A2
:109E40000027D0F8003743EA0141C0F800177047F7
:109E5000054B4FF0FF32072843F8202084BFC0187D
:109E600080F84820704700BF142C002010B5184916
:109E700091F8583053BB4FF0FF3222FA03F0C0077D
:109E800048BFC81803F1010348BF80F83020202BD9
:109E9000F3D10024E0B20134FFF7DAFF0C2CF9D142
:109EA0000C4B0022C0204A6583F80603402018604E
:109EB0004FF4BE70FFF7B0FF074B4FF00040C3F800
:109EC0000403012381F85830104610BD0820FCE738
:109ED000142C002000E100E000600040034B93F8E8
:109EE0005800003818BF0120704700BF142C002014
:109EF000F0B5394E331893F93030002B69DA8D788C
:109F0000C5F34005002D0BBF082300230C240824B3
:109F1000A34201D10420F0BD56F82370013743D18C
:109F200037185CB246F8232087F8304015B9F2188C
:109F300082F848008A78550716D4D70736D58200AC
:109F400002F1A042D2F8005725F00205C2F80057EE
:109F5000224FC50800F0070C012202FA0CF217F894
:109F600005C042EA0C027A558A780D7812F0020296
:109F700025D09B0003F1804303F5C0430002D3F8D2
:109F8000102522F4473222F44072C3F810252D0424
:109F9000D3F8102500F4F85005F440352843104359
:109FA000C3F810050020B6E70133B1E74D7800F59E
:109FB000E0724FF0A047AD0047F82250C8E7083CD8
:109FC00046FA84F494F8500040EA851584F850501D
:109FD000E8E708209FE700BF142C0020682C002031
:109FE00038B5204C251895F93020072A18DD083A95
:109FF00044FA82F494F850309B09032B0BD14FF0B4
:10A00000A043D3F81015C14001F001010231BDE8B1
:10A010003840FFF70DBF012B0CBF02210321F6E7EB
:10A02000D3B2072B1DD8930003F1804303F5C0433F
:10A03000D3F8100540F00100C3F8100502F140000C
:10A0400040B2800080B2FFF7E7FE51B195F93030A1
:10A0500054F823302BB1012303FA02F2024BC3F868
:10A06000042338BD142C0020006000404FF0A043B2
:10A07000D3F8103523FA00F000F00100704700001B
:10A080002DE9F74F00244E4D01944FF480720121C9
:10A0900002F1804303F5C04390B21B68012B06D147
:10A0A000D5F804330B4202D0FFF7B6FE0C4304325E
:10A0B000B2F5907F4FEA4101EAD1414BD3F87C31B0
:10A0C000012B0CD14FF4BE70FFF7A6FE4FF0A0435A
:10A0D00044F00044D3F820250192C3F82025E3B2D0
:10A0E000D3B1384F00250126344210D0AB0003F124
:10A0F000804303F5C043D3F81005D3F8101557F883
:10A10000253023B1C1F30141C0F304209847013544
:10A11000082D4FEA4606E7D1002C48DA294D4FF0CA
:10A12000A048294E4FF00009012716F9013B5A1C9F
:10A1300031D0C3F3C20208326A44DCB212F8042CF4
:10A1400003F03F0A03F0070307FA03F31A4222D091
:10A150000AF5E073504658F82330C3F3014BBBF1C6
:10A16000020F0CBF03210221FFF762FE07FA0AF378
:10A17000C8F8203505EB0A0393F9303055F8233041
:10A180004BB1A109032904D0BBF1020F12D101295F
:10A1900001D15046984709F10109B9F1040FC4D122
:10A1A000D8F820350193C8F82035002BB9D103B079
:10A1B000BDE8F08FBBF1030FEDD10229E8E700BF46
:10A1C00000600040142C0020642C0020014B1B6810
:10A1D000184700BF702C00200E4B984237B50C4634
:10A1E00002D0002003B030BD00230DF107008DF830
:10A1F0000730FDF795FB084B1D7915B901221C604E
:10A200001A719DF80700FDF7AFFB002DE9D0112072
:10A21000E8E700BF00200040702C0020034B98426C
:10A2200001BF034B00221A601A71704700200040E2
:10A23000702C00200023435082B043580193019BAF
:10A2400002B070470A4610B54FF48E71FFF7F2FF67
:10A25000136A9168C95C136A01331362C0F81C1554
:10A2600010BD8B690A4610B54FF4847123B9FFF70E
:10A27000E1FFD0F8183510BDFFF7DCFF536AD16855
:10A28000D0F81805C854536A01335362F3E700004D
:10A290001FB501238DF80030044BCDE90110D3E93F
:10A2A00000126846904705B05DF804FB782C00204A
:10A2B00030B54D4DD5F804339A0585B051D5D5F854
:10A2C0002431002B4DD04FF492712846FFF7B2FF96
:10A2D0004FF40173C5F80833444B93F829200AB9A9
:10A2E00001226A60404902228DF80020D1F88024C2
:10A2F000C1F8802403929A690292DA6801920022DE
:10A30000C3E906226846D3E9001290473648D0F8E0
:10A310001C315BB1354A5169136A99424DD992F8A3
:10A320002830002B49D11146FFF78CFF2E48D0F87A
:10A330004431002B56D04FF4A271FFF77BFF2B4B1B
:10A3400093F829200AB1012202609A69002A49D0B3
:10A35000586AD96800229A6105B0BDE83040FFF71D
:10A3600097BFD5F804335B07D0D5D5F80831002B5B
:10A37000CCD01E4C1C482146FFF773FF636AA269CC
:10A380009A42C3D1E369E1684BB1A3612369E360F9
:10A390000023606AE3616362FFF77AFFB6E794F82F
:10A3A00029300BB901236B600F4B4FF40172C3F8D6
:10A3B00008230023606AA361EEE70B484FF48E7117
:10A3C000FFF738FF5369002BB0D051690291002389
:10A3D00091688DF80030019153616846D2E900130D
:10A3E0009847A3E705B030BD00200040782C00203E
:10A3F0002DE9F843534D90F804802C2303FB0853B8
:10A40000064693F82A300C469146002B40F0968081
:10A410004D490068FFF7E0FE0746002840F09080B5
:10A4200022683068511C0BD04FF0A04101239340AB
:10A43000C1F8083502F5E0734FF0030C41F823C072
:10A4400061684B1C1FBF01F5E0734FF0A04C4FF04B
:10A45000000E4CF823E0A369C0F8243594F814C02A
:10A46000637DBCF1010F4CEA0303C0F86C35C0F802
:10A470001415C0F80C251DD1A268531C1FBF02F58E
:10A48000E0734FF0A0414FF0000C41F823C0E368A7
:10A49000591C0BD04FF0A04C01219940CCF8081565
:10A4A00003F5E0714FF0030E4CF821E0C0F80835D9
:10A4B000C0F810252C2202FB08F2AB18C3F8049058
:10A4C0002369AB50B9F1000F20D04FF48E71247F77
:10A4D000FFF7B0FE4FF4A2713068FFF7ABFE3268B1
:10A4E0001A4BC2F80433130B42F307326101002AFE
:10A4F000C9B21EDB1648841884F8001301215209E2
:10A5000003F01F0301FA03F340F8223033680422FA
:10A51000C3F800252C2303FB08530022C3E90622BD
:10A5200083F829205A61012283F82A203846BDE8A1
:10A53000F883084A03F00F03D154E7E70827F5E74B
:10A540001127F3E7782C0020B1A20200800002005E
:10A5500000E100E014ED00E0F8B503680579304C47
:10A560000022C3F800252C2202FB05425268A2B14A
:10A570002C4AC3F808231A0B43F30733002B0CDBD8
:10A5800002F01F015B0901228A402033264941F86D
:10A590002320BFF34F8FBFF36F8F0068D0F80C6597
:10A5A000D0F81415D0F80835D0F810254FF0FF3743
:10A5B000BE42C0F8147518BF06F5E076C0F80C75F9
:10A5C000C0F80875C0F810751EBF4FF0A0474FF0D7
:10A5D000020C47F826C04E1C1FBF4FF0A04601F5E5
:10A5E000E071022746F82170511C1FBF4FF0A041B7
:10A5F00002F5E072022641F822605A1C1FBF03F5E3
:10A60000E0734FF0A042022142F82310FFF706FE4C
:10A610002C2303FB0544002384F82A306360F8BD33
:10A62000782C00208402020000E100E00279044B53
:10A630002C2101FB02335869003818BF01207047F4
:10A64000782C00202DE9F84F064690F804808946C2
:10A650009246FFF7EBFF044600283CD1204F2C2503
:10A6600008FB057B4FF48E71CBF814A0CBF8089053
:10A67000CBF820008BF828003068FFF7DBFD30684E
:10A68000012383605946FFF7DDFDDBF804305D46AA
:10A690001BBB3068DBF814402B6A9C4211D833682E
:10A6A000D3F81C21002AFBD00122DA6000202C23E1
:10A6B00003FB087700237B61BDE8F88F95F828300D
:10A6C0003BB9D0F81C31002BF8D05946FFF7BAFD42
:10A6D000E2E70F20EBE71120EEE72046ECE700BFB2
:10A6E000782C00200023435082B043580193019BF3
:10A6F00002B070471FB501238DF80030044BCDE93F
:10A700000110D3E900126846904705B05DF804FBDC
:10A71000A42C00207FB5434AD2F82461002E60D0DB
:10A7200010464FF49271FFF7DDFF02238DF80030E1
:10A73000D2F88034C2F880340393D2F83C350293C7
:10A74000394BDA6801920022C3E906226846D3E950
:10A75000001290473348D0F8443173B14FF4A271DE
:10A76000FFF7C0FF304B9A693AB10022C3E90622D5
:10A77000D968D0F83C05FFF7BDFF2A48D0F8203152
:10A78000ABB14FF49071FFF7ADFF0123C360264BCF
:10A790005A6962B1D0F84C150291002299688DF87F
:10A7A000002001915A616846D3E9001290471D4884
:10A7B000D0F858319BB14FF4AC71FFF793FF1A4BAF
:10A7C0005A6962B1D0F84C150291002299688DF84F
:10A7D000002001915A616846D3E90012904704B005
:10A7E00070BDD2F81031002BB4D04FF488711046F0
:10A7F000FFF778FF0C4BD2F83C0599698842A9D144
:10A80000DC69D96864B1D2F8005225F02005C2F89D
:10A8100000521A699C61DA60DE61FFF76BFF99E70D
:10A820009C61FAE700200040A42C00202DE9F843A9
:10A830005A4E90F80480242303FB0863044693F8DF
:10A8400020300D469146002B40F0A380544900680B
:10A85000FFF7C2FC0746002840F09D802A68206868
:10A86000511C0BD04FF0A04101239340C1F8083593
:10A8700002F5E0734FF0030C41F823C069684B1CEC
:10A880001FBF01F5E0734FF0A04C4FF0000E4CF8E5
:10A8900023E0AB69C0F8243595F814C06B7DBCF19A
:10A8A000010F4CEA0303C0F86C35C0F80C25C0F862
:10A8B00014151DD1AA68531C1FBF02F5E0734FF099
:10A8C000A0414FF0000C41F823C0EB68591C0BD09D
:10A8D0004FF0A04C01219940CCF8081503F5E07128
:10A8E0004FF0030E4CF821E0C0F80835C0F81025F1
:10A8F000242202FB08F2B318C3F804902B69B3506A
:10A90000B9F1000F2FD04FF488712A7FFFF7EAFECC
:10A9100020684FF49071FFF7E5FE20684FF49271C4
:10A92000FFF7E0FE20684FF4A271FFF7DBFE4FF463
:10A93000AC712068FFF7D6FE23681A49C3F80413E8
:10A94000190B43F307335201002BD2B21CDB16481C
:10A95000C51885F8002301225B0901F01F0102FAE6
:10A9600001F140F8231023680822C3F800252423AE
:10A9700003FB08660023C6E906337361012386F8EA
:10A9800020303846BDE8F883084B01F00F015A54D7
:10A99000E9E70827F5E71127F3E700BFA42C00201B
:10A9A00015A702001003420000E100E014ED00E0F2
:10A9B000F8B5444C0579242303FB054302465B6844
:10A9C0000068ABB1404BC0F8083340F30733002BAD
:10A9D0004FEA10310CDB01F01F065B090121B14089
:10A9E00020333A4E46F82310BFF34F8FBFF36F8FDB
:10A9F000D0F8003223F02003C0F80032242303FBF8
:10AA000005439B692BB14FF4A271FFF76BFE012345
:10AA100043604FF4AC71FFF765FE0123C36024234C
:10AA200003FB0543D0F858110029FBD0996919B1EF
:10AA3000D0F844110029F5D00023C0F80035136880
:10AA4000D3F80C75D3F81465D3F80825D3F810158E
:10AA50004FF0FF3C6745C3F80CC518BF07F5E0771A
:10AA6000C3F814C5C3F808C5C3F810C51EBF4FF01E
:10AA7000A0434FF0020C43F827C0771C1FBF4FF0D4
:10AA8000A04306F5E076022743F826704E1C1FBF50
:10AA900001F5E0714FF0A043022643F82160531CFA
:10AAA0001FBF4FF0A04302F5E072022143F82210CD
:10AAB000FFF7B4FB242303FB0544002384F8203074
:10AAC0006360F8BDA42C00201003420000E100E008
:10AAD0000279044B242101FB02335869003818BF66
:10AAE00001207047A42C002001F06043B3F1005F07
:10AAF0002DE9F0470646884692463BD190F80490EF
:10AB0000FFF7E6FF0446002836D11D4F30682425A4
:10AB100005FB09754FF49071C5F814A0C5F80880BD
:10AB2000FFF7E0FD4FF4AC713068FFF7DBFD3368F1
:10AB30006A69A968C3F84415C3F8482501229A60D8
:10AB40006A68DAB9D3F82021D3F858011AB9002875
:10AB5000F8D00F2007E00028FBD10122DA60D3F8FB
:10AB60005821002AFBD0242303FB097700237B61B3
:10AB7000BDE8F0871020FBE71120F9E72046F7E752
:10AB8000A42C00200220FCF72FB900002DE9F0478B
:10AB900080460D46FCF748F90328044610D8012DDD
:10ABA00010D0022D30D05DB91A48FCF7AFFD1A4B1A
:10ABB00004EB440213449D78184B1B5DAB4219D043
:10ABC000BDE8F087144E00EB4003F218F55C5378B3
:10ABD000470053B1DFF84C900E484A464FF480418D
:10ABE000FCF766FD08B989F8008027443E440B4B0A
:10ABF000B2781A55002DE3D0094B1B68002BDFD02B
:10AC00002846BDE8F047184700EB400402480444DA
:10AC10006578EFE700230020CA2C0020E52C0020F7
:10AC2000E02C0020C82C002000780221FFF7AEBFE6
:10AC300008B5094B1B7853B10020FCF7ABF8012095
:10AC4000FCF7A8F8BDE808400320FCF7A3B8BDE86E
:10AC50000840FCF7ABB800BFC92C0020F8B57A4C0F
:10AC6000237805461BB100232370FFF7E1FF172D62
:10AC700000F28780DFE805F00C1717425364757FF8
:10AC8000878C878C949999999999C3C8D0D8E3E314
:10AC9000FFF7CEFF6D48FCF739FD6D4B00220446EF
:10ACA0001A702046F8BD0020FCF75AF8F0B10020D9
:10ACB000FCF770F8022D0CBF4FF4E1644FF47A6496
:10ACC000634B1D7000254FF400464FF47A702946FF
:10ACD0004FF4FA620023E4FB060105F009FC2A4662
:10ACE0000146BDE8F8405948FCF7E2BCFCF746F8DD
:10ACF000022D0CBFC8244FF4C874E1E70020FCF714
:10AD00002FF840B10020FCF745F84FF44874504B41
:10AD100003221A70D6E7FCF731F8C824F7E70020C1
:10AD2000FCF71EF838B10020FCF734F84FF47A64D1
:10AD3000474B0422EDE7FCF721F84FF4C874F7E71E
:10AD40000020FCF70DF848B10020FCF723F8404B39
:10AD500005221A7040F6CD410022C2E7FCF70EF83A
:10AD6000F5E70020FCF740F8394B06221A70002264
:10AD700040F26661B5E70020FCF700F8344B07228B
:10AD80001A7000248DE701202070FCF72DF8EEE703
:10AD900001202070FCF728F800224FF40051A0E7B2
:10ADA000FCF713F82A4B0C22EAE72A482A4EFCF754
:10ADB000ADFCD5F1110504461CD0D8B9012D13D036
:10ADC000C820454321464FF400474FF47A704FF4B2
:10ADD000FA620023C5FB070105F08AFB2246014603
:10ADE0001C48FCF765FC04460220FBF7C7FF012363
:10ADF000337056E70220FBF7CDFF0023F8E7FFF79B
:10AE000017FF134B1222BBE7FFF712FF0020FBF7DF
:10AE1000B5FF0F4B1322B3E7FFF70AFF0120FBF743
:10AE2000ADFF0B4B1422ABE7FFF702FF0020FBF74F
:10AE3000A5FF0120FBF7A2FF054B1522A0E7FBF7BA
:10AE4000C4FF034B1D709CE7DC2C00202023002056
:10AE5000E42C0020E0220020C92C0020044B1B68B9
:10AE6000DB0703D5034B1878FFF7F8BE704700BF28
:10AE7000D82C0020E42C002010B5002914BF032496
:10AE80000024FBF7E3FF800000F1A040D0F800278A
:10AE900022F44032C0F80027D0F8003743EA0443D8
:10AEA000C0F80037002010BD032801D8FBF7AEBF63
:10AEB00000207047044B1B6813F0010301D0FFF71B
:10AEC000CDBE1846704700BFD82C002038B51C4BAB
:10AED00018601C4B10F00204054619601AD01A4B7A
:10AEE0001A480E221A700F22DA7010229A7111225B
:10AEF0005A72042140F23332FCF748FA044648B94A
:10AF0000FCF79CFA044628B90146114A1148FCF79F
:10AF1000BDFB0446EB0711D50120FBF79DFF6CB983
:10AF200021460D4A0D48FCF7B1FB044630B9BDE897
:10AF300038400B4A0B480121FCF7A8BB204638BD1E
:10AF4000D82C0020E02C0020CA2C0020B8120300CE
:10AF500029AC0200DC1203005DAE0200E012030027
:10AF600085AB0200D8120300032811D8012A0AD1A8
:10AF700001290FD100F10E02D2B20D4B00EB4000BF
:10AF80001A54002070470129F7D0022904D049B192
:10AF9000072070470022F8E7054B00EB40001844FB
:10AFA0004270EEE7024B00EB400018448270E8E785
:10AFB000CA2C0020032802D80121FFF75DBF06201C
:10AFC000704708B5012202210020FFF7CDFF08B12C
:10AFD000072810D1072202210120FFF7C5FF08B181
:10AFE000072808D100210A220846FFF7BDFF10B14B
:10AFF000072808BF002008BD0388102B10B502D019
:10B00000112B1ED010BD1A4C2168B1B9012208467F
:10B01000FFF7AAFF08B1072824D107220221012047
:10B02000FFF7A2FF08B107281CD10422022100204B
:10B03000FFF79AFF08B1072814D123680133236072
:10B04000E0E70B4A1368013B1360002BDAD1FFF7EE
:10B05000B8FF0028D6D0074B1B68002BD2D0BDE824
:10B0600010401847034B1B68002BE6D09847E4E7D5
:10B07000F02C0020EC2C002008B50020FFF79AFFF0
:10B0800008B1062806D10120FFF794FF10B1062869
:10B0900008BF002008BD00000D4B10B518600C461D
:10B0A00029B10120FFF700FF40B102232370094BB3
:10B0B0001B6853B9BDE81040FFF783BFFFF7F4FEEC
:10B0C00008B10B23F2E72070F1E7002010BD00BFAC
:10B0D000EC2C0020F02C002076DF70477ADF7047E0
:10B0E0007CDF70478FDF7047FCF7BEB903883B2BCE
:10B0F00013B5044608D005D8102B0AD0212B1BD03D
:10B1000002B010BD562BFBD1A0881321FFF7E4FF3E
:10B110000BE00720FFF7CEFE08B1FCF7A5F90D4BB9
:10B12000A1880D48198002F01FFB0028E8D002B06A
:10B13000BDE81040FCF798B9002380888DF80430F2
:10B1400001A98DF80530FFF7CDFF0028D8D0FCF716
:10B150008BF9D5E7442300203C31002010B504468C
:10B1600003F084FE204603F0A5FE2046BDE8104013
:10B1700003F038BC10B5204B204A9B1ADB088CB07A
:10B180001B04032836D8DFE800F002272F3343F0F2
:10B19000030420461A49FBF757FC2C22002101A882
:10B1A00005F0C7FA44F250624FF496710123CDE9DD
:10B1B000051214488DF8083001A98DF8043000F00C
:10B1C000BEFE0021104801F05FF9104902462046FA
:10B1D000FBF73EFC0CB010BD0D4943F003000CB072
:10B1E000BDE81040FBF730BC0A4943F00100F6E728
:10B1F0000949FAE70949F8E7840803005C080300F5
:10B20000E4120300F42C002021B202001213030008
:10B21000291303004C13030085130300B21303002A
:10B2200013B513210190FFF757FF019A034660B150
:10B230000748084C0849241AE408240444F0020092
:10B2400002B0BDE81040FBF70CBC02B010BD00BF5F
:10B250005C08030084080300D9130300022807B523
:10B260000ED1094B09480A49C01AC008000440F031
:10B2700003000190FBF7E8FB06490198FBF7E4FBAC
:10B28000012003B05DF804FB5C08030084080300A0
:10B290001A14030047140300032807D14FF080431A
:10B2A000A922C3F820250020FEF774BB70470000D8
:10B2B00008B503784BB9054B3B211888FFF70CFF05
:10B2C00018B1BDE80840FCF7CFB808BD4423002002
:10B2D000072808B51FD00A280AD0042807D1134B25
:10B2E00013211888FFF7F8FE30F008030FD108BDCE
:10B2F0000020FFF7DFFD08B1FCF7B6F8FFF7BCFE52
:10B3000008B1FCF7B1F804F053FF0028EFD0BDE816
:10B310000840FCF7A9B8054B1A884FF6FF739A420C
:10B32000E5D1034800F0EDFDDEE700BF4423002037
:10B33000F42C002008B50548032100F0A3FC18B147
:10B34000BDE80840FCF790B808BD00BFF42C002011
:10B3500008B548B103280BD10220FFF7ABFD38B187
:10B36000BDE80840FCF780B8BDE80840FFF7E2BF41
:10B3700008BDFCF779B8000030B54FF48041AFB09C
:10B380000020FBF7C3F908B1FCF76EF8FBF7FCF8F7
:10B3900004F0CEFD08B1FCF767F8FCF745F908B1F9
:10B3A000FCF762F8FEF7A4FA08B1FCF75DF86F4904
:10B3B0000320FFF78BFD08B1FCF756F803A9002026
:10B3C000FFF76AFE08B1FCF74FF89DF80C5004F047
:10B3D000B1FE08B1FCF748F8002303A9012003934C
:10B3E00004F074FF08B1FCF73FF803A805F012F869
:10B3F00008B1FCF739F802F0B5FF08B1FCF734F8F2
:10B4000031238DF80C3007238DF80D3010238DF883
:10B410000E3003A803238DF80F308DF8103003F0A1
:10B4200041F808B1FCF720F8514803F023F808B1BF
:10B43000FCF71AF8082211234E498DF808300DEB5D
:10B440000200FFF74DFE08B1FCF70EF80023ADF83F
:10B4500010301823ADF80C305023ADF80E3003A88F
:10B460004FF4C873ADF81230FFF738FE08B1FBF7A0
:10B47000FBFF4148002102F065F808B1FBF7F4FF3B
:10B48000AC22002103A805F054F902238DF80C30FA
:10B4900040F20163ADF80E300124384B08930021CF
:10B4A0002C2221A8ADF81C4005F043F94FF4967109
:10B4B00044F25063CDE925133148324B8DF8884072
:10B4C00003A92C9300F061FB08B1FBF7CDFF2C48DA
:10B4D000012100F057FB002303932B482B4B0293D1
:10B4E00002A902F02FF908B1FBF7BEFF284B039326
:10B4F00003A804F0A1FC08B1FBF7B6FF1422002159
:10B5000003A805F016F94FF4F0234FF4A032CDE96B
:10B51000042303238DF818301E4B089303A81E4BF9
:10B52000099300F019FE08B1FBF79EFF1B4B1C4866
:10B530001C49C01AC008000440F003000190FBF74A
:10B5400083FA022D0FD118490198FBF77DFA02F01A
:10B55000D5FF08B1FBF788FFFBF72AF90028FBD1DC
:10B56000FEF7F0F9F8E7FFF7E5FEF5E7D1B20200E4
:10B570005DB1020076140300283100204023002032
:10B58000F42C002051B302003C310020E9B002004D
:10B5900075B10200B1B2020073B302005C0803008F
:10B5A000840803007F140300A314030013DF704713
:10B5B00038B50023134CD3F8F85F134BE41AE408B2
:10B5C0006A1C4FEA044404D14FF010235D696B1CE0
:10B5D00011D02A460D4944F00300FBF739FA2846FA
:10B5E000FFF7E4FF054620B1094944F00100FBF7ED
:10B5F0002BFA284638BD074944F00100FBF724FA2E
:10B600000425F6E7840803005C080300B014030077
:10B61000DB1403000E15030038B50B4B0B4C0C4A22
:10B620000C49E41AE408240444F00300FBF710FA80
:10B630000748FFF7BBFF054620B1074944F001006A
:10B64000FBF702FA284638BD5C08030084080300B3
:10B650000060020026150300DB1403006DDF704755
:10B6600079DF70477DDF704764DF70472DE9F04F69
:10B6700085B000250E9CBDF83CB0B4F800A0019147
:10B68000074690461E46A9463A884A450DDC45B114
:10B690002388013BA3EB0A039BB2FF2B3AD806F8A1
:10B6A0000A30002005B0BDE8F08F7A6852F8290012
:10B6B000039000220DF10B0103A8FFF7D5FF00282E
:10B6C000F0D19DF80B20424521D12288002D14BFD6
:10B6D0000020022002EB0801014459451ADC3DB963
:10B6E000013292B2019B2280B3542288013222801F
:10B6F00022880DF10B01324403A8FFF7B5FF0028A3
:10B70000D0D121889DF80B200A442280012509F11F
:10B710000109B9E70C20C5E72DE9F341089FBDF801
:10B7200024801546CDE90078022204461E46FFF724
:10B730009DFF50B93346102229462046CDE90878AE
:10B7400002B0BDE8F041FFF791BF02B0BDE8F08163
:10B750002DE9F04F00231788138090F82D3085B025
:10B7600006460D4614465BB3082F01D80C2028E18D
:10B7700002A8FFF773FF002840F023812388DDF83B
:10B7800009100822EA54238801339BB21B2223802C
:10B79000EA54238801339BB2EA182380E950BDF8AC
:10B7A0000D30938023889DF8082006339BB212F059
:10B7B000FE0218BF01222380EA542388013323802C
:10B7C000B378FBB123880433BB42CFD802A8FFF77C
:10B7D00047FF002840F0F58023880322EA5423889D
:10B7E00001339BB219222380EA542388BDF8082034
:10B7F00001339BB2E9182380EA54120A4A70238865
:10B8000002332380F2789AB12388D91CB942ADD88B
:10B810000221E954238801339BB201212380E9549A
:10B8200023880B449BB22380EA5423880B44238053
:10B830007268AAB12388D91CB94297D8022192F91B
:10B840000020E954238801339BB20A212380E95464
:10B85000238801339BB22380EA5423880133238059
:10B860003389002B40F0A180338A5BB1CDE90047DA
:10B870002B460722032106F11000FFF74DFF002899
:10B8800040F09F80338B5BB1CDE900472B461522FA
:10B89000142106F11800FFF73FFF002840F09180C7
:10B8A000326A002A40F09080D6F82480B8F1000F68
:10B8B00030D0B8F804302188981C8A1C0244BA425F
:10B8C0003FF654AFFE283FF651AF03336B54238845
:10B8D00001339BB2FF222380EA54238801339BB2B9
:10B8E0002380B8F80020EA54E918120A4A70208828
:10B8F000023080B22080B8F804205AB1D8F808107D
:10B9000000296BD0284404F0EBFE2388B8F804200B
:10B910001344238096F82C30002B40F09880307828
:10B9200000284ED03388012B58D0228802F1020C17
:10B93000BC453FF61BAF012805D173780233134491
:10B940009F42FFF413AF023FBF1ABFB202A905EB3B
:10B950000C00ADF80870FFF785FE90BB3178BDF89C
:10B960000830022900F0B98072789A4202D39F42CF
:10B9700080F0B180012940F0B280974293B2C0F0CC
:10B98000AE80ADF808300821BDF80830FE2B3FF638
:10B99000EDAE22880133AB542288013292B222806C
:10B9A000A9542288134423800BE0CDE900472B469D
:10B9B0000622022106F10800FFF7AEFE00283FF440
:10B9C00053AF05B0BDE8F08FB4F800C00CF106032A
:10B9D000BB423FF6CBAE1188052901D80720F0E71E
:10B9E0006FF4486E01EB0E039BB24FF27D3E734540
:10B9F000F4D95388052BF1D96FF44860181880B238
:10BA00007045EBD94FF6FF70814201D09942E5D8DD
:10BA1000052305F80C30238801339BB212212380C3
:10BA2000E954238801339BB223801188E954E81834
:10BA3000090A4170238802339BB223805288EA545A
:10BA4000E918120A4A702388023323802CE7B36A6C
:10BA5000002BC3D04FF000084FF00C0A4FF0160B2C
:10BA6000B16A5FFA88F20AFB02F201EB0209B9F847
:10BA70000430981CFE283FF679AE208803332B54FF
:10BA8000238801339BB2238005F803B02388013358
:10BA90009BB223808A5AEA54E918120A4A70208815
:10BAA000023080B22080B9F804205AB1D9F80810C9
:10BAB000002993D0284404F013FE2388B9F8042009
:10BAC0001344238096F82C2008F101085FFA88F3CC
:10BAD0009A42C5D823E7092156E79F42FBD2ADF829
:10BAE000087050E730B5C8B1F2B10024651C8D4232
:10BAF00006DA1588A54212D805196D789D420ED137
:10BB0000A14211D9005D48B1013880B230B1023490
:10BB1000A3B210FA84F4A14206DB138030BD055DA8
:10BB200001352C44A4B2E1E70020F7E713B5134632
:10BB30000022ADF806200DF106020446FFF7D2FF01
:10BB400010B1BDF80630E01802B010BD72DF7047CA
:10BB500073DF704774DF704738B5012204460D4625
:10BB6000B0F81414D0F81004FFF7E0FF00B105702E
:10BB700004F13C0204F5826104F15400BDE8384050
:10BB8000FFF7E4BF80F830107047F8B504460F4661
:10BB9000002973D0002871D091F87A301BB191F848
:10BBA0009830002B6CD1D7F8A030042B68D0D7F890
:10BBB0009C30042B64D04FF0000C84F802C007F1D5
:10BBC00078060FCE251D0FC50FCE0FC596E80700CE
:10BBD00085E8070084F830C0D7F8A4306363D7F84D
:10BBE000A830A36304F582624FF6FF73C4F826C43D
:10BBF000A4F82434C4F82024C4F829C422780AB94B
:10BC000084F8543094F82430002B14BFEE231F2303
:10BC100004F15501C4F81014A4F8143404F21442C9
:10BC20003846FFF795FD40BB94F82430002B14BF35
:10BC3000EE231F2304F23121C4F81814A4F81C3495
:10BC400004F21C4207F13C00FFF782FDA8B9A3698A
:10BC5000A4F848304FF480730125A4F8503063698C
:10BC60002064014684F83C50636404F13C0204F112
:10BC70005400FFF76BFF00B92570F8BD0E20FCE7FC
:10BC80000720FAE7F8B5077804460D46002F00F0C4
:10BC900001810023C0F82634C0F82934C38881709C
:10BCA00000F226460BB1012903D0E37943B1022DFE
:10BCB00006D1636BABB1012284F82D24082098478C
:10BCC00004F2274304F22D4113F8012B12B99942D3
:10BCD000FAD117466B1E032B4ED8DFE803F0050B95
:10BCE0000F1284F82D34EBE7A3791BB194F82430BC
:10BCF00003B95FB9E3790BB1002F3FD1237A002B51
:10BD00003ED1637A002B0CBF00250425636BA57020
:10BD1000002B37D0033D012D34D8627992B394F8CB
:10BD20002E247ABB84F83024012284F82F240720A3
:10BD3000984704F13C0518220021284604F0F9FC3C
:10BD4000E26A531E0121022B28BF0A4684F85120C3
:10BD500094F8242084F83C1032B1A36A581E0228BB
:10BD600028BF0B4684F85230A378042B1CD8DFE898
:10BD700003F0780D23365A000025C7E70225C5E7F2
:10BD80000325C3E7002384F82F34D2E7012384F886
:10BD900031300023C4E91063C4F82034022384F84E
:10BDA0003C308023A4F84830A378002B5DD1636B2E
:10BDB000002B6BD1002068E00223002A84F8313088
:10BDC00014BF0723032384F83C302369A4F84830C8
:10BDD0000023C4F82034E36826646364E4E76369FD
:10BDE0006364A369A4F8483012B1062384F83C3098
:10BDF0006379B3B194F82E349BB994F8303483B19D
:10BE0000022384F8503004212046FFF7A5FE0028C5
:10BE1000CAD1052384F8313004F58263C4F8203494
:10BE2000C2E70323F6E7E3696364236AA4F84830B2
:10BE300012B1062384F83C30637983B194F82E3430
:10BE40006BB994F8303453B1022384F85030042194
:10BE50002046FFF781FE0028A6D10623DAE7042357
:10BE6000D8E7002384F831309EE7D4F820142A461E
:10BE700004F15400FFF76AFE38B994F8301094F8D2
:10BE80005400FFF765FE002891D0F8BD94F831000A
:10BE900098478FE70820F8E70388112B10B50C4668
:10BEA0000AD0262B1FD0102B05D1C37B012B02D12A
:10BEB0008388A1F8243410BD0022838881F82E24C1
:10BEC000B1F824249A42F6D10B79002BF3D1012149
:10BED0002046FFF7D7FE0028EDD0A36B002BEAD059
:10BEE000BDE810401847037A013B012BE3D889785D
:10BEF00005230131B1FBF3F303EB8303C91AC9B284
:10BF0000E6E738B5044690F85400FFF723FE012316
:10BF100084F82E34002384F8303484F8503006211D
:10BF20002046FFF719FE054638B9A1782046FFF7ED
:10BF3000A9FE10B1A36B03B19847284638BD30B5B0
:10BF40000D46041D0FCD0FC40FCD0FC495E807009B
:10BF500084E8070030BD75DF704776DF70477ADF11
:10BF600070477BDF70470000034B1A8882420CBF8A
:10BF700018460020704700BF64310020024B9B69C7
:10BF800003B11847704700BF4831002073B585B230
:10BF90002846FFF7E9FF044638B3174E027A337B91
:10BFA0009A420CD200F10A012846FFF7D4FFF0B103
:10BFB00011281AD002B0BDE87040FFF7DFBF0023A0
:10BFC0000372337C43B13B212846FFF7C6FF30F0B4
:10BFD000080301D0FFF7D2FF736933B100228DF857
:10BFE0000420ADF8065001A8984702B070BD237A2E
:10BFF00001332372F9E700BF4831002037B50B4603
:10C00000497A0F4A79B9D2E901141D7A0246002D06
:10C0100018BF21465868FBF74BFB78B103B0BDE869
:10C020003040FFF7ABBF00211972536933B10122D1
:10C03000ADF806008DF8042001A8984703B030BD84
:10C04000483100204B8802889A4212D842889A428E
:10C050000FD380888B8840F2F311884294BF021A74
:10C06000421A9A4205D80844984234BF0020012061
:10C0700070470020704700000388122B70B50146FE
:10C0800059D004D8102B1ED0112B44D070BD502B8A
:10C09000FCD12F4BC288DB899A42F7D1038A022B4D
:10C0A000F4D186883046FFF75FFF05460028EDD0C3
:10C0B00001F1120000F023FA38BB6868FBF726FB99
:10C0C0000028E3D009E0C37B012BDFD14FF6FF70DE
:10C0D000FFF74AFF054620B90420BDE87040FFF78E
:10C0E0004DBF1C4A8E880680002303721368C0F877
:10C0F0000A305368C0F80E3010310A30FFF7A2FF43
:10C10000134B6872DB89002BC0D129463046BDE84D
:10C110007040FFF773BF8088FFF726FF04460028B2
:10C12000B4D04068FBF7F2FA08B1FFF727FF4FF6EB
:10C13000FF732380AAE786883046FFF715FF054680
:10C140000028A3D008310A30FFF77CFF6872DCE7D3
:10C150004831002078310020F8B5064648B305463E
:10C160000FCD154F3C460FC495E8070084E8070043
:10C170003068124C3C60B0B1FFF7F1FEC0B93268D4
:10C1800013682360536863600D480E4A4FF6FF73CF
:10C1900003800D4B40F8043F0021FBF777FA00289D
:10C1A00018BF032004E02046FFF7DBFE0028EBD099
:10C1B000F8BD0E20FCE700BF483100207831002098
:10C1C000643100208DBF020080310020F7B5174692
:10C1D00001900E4691B1019C6CB100252C46294678
:10C1E00001A8FCF74AFD18B13946A8B2B04701349E
:10C1F0000135142DF3D1204603B0F0BD0C46FAE70B
:10C200000AB1FCF719BDFCF72EBD73B50191019C75
:10C2100006466CB100252C46294601A8FCF72DFDE9
:10C2200018B106EB440301349D800135142DF3D180
:10C230003046346002B070BD2DE9F0470388848831
:10C24000103B8CB005460A2B21D8DFE803F00640EE
:10C2500020202020202020654700DFF8E880D8F843
:10C260000830DB430093D8F804106846FCF76AFDF9
:10C27000009901A8FFF7C9FF0DF108090027019BEC
:10C280009F4207D3132C12D90420FBF7EDF80CB012
:10C29000BDE8F08739F802AB00260136514608EBBD
:10C2A0008600FCF7E0FC1E2EF7D10137E7E71F48B8
:10C2B0002146FCF7C1FC1E482146FCF7BDFCEB7B88
:10C2C000022BE4D11B482146FCF7B6FCDFE71748F8
:10C2D00021460CB0BDE8F047FCF7C5BC027A164811
:10C2E0003F2A4FEA1215214694BF00220122FFF790
:10C2F00087FF022D94BF0022012210482146FFF73C
:10C300007FFF012D0E4894BF0022012221460CB070
:10C31000BDE8F047FFF774BF037A002BB7D1427A2C
:10C320000548C2F3C0022146F1E700BFA831002052
:10C33000A4310020AC310020B8310020B4310020FD
:10C34000B0310020A03100201328014602D8024855
:10C35000FCF793BC00207047A431002007B5019082
:10C36000FFF7F2FF019930B10448FCF786FC002882
:10C3700014BF0220012003B05DF804FBAC310020A3
:10C3800007B50190FFF7E0FF019930B10448FCF7D1
:10C3900074FC002814BF0220012003B05DF804FBE8
:10C3A000A831002007B50190FFF7CEFF019928B111
:10C3B000044803B05DF804EBFCF75FBC03B05DF824
:10C3C00004FB00BFB031002007B50190FFF7BCFFB0
:10C3D000019928B1044803B05DF804EBFCF74DBCAB
:10C3E00003B05DF804FB00BFB431002007B5019035
:10C3F000FFF7AAFF019928B1044803B05DF804EBE8
:10C40000FCF73BBC03B05DF804FB00BFB831002073
:10C4100008B518210248FCF739FCC0B208BD00BFBE
:10C42000A031002070B50A4E054630460C46FCF798
:10C4300024FC58B12846FFF787FF38B10734294656
:10C4400006EB8400BDE87040FCF717BC002070BD0F
:10C45000A0310020F8B50B4F054638460C4616466D
:10C46000FCF70BFC60B12846FFF76EFF40B10734C4
:10C470003246294607EB8400BDE8F840FFF7C0BE0E
:10C48000F8BD00BFA0310020034B9B680A4601465F
:10C490001846FFF79BBE00BFA031002073B50B4DBF
:10C4A000019204460E4601462846FCF7E6FB50B1D1
:10C4B000063405EB8404019A6068314602B0BDE899
:10C4C0007040FFF783BE02B070BD00BFA0310020F6
:10C4D000AADF7047002301380B70042806D8DFE874
:10C4E00000F00306080A0C0011230B70704721238B
:10C4F000FBE73123F9E71223F7E72223F5E700886A
:10C5000000F0010070470088C0F340007047F0B5AC
:10C510008B7891B00C46012B38BF012300278DF892
:10C520000E3005460B88607CADF80C306946ADF8DE
:10C5300000708DF80270FFF7CDFFA07C0DF10101B6
:10C54000FFF7C8FF1646237BE27B217D43EAC20347
:10C55000227C43EA02139DF80220B94222F019021C
:10C5600003F0190314BF02210121134361F34203B5
:10C570001C22394609A88DF8023004F0DAF8637BF2
:10C5800013F0300F14D00DF10901E07CADF8087004
:10C590008DF80A70FFF79EFF11238DF808309DF883
:10C5A0000A30012102AA61F342038DF80A300E928B
:10C5B000637B8DF82430A37B8DF825300023CDE9F3
:10C5C0000633089303AB0493A388ADF81C30A3682B
:10C5D000CDF814D01BB1E288ADF818200893A369F8
:10C5E00073B301A90022ADF804208A701A88ADF84F
:10C5F0002C205A88ADF82E205A680D91187B0A928B
:10C60000FFF768FFA3690DF10501587BFFF762FF93
:10C61000A3699A7A197A41EAC201DA7A9B7B41EAE4
:10C6200002119DF80620002B01F0190122F01902D9
:10C6300014BF02230123114363F342018DF8061056
:10C64000E36903B10C93334604AA09A92846FFF70E
:10C650003FFF11B0F0BDA0DF7047A1DF7047ADDF35
:10C660007047B3DF7047B4DF704710B504464088A9
:10C6700000F0B8FDA0802046BDE8104001F06CBE7F
:10C6800030B587B005460C461422002101A804F0FD
:10C6900050F8082301A88DF80430ADF80650039433
:10C6A000FFF7E3FF07B030BD70B586B00546142232
:10C6B000002101A804F03DF84FF6FF739D42ADF84C
:10C6C00006503FD0284600F07FFC1128044633D0A6
:10C6D00016D8D8B10B2820D02046FDF71FFA1A4EE5
:10C6E0001A4902461A48361AF608360446F001007E
:10C6F0002B46FAF7B6F921462846FFF7C1FF03E0BB
:10C7000043F202039842E7D1002216E00F238DF88E
:10C71000043001A8FFF7A9FFF6E710238DF80430D5
:10C7200009480B4B0B49C01AC00800042A4640F0C8
:10C730000200FAF78DF9ECE70122074B2846197839
:10C74000FFF788FE06B070BDD4080300CF150300C4
:10C750005C0803004F15030023320020FFF7A4BF3D
:10C76000024B034918780022FFF798BE25320020BB
:10C7700075C702002DE9F047DFF8348188B098F8DA
:10C7800000100446FFF74EFE0646002840F0848065
:10C79000204600F07DFC0828054632D016D808B3A4
:10C7A00006285BD02846FDF7B9F93D4F3D490246C2
:10C7B0003D483F1AFF083F0447F001002346FAF7BF
:10C7C00050F929462046FFF75BFF09E043F20203D8
:10C7D000984205D043F20143984259D01128E1D143
:10C7E000012546E03146142203A803F0A2FF1123DD
:10C7F00003A88DF80C30ADF80E400126FFF735FF89
:10C80000EEE70DF10600FFF72CFF354601274FF04C
:10C81000020A0DF10809BDF80630BB421ED90022FC
:10C8200049463846CDE903A9FFF71DFFB0B9BDF869
:10C8300008303DB942F605255B1B5D425D4101377D
:10C84000BFB2E8E742F602129342F8D101AB03AA65
:10C85000394620460493FFF702FF30B1204600F02E
:10C86000C1FC00F041FC002503E0BDF80430002BC2
:10C87000F4D00E4B2A4619782046FFF7EBFD98F8C6
:10C8800000103246204608B0BDE8F047FFF7E2BD91
:10C890002046FFF709FFA3E708B0BDE8F08700BF17
:10C8A000D4080300201603005C0803002532002092
:10C8B0002632002013B5044600F094FC00236A469B
:10C8C000092101F0E3F8052805D1044B012219786C
:10C8D0002046FFF7BFFD02B010BD00BF213200208F
:10C8E00008B5084B084918780022FFF7D7FD024623
:10C8F00030B9064B06491878BDE80840FFF7CEBDB1
:10C9000008BD00BF2432002051C90200213200209E
:10C9100015C9020037B542F6A623ADF800300A4B20
:10C92000044618680190012501AA69462046ADF821
:10C930000250FFF790FE28B9044B2A46197820468A
:10C94000FFF788FD03B030BD5E18030020320020E1
:10C9500070B5012186B006462B48FCF7C4F90446A1
:10C96000BFF35F8F00284AD1304600F0A1FA1128AA
:10C97000054639D018D8002843D00B2832D0284695
:10C98000FDF7CCF8214C224902462248241AE4083B
:10C99000240444F001003346FAF763F82946304690
:10C9A000FFF76EFE00241DE0862803D043F2020349
:10C9B0009842E3E71422214601A803F0BAFE0723B8
:10C9C0008DF804301148134B1349ADF80660C01AB6
:10C9D000C008000440F002003246FAF739F801A816
:10C9E000FFF743FE224600E001220C4B3046197847
:10C9F000FFF730FD1CB9BFF35F8F034B1C6006B01F
:10CA000070BD01240246F0E71C320020D408030068
:10CA1000951603005C080300601603002432002012
:10CA200038B503780446A3B94088FFF73DFE658812
:10CA3000284600F01BFB28B1064B01221978284636
:10CA4000FFF708FD6088FFF735FFBDE83840FFF7C6
:10CA500047BF38BD2532002037B50378092B04467F
:10CA600030D1427A72BB057A072D1BD0082D2ED00B
:10CA7000012D27D180886A46294601F08DFA08BB2E
:10CA8000019B1B78F3B1A08800F0DAFB4FF6FF732F
:10CA9000984217D0124B2A461978FFF7DBFCFFF7B4
:10CAA0005FFE0FE0808800F0CBFB4FF6FF739842EB
:10CAB000044607D00B4B01221978FFF7CBFC204628
:10CAC000FFF7F8FE03B0BDE83040FFF709BF064BA3
:10CAD00019680129F6D1BFF35F8F1A60F2E700BF32
:10CAE00025320020243200201C3200202DE9F8439A
:10CAF000FFF78EFCDFF8B090DFF8B08089F8000017
:10CB0000FFF786FC88F80000FFF782FC1D4F1E4EE1
:10CB10003870FFF77DFC3070FFF77AFC1B4D1C4C22
:10CB20002870FFF775FC2070FFF772FC194B187026
:10CB300099F80030182B11D098F80030182B0DD030
:10CB40003B78182B0AD03378182B07D02B78182B6A
:10CB500004D02378182B01D018280CD10E4B0F4885
:10CB60000F49C01AC008000440F00100F9F76CFF3B
:10CB70000320BDE8F8830B4B00201860BFF35F8FE4
:10CB8000F7E700BF253200202632002021320020A6
:10CB900020320020223200205C080300D408030069
:10CBA000D21603001C320020243200202332002041
:10CBB00037B5134B0022CDE90032124B0D461978E0
:10CBC0000446FFF747FC1049104B2046002D08BFD4
:10CBD0000B46019300F006FB0022694600F0C2FFFD
:10CBE00060B1FCF79BFF0A4B0A4902460A481B1A30
:10CBF000DB081B0443F00200F9F72AFF03B030BD45
:10CC000001000900213200206418030068180300A5
:10CC1000D4080300411703005C08030070B50388C3
:10CC20008488502B86B0054639D00FD8352B49D093
:10CC3000362B00F08D80584B584918780022FFF7AA
:10CC40002DFC06B0BDE87040FFF78ABD522B22D004
:10CC5000542BF0D11422002101A803F06AFD122305
:10CC600020468DF80430ADF8064000F0BBFAADF870
:10CC7000080000F039FA4A4B204619780022FFF7E5
:10CC8000E9FB484B204619780022FFF7E3FB01A897
:10CC9000FFF7EBFCCFE72046FFF706FDCBE7037B72
:10CCA000012BC8D1827A012AC5D1018942F602132B
:10CCB0009942C0D13C4B20461978FFF7CBFBFFF7D8
:10CCC0000FFEB8E7394E20463178FFF7ABFB00285E
:10CCD000B1D0002231782046FFF7BCFBEA88B2F5DC
:10CCE000857F0AD072B13248324BC01AC0080004A6
:10CCF000314940F00200F9F7ABFE00212046FFF772
:10CD000057FF98E76A89012A09D02948294B2B49FE
:10CD1000C01AC008000440F00200F9F799FEAE897D
:10CD2000012E07D02248234BC01AC0080004324607
:10CD30002349DEE7E98900222046FFF78EFC002820
:10CD4000DBD1204B324619782046FFF783FB72E790
:10CD50001C4E20463178FFF765FB00283FF46BAF8F
:10CD6000317800222046FFF775FBEE8836B1104877
:10CD7000104BC01AC00800043246B9E7EA89012AFC
:10CD800005D00B480B4BC01AC0080004D0E7297C23
:10CD9000003918BF0121B1E7233200205DC702002E
:10CDA00026320020253200202432002020320020AC
:10CDB000D40803005C0803009E170300D817030083
:10CDC0001218030022320020AFDF7047B1DF704736
:10CDD000B2DF7047B3DF704710B50446808800F0BB
:10CDE0002FFA60802046BDE8104001F0B7BA00007D
:10CDF000F0B5204B204E93E8030089B001AD85E8E3
:10CE000003004FF6FF773088B84217D0002229463A
:10CE100000F0A8FE044638B31422002103A803F052
:10CE200088FC3388ADF81030112C07D0862C07D140
:10CE300007238DF80C3003A8FFF7CEFF09B0F0BD33
:10CE40002046FCF76BFE0D4D33880D4902460D4818
:10CE50002D1AED082D0445F00100F9F702FE082314
:10CE60008DF80C300594E6E7308800F0E8FE30805D
:10CE7000C9E700BF501A030028320020DC08030075
:10CE80006C1803005C080300044B1A884FF6FF730C
:10CE90009A4201D0FFF7ACBF704700BF2832002094
:10CEA000024B4FF6FF721A80002070472832002094
:10CEB0002DE9F04F87B0804600F094F94FF6FF73EC
:10CEC0009842064675D03C4D3C4BED1AED082D04BA
:10CED00045F0010501273A4602AB0821304601F032
:10CEE0005FF80137BFB2044600285DD1DDF80CB011
:10CEF000DA464FF003094AF8069B4B460BF1040251
:10CF000051464046FFF764FF034698BB04AA082138
:10CF1000304601F041F858B1052814D0FCF7FEFD69
:10CF20002749024643462846F9F79BFD4B4610E049
:10CF30000599BBF804308A889A4204D106315046DC
:10CF400003F094FB48B132460821304601F0ECF87A
:10CF50000346184607B0BDE8F08F0821304601F0BF
:10CF600091F828B1FCF7DAFD164903463246DAE7B4
:10CF70000B23EEE70C2815D0052800D12346082105
:10CF80003046019301F07EF8019B40B1FCF7C6FDED
:10CF90000C49034632462846F9F763FD0323002C6B
:10CFA00099D1D6E70124EAE7072814BF03460C23EA
:10CFB000CFE743F20203CCE7DC0803005C08030080
:10CFC000C1180300F91803002DE9F341054600F0EC
:10CFD00009F94FF6FF73984222D100240326274611
:10CFE0004FF001083346224639462846FFF7EEFE49
:10CFF00004282BD0082830D00B2828D116F00203A3
:10D0000019D1E7B9FCB91648164B17491B1ADB08AA
:10D010001B042A4643F00100F9F71AFD0B2019E022
:10D020006A46082100F0B8FF0028D6D1019B9C88F1
:10D030001E689F1DD4E701264FF00008D2E70326A3
:10D040001C461F46F8E703263C46F5E71120B8F1D9
:10D05000000FE3D002B0BDE8F0810020F7E700BF89
:10D060005C080300DC080300781903001FB50DF10C
:10D070000703039300F0B6F802AA012100F08CFF29
:10D0800020B9039B187805B05DF804FB0020FAE78F
:10D0900070B505461048FFF79DFE70B90E4C43F27F
:10D0A000030621884FF6FF722846FFF78DFEB04237
:10D0B00011D1238801332380F3E7FCF72FFD074BC1
:10D0C0000749024607481B1ADB081B0443F001000E
:10D0D000F9F7BEFC032070BD2A320020DC080300F3
:10D0E000F01903005C08030013B5074A044692E8F0
:10D0F00003006B4683E8030000221946204600F037
:10D1000031FD02B010BD00BF581A030046DF704762
:10D11000421E00F10F0312F8010F10B99A42FAD122
:10D1200070470120704708B570B171B103780A7873
:10D13000534013F0FE0F08D106220131013003F0F5
:10D1400095FAB0FA80F0400908BD0020FCE72DE90F
:10D15000F04700F101084F1C06460D4600F1110989
:10D1600001F1110A10223946404603F07FFA0446C5
:10D17000D0B94046FFF7CCFF18B13846FFF7C8FFDB
:10D18000044651464846FFF7CEFF737C03F0FC038C
:10D19000042B05D06B7C03F0FC03042B18BF044662
:10D1A00004F00100BDE8F0870024EAE77FB50546FA
:10D1B0000E4600F0A1FC02AA0DF10601072000F0C6
:10D1C000A3FC10B94FF6FF7409E0BDF80640B44265
:10D1D000F1D003992846FFF7BAFF0028EBD020468C
:10D1E00004B070BD132810B5044602D94FF6FF7085
:10D1F00010BDFFF7A9F80028F8D00A20014B4443DE
:10D20000185BF5E72C320020132838B505460C468C
:10D2100002D943F2020038BDFFF796F80028F8D093
:10D22000064B0A2000FB0530D0F802302360C3888B
:10D23000A380037AA3710020EDE700BF2C32002009
:10D240004FF6FF7398422DE9F04105460CD00C4F84
:10D2500000244FF00A0808FB04F3A6B2DB5BAB42E4
:10D2600005D00134142CF6D14FF6FF7604E0304699
:10D27000FFF76AF80028F4D03046BDE8F08100BF1F
:10D280002C320020038843B9821C0A3012F8013B7B
:10D290001BB98242FAD1184670470120704710B579
:10D2A0000446FFF7EFFF58B122880B889A4208D155
:10D2B00008220231A01C03F0D9F9B0FA80F040092D
:10D2C00010BD0020FCE730B585B0044600F014FC2A
:10D2D00002AA0DF10601072000F016FC10B94FF666
:10D2E000FF700FE0039D204605F14601FFF7D7FFD1
:10D2F00030B905F12A012046FFF7D1FF0028E7D019
:10D30000BDF8060005B030BD13289FBF0A2358435F
:10D31000014B1952704700BF2C32002038B505462A
:10D32000FFF78EFF0446284600F0B6FE38B9132CEE
:10D3300005D80A235C43024B4FF6FF721A5338BDDF
:10D340002C32002070B58CB014466A460D4600F1B0
:10D350001003164613F8011D02F8011B9842F9D17B
:10D360000D22002104A803F0E4F92B788DF81F307A
:10D370006B788DF81E303046AB788DF81D30FFF796
:10D38000C5FE9DF82F3023709DF82E3063709DF8F8
:10D390002D30A3700CB070BD1FB5034608461A7837
:10D3A00002F0FE02042A1BD1DA78B3F801108DF8DE
:10D3B00006209A88ADF804109B79ADF80C2003A9DB
:10D3C00002AA8DF80E30FFF7BDFF032202A901A8C3
:10D3D00003F04CF9B0FA80F0400905B05DF804FBA9
:10D3E0000020FAE730B50388102B93B04ED1041D0E
:10D3F0000FCC07AD0FC50FCC0FC594E807009DF803
:10D40000203003F0FE03062B85E8070009D000F06A
:10D4100073FB9DF82030032B4FEA530204D9022AF4
:10D420003DD04FF6FF7310E002AA0DF10601072070
:10D4300000F06AFB0028F4D0039908A81131FFF727
:10D4400072FE0028F0D0BDF80630BDF81C40184828
:10D450000A226243811883529DF8262008980A7296
:10D460004FF6FF72C1F802009342BDF82400C88055
:10D470000CD0ADF80C3002A80023ADF80A408DF8AE
:10D48000083000F06DFF02A8FFF7CAFA13B030BDF4
:10D49000039908A80131FFF77FFF0028D3D102AA22
:10D4A0000DF10601072000F02FFB0028F0D1B8E7AE
:10D4B0002C32002090DF7047A5DF7047B5DF704742
:10D4C0007FB50023ADF80810ADF80A106A4602A92E
:10D4D0000646ADF80C30ADF80E300093ADF80430D0
:10D4E000FFF7E8FF054600B3114B124CE41AE408BD
:10D4F000FCF714FB240444F0010403460E493246B1
:10D500002046F9F7AEFABDF80020BDF8023052EA25
:10D51000030103D009492046F9F7A3FABDF8042016
:10D520001AB107492046F9F793FA284604B070BDAE
:10D530005C080300A4080300781A0300C21A030061
:10D54000011B030078B14FF0171303601B23037115
:10D550001723C380038141F61B32002301614381FD
:10D560008281184670470E207047000013B50346AD
:10D5700080880C46B8B91A88242A00F09B8014D8F9
:10D58000112A74D0232A00F0A680102A3ED0A37A54
:10D590004BB1E1880020FFF78FFF002840F0A18009
:10D5A0004FF48073638102B010BD3A2A67D0552AC8
:10D5B000EDD1DB88C988A072172B38BF17238B42A7
:10D5C00028BF0B462381FFF779FF60B1FCF7A6FA6D
:10D5D0004D4B4E4902464E481B1ADB081B0443F0D4
:10D5E0000100F9F735FAE27A002AD0D12369002B3D
:10D5F000CDD040F67721ADF802202289ADF8001099
:10D60000ADF80420694620469847C0E7DB7B0A79DD
:10D610000A73012B13D0022B14D0E18823898B428B
:10D6200005D20020FFF748FF70B90123E372217B88
:10D63000637B8B42ABD20020FFF742FFA7E70B884A
:10D64000E380EAE74B88FBE7112802D10123A372AC
:10D65000EDE7FCF763FA2C4B2E4902462C481B1AC7
:10D66000DB081B0443F00100F9F7F2F9DFE71723A9
:10D67000CB800B8141F61B3348818B8187E75B8927
:10D68000CA88934228BF1346172B0A6938BF17234D
:10D690000B8162B1C97A51B140F67721ADF8001023
:10D6A000ADF80200ADF804306946204690470023EB
:10D6B00063816CE71A7A0B694A73002B3FF467AFFA
:10D6C0004DF67A218DF80500ADF80010ADF8020096
:10D6D0008DF8042096E7197A237B994228BF1946D2
:10D6E000AAE711283FF45FAFFCF718FA064B094987
:10D6F000024607481B1ADB081B0443F0010002B076
:10D70000BDE81040F9F7A4B9A4080300881B030082
:10D710005C080300571B0300B0DF704766DF7047EB
:10D7200010B5002104464088FFF7F8FF034608B90A
:10D73000237210BD112801D10123F9E76368BDE808
:10D740001040184760B159B10378DE2B0AD00B683E
:10D750004360DE2303704FF6FF7343800020704761
:10D760000E2070470820704728B10378DE2B04D1C3
:10D770004180002070470E20704708207047F0B5A8
:10D78000054685B00C46002942D0002840D00B78D1
:10D79000DE2B3DD182884B889A4204D10B7A13B19B
:10D7A0000846FFF7BDFF2B88112B33D0512B0FD02C
:10D7B000012B2DD12B7A012B2AD1A9886288914285
:10D7C00026D12046237205B0BDE8F040FFF7A8BF80
:10D7D000AE886388B3421BD1AF79022F18D1AD7BDD
:10D7E0002B1F022B14D800211022684602F0A1FF43
:10D7F000052D18BF4FF4C0736946304618BFADF809
:10D8000004308DF80070FFF787FF08B16368984710
:10D8100005B0F0BD6388AA889A4204BF4FF6FF7333
:10D820006380F5E7012804D0043805288CBF002068
:10D83000012070474FF6FF73438000F0DBBA000011
:10D840002DE9F041264F00238AB04FF6FF70CDE955
:10D8500000333B7000F01CFD4FF6FF78044648F2A1
:10D860000966444513D0A4F58045ADB26A4602A9C5
:10D870002846FBF7A1F8B0420CD02846FBF734F855
:10D8800048F20763984206460CD101233B700AB068
:10D89000BDE8F081204600F09DFC204600F0F8FC39
:10D8A0000446DEE7002EF2D00E480F4D0F492D1A28
:10D8B000ED082D042346324645F00100F9F7D1F872
:10D8C000142200210DEB020002F033FF082305A80B
:10D8D0008DF81430ADF818400796FFF7ABFFD6E788
:10D8E000FC3200205C080300FC080300C41B03009A
:10D8F00070B5044686B014263246002101A802F015
:10D9000018FFA0892378304D00F5804080B2042BA9
:10D91000ADF808003CD008D85A1E022A11D92B783D
:10D920000BB1FFF78DFF06B070BD052BF7D1636813
:10D93000002B43D18DF804604FF6FF73ADF808302B
:10D940001DE043F6FE76B042E18904D901F580423C
:10D9500092B2B242E3D8DA1E534253418DF80D30F1
:10D96000A368049363688DF80C1063B909238DF8DC
:10D9700004309DF8143043F001038DF8143001A8F1
:10D98000FFF758FFCBE70A228DF804200593F6E74E
:10D9900043F6FE739842C2D8E389002BBFD1636877
:10D9A0003BB90B238DF8043000F014FC01232B70DD
:10D9B000E5E70C228DF804200393F7E715228DF894
:10D9C00004200393B8E700BFFC32002007B5002312
:10D9D000A1F58041A0F58040CDE9003389B26B46C6
:10D9E00080B2FAF7CFFF002818BF052003B05DF81A
:10D9F00004FB000030B5204889B0FAF7EFFD70B1A4
:10DA00001E4A1F4B1F499B1ADB081B04024643F0AA
:10DA10000100F9F71DF80324204609B030BDFAF7DC
:10DA2000F3FD044660B1154B15481749C01AC008EC
:10DA30000004224640F00100F9F70AF88624EBE7DB
:10DA400000F0A8FBCDE9034403AA05A94CF20700A6
:10DA5000FAF7A5FF0028DFD101A905A8FAF7EEFE25
:10DA6000019B9D8805F58045ADB205A8FAF70CFF2E
:10DA7000284600F097FBE7E7F1D802005C080300B6
:10DA8000FC080300101C0300521C0300F0B5FF2823
:10DA900087B004460E4615461F462BD80846FFF7AA
:10DAA000C1FE38B303AA2046FFF790FF18B1052442
:10DAB000204607B0F0BD01A903A8FAF7BFFE04464F
:10DAC0000028F4D1019BAE705E8802992E8027B9A0
:10DAD000696003A8FAF7D8FEEAE73F686868B6000D
:10DAE000B74228BF37463A4602F0FAFDBE42F0D9A7
:10DAF0000C24DDE70724DBE7024B0022C3E9002208
:10DB0000704700BFF4320020F0B587B00646FFF73B
:10DB100089FE0F4615460446F8B1A6F58040104A26
:10DB200003A980B2FAF73BFF18B10024204607B0E2
:10DB3000F0BD01A903A8FAF781FE0028F5D1019BE9
:10DB4000AE705A889B882A8003F58043029A6A60E7
:10DB500003A83B80FAF798FEE8E70124E6E700BF58
:10DB6000F432002070B5FF2886B006460B461546F5
:10DB70004AD889780846FFF755FE002844D0A6F514
:10DB80008042ADF80020A1F58042ADF802205A682D
:10DB900001921B88029303AA3046FFF717FF05285E
:10DBA000694603A812D1FAF793FE0446A8B1A0F57E
:10DBB0000643023B0B2B19D80B2B17D8DFE803F0D9
:10DBC000141616160926161616161626FAF784FEC9
:10DBD000EBE78624204606B070BD002DFAD029461A
:10DBE00003A8FAF7F6FEF5E71024F3E70848094D15
:10DBF00009492D1AED082D042246334645F001004F
:10DC0000F8F72FFF0324E5E70724E3E71124E1E712
:10DC10005C080300FC080300901C03004FF6FF7033
:10DC200000F0C0BAFF2808B505D800F0C1FAFFF728
:10DC300007FE002008BD0720FCE700F0E1BA00F075
:10DC40000DBB00F025BB00000A68084B70B50C2521
:10DC5000032A01D9002006E005FB02F4E65A8642B9
:10DC600002D10A60181970BD0132F1E75434002066
:10DC700037B500230D460446019301A9FFF7E4FFE1
:10DC800038B18378AB4206D1837A9B0703D14368CE
:10DC90000BB903B030BD019B0133019301A92046AC
:10DCA000ECE710B5044600F00FFD204601F072FFCE
:10DCB0002046FFF7E9F82046BDE81040FEF7CCBE4D
:10DCC00070B50E4E04460025237AAB420DD84FF6B0
:10DCD000FF732380A370002363604FF47F4323818D
:10DCE000A37A23F00303A37270BD617A2944C9B2F9
:10DCF000304601F034F90135E6E700BF4434002036
:10DD000037B50023CDE90033417A83788DF80230AE
:10DD10000446324801F00AF960B93148314B627A61
:10DD20003149C01AC008000440F00100F8F790FE25
:10DD3000032046E0237AA2788DF8022003EB8303C8
:10DD40009B00ADF80030531E0190072B08D8DFE888
:10DD500003F022070707072204241423ADF800303C
:10DD60002246694632F8040BFFF7FCFE11282AD040
:10DD700017D810B3072824D0FBF7D0FE184D2388FE
:10DD80001A49024617482D1AED082D0445F00100E6
:10DD9000F8F767FECCE70123E0E7838809339B08A7
:10DDA000DCE78628E8D1A37A23F0030343F00103DC
:10DDB000A3720F4B01221A7003E0A37A23F003032E
:10DDC000A37203B030BDA37A23F0030343F0020330
:10DDD000A372074B01221A700020F2E7443400209E
:10DDE000F40803005C080300F71C0300371D030060
:10DDF000403400202DE9F0473E4FC16886B005460B
:10DE00003A4600233E46506881421BD10C2000FB5D
:10DE100003602B78DFF8EC800A2B1AD0142B4AD041
:10DE2000092B4AD16C7A002C47D1002847D0FFF744
:10DE300047FF2846FFF735FF98F800308BB906B04A
:10DE4000BDE8F0870133042B02F10C02DBD1002086
:10DE5000DFE76C7A8CBB90B3837A446043F00203B3
:10DE60008372002588F800504FF00C094FF0010A2A
:10DE700009FB05639B7A9907C3F3400201D4DB07D2
:10DE800032D588F800A002B974B33846FFF738FFDE
:10DE900050B34FF6FF72ADF806200C22554386288A
:10DEA000725BADF808200CD107238DF8043001A86F
:10DEB000FFF7F7FEC3E70124BBE70024B9E70446F8
:10DEC000B7E708228DF804200390FBF727FE0A4CE1
:10DED000735B0A4902460A48241AE408240444F001
:10DEE0000100F8F7BEFDE2E70135042D07F10C074C
:10DEF000BED1A4E754340020F4080300661D0300DB
:10DF00005C080300403400201C4BF7B500221E467D
:10DF10004FF6FF754FF0FF0C0C27104607FB02640D
:10DF20001D809D7083F809C0A17A013221F00301A0
:10DF3000042AA17203F10C0303F8040C43F8080C43
:10DF4000ECD15023CDE900230D490E4B0E484FF480
:10DF5000A07200F0D7FF034668B1FBF7DFFD0B4B63
:10DF60000B4902460B481B1ADB081B0443F0010057
:10DF7000F8F76EFD0323184603B0F0BD54340020BB
:10DF8000003300208434002044340020F4080300CF
:10DF9000C61D03005C0803000023FFF777BD0000E7
:10DFA0002DE9F04180460E4614461F46002B5DD0F9
:10DFB000CB1F012B5CD8531E032B59D8FFF758FEFB
:10DFC000054610BBFF214FF6FF70FFF751FE0546D7
:10DFD000C8B1A0F8008086706B7AFF2B1AD1254853
:10DFE000214600F0D4FFFF28687229D14FF6FF7355
:10DFF0002B8000236B604FF47F432B81AB7AA8709A
:10E0000023F00303AB72112018E0037AA342E3D09C
:10E010000F2013E04FF00008697A16482C7200F0C8
:10E0200085FF80B9144B15486A7A1549C01AC00893
:10E03000000440F00100F8F70BFD0320BDE8F0817B
:10E040004FF00108E8E704EB840424010334C4F32F
:10E050008D04BE7078603C80B8F1000F04D0082EAB
:10E0600002D1A400063C84800020E7E70E20E5E70B
:10E070000720E3E7443400205C080300F4080300B1
:10E08000E41D030008B5FFF7F3FD18B1FFF718FE14
:10E09000002008BD0520FCE77FB50023054603935B
:10E0A00003A9FFF7D1FD0446A8B92846FFF7BAFD3A
:10E0B000014640B3072826D0FBF730FD164C174920
:10E0C00003461748241AE40824042A4644F00100B1
:10E0D000F8F7C7FC16E0A1782846FFF7D3FFA8B1F0
:10E0E000052813D0FBF71AFD0B4EA37800930246C8
:10E0F0000B480C49361AF60836042B4646F0010048
:10E10000F8F7B9FC0321084604B070BD039B013346
:10E11000039303A92846C4E7F4080300AE1E0300D6
:10E120005C080300581E0300CB1F012B70B5064688
:10E130000C46154601D9072070BD1046FFF77DFD3E
:10E140000028F8D021463046FFF792FD28B18470B0
:10E150000580BDE87040FFF7D3BD0520ECE710B5A2
:10E160004FF6FF7304469C4208460AD14FF4807173
:10E17000FAF78CFD84B2B4F5807F09D14FF6FF74B5
:10E1800006E0FF2CFAD82146FAF75FFD0028F5D10A
:10E19000204610BD02484022002102F0CABA00BF4A
:10E1A000883400200149FFF7DABF00BF883400201F
:10E1B0004FF6FF73984210B5044606D00449FFF7A6
:10E1C000CEFF231A5842584110BD0020FCE700BF83
:10E1D000A8340020FF2807B501460AD80190064858
:10E1E000FAF741FD0199054803B05DF804EBFAF731
:10E1F0003ABD03B05DF804FB88340020A834002049
:10E20000FF28014602D80248FAF737BD00207047C0
:10E2100088340020FF28014602D80248FAF72DBDB5
:10E2200000207047A83400204FF6FF73984270B565
:10E2300018BF441C0E4614BFA4B20024A5B2FF2D83
:10E2400002D94FF6FF7506E021463046FAF715FD74
:10E2500001340028F2D0284670BD000070B50B498B
:10E260000A4EFFF7E1FF4FF6FF750446AC4201D1BD
:10E27000204670BD2046FFF7CDFF0028F8D020468D
:10E280003146FFF7D1FF0446F0E700BF8834002095
:10E290000149FFF7C9BF00BFA8340020F8B5074DFA
:10E2A000074E074600243378A34200DCF8BD55F83A
:10E2B000043B384698470134F5E700BFD0340020CE
:10E2C000DF34002070B5204B1B7886B00446002B4D
:10E2D00037D0038885881D4E102B2DD100211422A4
:10E2E00001A88DF8031002F024FA01238DF8043000
:10E2F0004FF6FF73ADF8083004F10803039301A84B
:10E300000DF103030493ADF80650FFF7C7FF28464D
:10E310009DF803203178FEF79DF89DF8030080B941
:10E320002046FFF75FF8204601F082FC204606B049
:10E33000BDE87040FEF772BC31782846FEF772F8EF
:10E34000EDE706B070BD00BFDE340020462300209C
:10E3500008B1FFF7A3BF7047FFF7A0BFFFF79EBF4D
:10E36000FFF79CBF10B5FFF745FB80B1FBF7D6FB6D
:10E37000324C334A334903463348241AE408240410
:10E3800044F00100F8F76DFB0324204610BDFFF7B1
:10E39000BBFD50B1FBF7C2FB284C294A2B49034671
:10E3A0002948241AE4082404EAE701F013FC50B1D8
:10E3B000FBF7B4FB214C224A254903462248241A84
:10E3C000E4082404DCE700F015FF50B1FBF7A6FBDE
:10E3D0001A4C1B4A1F4903461B48241AE40824040C
:10E3E000CEE7FEF783FB50B1FBF798FB134C144AC2
:10E3F000194903461448241AE4082404C0E7FEF728
:10E400004FFD044650B1FBF789FB0C4C0C4A1349F5
:10E4100003460D48241AE4082404B1E7104B4FF6D4
:10E42000FF721A800F4B18600F4B18700F4B0122B0
:10E430001A70FDF7EDFF0E4B1870A6E7CC0803002D
:10E4400004210300111F03005C0803003B1F0300AD
:10E45000651F03008E1F0300B81F0300E21F0300A7
:10E46000DC340020E4340020E0340020DE340020DE
:10E4700046230020084B1B7853B1084A1378022B1F
:10E4800008D8074941F82300013313700020704772
:10E490000820704704207047DE340020DF3400205D
:10E4A000D0340020034B1B780BB101F0DBBB0820FC
:10E4B000704700BFDE34002008B5054B1B782BB138
:10E4C00001F0EEFB082808BF112008BD0820FCE77A
:10E4D000DE340020034B1B780BB101F0B9BA0820E1
:10E4E000704700BFDE340020034B1B780BB1FEF7F2
:10E4F00015BF0820704700BFDE340020F0B5224B66
:10E500001B7889B0002B3CD0204F01234FF6FF70C1
:10E510003B70FFF794FB4FF6FF76B042044619D1EB
:10E5200000251422294603A83D7002F002F90D23AC
:10E5300003A88DF80C30ADF81040ADF80E40FFF791
:10E54000ADFE284609B0F0BD2046FFF778FBB0428B
:10E550000446F6D02046FFF7C7FF05460028F3D053
:10E56000FBF7DCFA0A4D0B4A0B49009403460B48B3
:10E570002D1AED082D0445F00100F8F77CFA03256B
:10E58000DFE70825DDE700BFDE340020CC340020C3
:10E59000CC080300F42003000D2003005C080300F6
:10E5A0002DE9F04F87B081460193334B1B788846A5
:10E5B0001646002B5ED04FF6FF70FFF740FB00259C
:10E5C0000423CDE9025302AB059304AA03AB062151
:10E5D00004460495FFF75AFA072849D04FF6FF770B
:10E5E000BB464FF0FF3AF0B1052825D04FF6FF7338
:10E5F0009C422DD1A34529D0A7420CBF0520002065
:10E60000B9F1000F01D0A9F800B0B8F1000F01D0A6
:10E61000C8F8005006B13780019B0BB1C3F800A0C9
:10E6200007B0BDE8F08F029BAB4224BFA3461D4656
:10E6300053453CBF27469A462046FFF700FB03ABF5
:10E6400004AA06210446FFF721FACCE70520D7E704
:10E65000FBF764FA094D0A4902460A482D1AED08EB
:10E660002D0445F001002346F8F7FBF90320D7E716
:10E670000520D5E70820D3E7DE340020CC080300CE
:10E68000552003005C08030038B50C4C0C4D0023EA
:10E690001A4621462846FFF783FF05280AD14FF680
:10E6A000FF732B8000232360431F58425841054BC2
:10E6B000187038BD0028F7D10120F8E7C8340020D1
:10E6C000DC340020E0340020F0B5044687B08088B8
:10E6D000FEF7B6FD23786080093B032B20D8DFE8E6
:10E6E00003F002253569637A5BB9414A116851B17B
:10E6F000E068814207D113603E4AA1881180E3603F
:10E700000EE0012B0CD13C4B1B784BB1394BA2884E
:10E710001B889A4204D1237A062B01D1FFF7B4FF5C
:10E72000204607B0BDE8F040FFF7B8BD637A002B84
:10E73000F6D12F4A11680029F2D0E0688142EFD16A
:10E740002E4913600A68013A0A60D8E72C4F3B78DB
:10E750006BB90125284B1B7833B1264BA2881B8847
:10E760009A4201D1FFF790FF002D3ED0D8E74FF637
:10E77000FF70FFF764FA4FF6FF7398420546E8D141
:10E78000FFF75FFAA8420646E3D100251422294686
:10E7900001A83D7001F0CDFF0D2320468DF8043017
:10E7A000ADF80860ADF80660FFF778FD01A8FFF747
:10E7B00075FDCFE7124B1A78002AB1D00021142240
:10E7C00001A8197001F0B5FF0E238DF804304FF643
:10E7D000FF73ADF80830ADF806302046A368039308
:10E7E000FFF75CFD01A8FFF759FD07B0F0BD00BFC2
:10E7F000E4340020DC340020E0340020C834002061
:10E80000CC3400202DE9F041374B1B7888B0054609
:10E81000002B65D0354B364C93E80300237801AFCD
:10E8200087E803004BB1DFF8D480D8F8004054B13A
:10E830001124204608B0BDE8F081FFF725FF2378BA
:10E84000002BF5D0EFE72B4A2B4E12883368AA42F3
:10E850001DD1F3B11422214603A801F06AFF092358
:10E8600028468DF80C30FEF7EBFC0623ADF814308B
:10E870009DF81C30ADF80E0064F3000303A8ADF85A
:10E88000105006948DF81C30FFF708FDD1E75A1C94
:10E8900028D00133194A336039462846FFF762F918
:10E8A00004460028C5D00023C8F80030336811287A
:10E8B00003F1FF333360BBD08628BAD00728B8D025
:10E8C000FBF72CF90E4C0F4902460F48241AE408B6
:10E8D000240444F001002B46F8F7C3F80324A8E70A
:10E8E0000824A6E71324A4E7DE340020EC2003006C
:10E8F000E0340020DC340020C8340020E434002060
:10E90000CC0803009D2003005C08030076DF7047FD
:10E9100073B5054669B901A9FFF7DCFD43F20202B0
:10E92000904202D008B1F8F79FFD9DF804309B0794
:10E9300048D400212846FFF7BFFD0646002841D0F5
:10E9400011283FD0204C214BE41AE4080D284FEA4F
:10E95000044416D144F002041D4920462A46F8F723
:10E9600077F813212846FFF7D1FF58B3FBF7D6F805
:10E97000184902462B46204602B0BDE87040F8F721
:10E9800070B80B2808D114492A4644F0020002B09E
:10E99000BDE87040F8F75CB843F20203984202D138
:10E9A0000E492A46F1E7FBF7B9F80D4902462B4616
:10E9B00044F00100F8F755F8304602B0BDE8704069
:10E9C000F8F752BD02B070BDE40803005C08030014
:10E9D0000C2103007D210300B42103001222030057
:10E9E0005C2203002DE9F0410378152B86B0044624
:10E9F00004D8062B05D84BB3032B4DD006B0BDE889
:10EA0000F081073B0E2BF9D801A252F823F000BF8A
:10EA1000B7EA0200FDE902006BEB0200FDE902002B
:10EA20006BEB0200FDE90200FDE90200FDE90200D6
:10EA3000FDE90200FDE90200FDE90200FDE9020036
:10EA4000FDE9020073EB0200BFEB02008088FFF7D4
:10EA5000D9FE862801D0112813D16049604A0B687D
:10EA6000A08822F8130001335A4202F0070203F093
:10EA7000070358BF53420B6006B0BDE8F04100F0F9
:10EA8000C3B8132803D8574BC340DB07B6D406B02E
:10EA9000BDE8F041F8F7E8BC037A012BAED88488D2
:10EAA0001422002101A801F044FE01A8ADF808409D
:10EAB000FFF798FFA2E74C4E3378002B9ED14B4BCB
:10EAC0004B4D4C4F4C49ED1AED082D0445F0030811
:10EAD0004046F7F7B9FF3B78002B3AD101A8F9F788
:10EAE00081FF044608B1F8F7BFFCBDF80A30002BDF
:10EAF00014BF012200223A7028D101AA19461846F3
:10EB0000FFF74EFD044678B9BDF804203B49404666
:10EB1000F7F79EFFBDF80400FFF7E6FC044608B1D6
:10EB2000F8F7A2FC01233B70052C05D1344945F0D0
:10EB30000100F7F789FF61E7062C03D1314945F061
:10EB40000200F6E72CB12046F8F78EFC002C7FF48B
:10EB500055AFF9F7F1FE10B9012333704EE748F2D3
:10EB6000076290423FF44AAF91E7224B01221A70AC
:10EB700044E71D4B1A4D00241C701E4B1C70174B94
:10EB80001F684FF6FF76E3195A4202F0070203F0BE
:10EB9000070358BF534235F81380B0450BD025F812
:10EBA00013601422002101A801F0C3FD01A8ADF8F3
:10EBB0000880FFF717FF0134082CE4D11EE70A4B49
:10EBC00000221A70836848F20D6293423FF454AFFA
:10EBD000B3F5064F7FF412AF4EE700BFEC340020D0
:10EBE00048230020C1000800E83400205C0803002E
:10EBF000E40803004723002097220300B222030009
:10EC0000DC220300FA2203007FB51422002101A8B0
:10EC100001F08FFD072301A88DF80430FFF7E2FE15
:10EC200007B05DF804FB000030B5027885B00446FB
:10EC3000152A00F2E780DFE812F02C002C002C00EF
:10EC400016002E002C002C004700540061007C00B0
:10EC50009700A500B900C2002C00CD002C002C00AC
:10EC60002C002C00D80040886B4DFDF777FB6B4BD8
:10EC7000227A6B49ED1A6B4BED0853F822306A4A41
:10EC800000932D0452F82020638845F00300F7F725
:10EC9000F2FE05B030BD40885F4DFDF75FFB5F4B76
:10ECA0006249ED1A63890193227A5E4B53F8223050
:10ECB00000935D4A638852F82020ED082D0445F04A
:10ECC0000300F7F7E4FEE4E75348544B5849C01AF1
:10ECD000C008000440F0020005B0BDE83040F7F77E
:10ECE000B3BE8068FAF71AFF4B4B524902464B48B5
:10ECF0001B1ADB081B0443F001003EE0474B46486B
:10ED0000617A4D4D227AC01A4C4B53F82110237C66
:10ED100013F0010F4A4B18BF2B46CDE90013C00872
:10ED2000484B494953F82230A288000440F00300C0
:10ED3000C7E7017A434B828853F82130407A3F4934
:10ED4000039251F8205020690293334CFAF7E6FE03
:10ED50003249641AE4082404CDE90050DDE90232A6
:10ED60003A4944F00200ACE72B482C4BA2883849C2
:10ED7000C01AC008000440F0010005B0BDE83040F2
:10ED8000F7F766BE828880680292FAF7C7FE224CC7
:10ED9000029A304903462148241AE408240444F026
:10EDA000010005B0BDE83040F7F75BBE1A481B4BC9
:10EDB0002949C01AC008000440F003008CE78068AD
:10EDC000FAF7ACFE144B2549024614481B1ADB081F
:10EDD0001B0490E7114B104862882149C01AC008F3
:10EDE0000004A38840F00200DBE78068FAF796FE93
:10EDF000094B1C49024609481B1ADB081B0443F057
:10EE00000200BAE70448054B1749C01AC0080004BD
:10EE100040F00200B1E700BFE40803005C08030013
:10EE20003923030004270300F82603007623030098
:10EE3000C8230300DE2303000B0A0300C8260300D7
:10EE400009240300D02603001524030058240300DE
:10EE5000A2240300C9240300F624030009250300AB
:10EE60002D250300692503009825030010B50446ED
:10EE7000FFF7DAFE217821B96088BDE81040FFF77E
:10EE800047BD08290FD10848084B09491B1ADB0860
:10EE90001B0443F00100F7F7D7FDA06818B1BDE8E7
:10EEA0001040F8F7E1BA10BD5C080300E408030065
:10EEB000B625030010B50378042B04461AD10E487A
:10EEC0000E4B62880E491B1ADB081B0443F002003C
:10EED000F7F7BEFD60881321FFF718FD43F2020229
:10EEE0009042034606D033F0080303D0BDE810403B
:10EEF000F8F7BABA10BD00BF5C080300E4080300CD
:10EF00005F21030070B5DDE9045468B161B15BB104
:10EF100004FB05F6964207D835B12CB1C0E90013C1
:10EF2000C0E90254002070BD0720FCE738B50D464B
:10EF3000044608B9002038BD0368002BFAD04068A9
:10EF40000028F7D0FF29F5D0BFF35F8FF9F795FEC2
:10EF50000028EFD0E068236800FB0530EBE738B508
:10EF60000D46044690B1036883B1406870B1FF2933
:10EF70000CD0BFF35F8FF9F780FE38B16068BFF344
:10EF80005F8F2946BDE83840F9F76DBE38BD2DE9E1
:10EF9000F0418846064618B9FF242046BDE8F081B6
:10EFA0000368002BF8D04368002BF5D00027FF241E
:10EFB000B368FDB2AB42EFD970682946F9F745FE58
:10EFC000BFF35F8F40B9FF2C08BF2C462D1B0135C6
:10EFD0004545E2D00137EBE7FF2C07D1FF24F9E7E5
:10EFE00021463046FFF7BBFF0134E4B2AC42F7D311
:10EFF000F4E77EDF70477FDF704786DF704710B52C
:10F000000378182B044602D1FDF702FA207010BDD8
:10F0100010B504464088FEF7E5F8A0802046BDE81C
:10F02000104000F079BD10B586B0044614220021CE
:10F0300001A801F07EFB052301A88DF80430ADF88E
:10F040000640FFF7E5FF06B010BD30B587B00546B6
:10F050000C461422002101A801F06BFB082301A833
:10F060008DF80430ADF806500394FFF7D1FF07B0D8
:10F0700030BD0000F0B587B004460F4616460021AB
:10F08000142201A81D4601F054FB04238DF804301E
:10F09000094BADF8064019788DF80C700022204617
:10F0A000ADF80E608DF81050FDF7D4F901A8FFF708
:10F0B000AFFF07B0F0BD00BF592300207FB5032389
:10F0C0008DF804300388ADF8063043798DF80D10C3
:10F0D00013F0040F14BF0123022301A88DF80C3094
:10F0E000FFF796FF07B05DF804FB000030B5144B46
:10F0F00087B00C46012219780546FDF7ABF9114B94
:10F10000221E1978284618BF0122FDF7A3F9631EB5
:10F110005A425A410C4B28461978FDF79BF91422A4
:10F12000002101A801F005FB022301A88DF804309D
:10F13000ADF806508DF80C40FFF76AFF07B030BD00
:10F14000592300205B2300205A2300202DE9F0479B
:10F15000224B0F46197804469046FDF763F90028C4
:10F1600039D01F4B20461978FDF75CF9014678B37A
:10F170001C4B20461978FDF755F9002804F58070DE
:10F180004FF0070180B214BF4FF001094FF00209A0
:10F19000FEF778FF064698B1052811D0FAF7BEFCB5
:10F1A000114D1249024612482D1AED082D0445F062
:10F1B00001002346F7F755FC31462046FFF745FF8F
:10F1C00043463A4649462046BDE8F047FFF752BF5E
:10F1D00043463A46F7E7BDE8F08700BF59230020D1
:10F1E0005B2300205A2300200C0903001027030092
:10F1F0005C080300F8B5154F154E164D164C3846F1
:10F20000FFF7FDFE3046FFF7FAFE2846FFF7F7FE50
:10F210002046FFF7F4FE3B78182B08D03378182BE4
:10F2200005D02B78182B02D02378182B0BD10B4B41
:10F230000B480C49C01AC008000440F00100F7F761
:10F2400003FC0320F8BD0020FCE700BF5923002089
:10F250005B2300205A230020582300205C08030071
:10F260000C090300D21603002DE9F0418AB00D46C7
:10F2700090460446FDF772F820220646002102A8B7
:10F2800001F057FA012E08D1424B0022197820468E
:10F29000FDF7E0F835B9852716E0002EFAD143F2E4
:10F2A00002014AE02046FDF79DFF4FF6FF739842AA
:10F2B00012D100272B78DB0722D4374BCDF81480EE
:10F2C0000993012E18BF0025394602AB2A46204675
:10F2D000FFF791FE014630E0012EEAD12D4F204686
:10F2E0003978FDF79FF80028E3D12046FFF79BFE11
:10F2F00039782046FDF796F80028DAD18527D9E736
:10F30000852FDED004F5807007216B46012280B284
:10F31000FEF746FE112801460FD090B1FAF7FEFB2A
:10F320001E4D1F4902461F482D1AED082D04234685
:10F3300045F00100F7F795FB032108460AB0BDE848
:10F34000F0810198502201F0F4F901990B46204612
:10F3500003F8346B029301F1180306934B1C0793D7
:10F3600011310D4BCDF814800993FDF74DFF0028A6
:10F37000A7D0FAF7D3FB094D0B49024609482D1ACD
:10F38000ED082D04234645F00200F7F76AFB08213B
:10F39000D3E700BF58230020F03400200C090300FD
:10F3A000792703005C080300DB27030038B5054616
:10F3B0000C46FCF7D3FF012808D154B1214628465A
:10F3C000FFF717FE042808BF112038BD43F20200E2
:10F3D000FBE72046F9E700002DE9F0470388113BE1
:10F3E0008AB00446092B65D8DFE813F00A006400F0
:10F3F00019003A006400640064006400A600530130
:10F40000037A80883D2B41F23D014FF0000218BF86
:10F410004FF488510AB0BDE8F047FFF797BE8088E7
:10F42000FCF79CFF012808D1217AA08801F0010196
:10F43000C1F10201C9B2FFF759FE34F8045F14228A
:10F4400000210DEB020001F074F9043406238DF85D
:10F450001430ADF81650079405A8FFF7D9FD29E040
:10F4600000F110073846FDF72EFF4FF6FF73984264
:10F470000546A08821D1FDF7B5FE0546A0880021EC
:10F48000FFF734FE4FF6FF739D421AD1002600238A
:10F49000A0881A463146FFF7B0FD0828074629D153
:10F4A00099489A4B9A49C01AC008000440F00200DB
:10F4B000F7F7CAFA0AB0BDE8F0872946FDF724FF3E
:10F4C000DCE705AA07212846FEF766FD0028DDD106
:10F4D000A37ED907DAD5069E96F84430DA0701D51F
:10F4E0003436D4E7394606F14600FDF7D8FE002849
:10F4F000F6D1CBE798B1FAF711FB834E009502469F
:10F500008248A3888349361AF608360446F001007B
:10F51000F7F7B1FAA0883946FFF797FDCAE7A37E4F
:10F52000DB07C7D5002EC5D1A088334641F20602BD
:10F530003146FFF79FFDBDE790F808808588B8F158
:10F54000000F40F0A080744B061D197842462846F3
:10F55000FCF780FF617A11F0040105D130460AB052
:10F56000BDE8F047FFF7AABD05F580791FFA89F9D4
:10F5700003AB012207214846FEF712FD0746B0B152
:10F58000FAF7CCFA604C654902466048241AE40850
:10F5900024042B4644F00100F7F763FA3946284665
:10F5A000FFF753FD41463046FFF788FD82E72846C6
:10F5B000FDF718FE4FF6FF7398420446824630D19D
:10F5C00001460498FDF7F2FD50450446804600F0E0
:10F5D0008580DFF858A101462846FDF795FE9AF888
:10F5E00000102846FCF71EFF8046D0B92846FFF7DA
:10F5F0001AFD9AF800102846FCF714FF014600286F
:10F60000D1D0484622460721FEF78EFD814650B9EB
:10F610000121C8E721462846FDF776FE4FF0010894
:10F62000EFE7B846EDE786280ED1142200210DEB56
:10F63000020001F07EF8072305A88DF81430ADF81C
:10F640001650FFF7E5FCE3E7FAF768FA2E4F344966
:10F65000009402462D483F1AFF083F042B4647F00E
:10F660000100F7F708FA49462846FFF7EEFC0021AB
:10F670003046FFF723FDB8F1000F3FF41BAF2046E3
:10F68000FDF74CFE16E7427A414602F00302284697
:10F69000C0E6244B80881978FCF7C4FE0546002894
:10F6A0007FF408AFA088FCF77DFE0146A08839B939
:10F6B000012341F206020AB0BDE8F047FFF7DABCC9
:10F6C000154B2A461978FCF7C5FE03238DF8143034
:10F6D000A388ADF81630ADF81C50BDE6FEF79EFAD3
:10F6E0004045044696D1094B07480F49C01AC00847
:10F6F000000440F00100F7F7A7F904212846FFF7BE
:10F70000A4FC39464FE700BF0C0903005C08030066
:10F710002928030099280300592300200929030000
:10F72000962903005B23002064290300582300204E
:10F7300058B3027802F08203802B25D0C2F3021363
:10F74000042B21D802F0F203322B1DD041788378AC
:10F75000994219D8062917D9102B15D8C17811F05C
:10F76000040311D1007943070ED4084301070BD4D9
:10F77000D30700F0030003D4B0FA80F040097047CB
:10F78000003818BF012070470020704770B515463B
:10F790000E4614220021044600F0CBFF2846FDF758
:10F7A00021FD2670A0806580204670BDFEF7D0BD8B
:10F7B00010B50378182B044602D1FCF729FE2070FF
:10F7C00010BD0000F0B531F0080387B006460D46C5
:10F7D000174628D0112926D01D4C1E4BE41AE408E8
:10F7E0000D294FEA044422D102461B4944F002008D
:10F7F000F7F72EF9042132460DEB0100FFF7C6FFA3
:10F800009FB13B7803F00103C3F10203DBB28DF833
:10F810000C3000238DF8103041F20113ADF80E309A
:10F8200001A8FFF7C3FF07B0F0BD0223EFE70846CA
:10F83000FAF774F909490246334644F00100F7F734
:10F8400010F93246082101A8FFF7A0FF0395E7E76A
:10F85000040903005C080300FD290300B22A030029
:10F860002DE9F0411B4B88B00027CDE904771B68D8
:10F87000039303AD0446884695E807006E4686E884
:10F880000700224606212846FFF780FF2846CDE9DB
:10F890000586FFF78BFF104B00991A682046FFF78B
:10F8A000E3FCA0F111035A425A410C4B054619786A
:10F8B0002046FCF7CFFD0A4B3A4619782046FCF764
:10F8C000C9FD009A29462046FFF77CFF08B0BDE835
:10F8D000F08100BF3C350020303500205F23002040
:10F8E0005E2300200021FFF7BBBF00002DE9F0439D
:10F8F000054689B0914698460E4601BB3F4BCDE97F
:10F9000004111B68039303AC94E807006F4687E873
:10F9100007002A4606212046FFF738FF2046CDE99A
:10F920000567FFF743FF364B009F1B7843B99DF8EF
:10F9300009302BB90526304609B0BDE8F083002711
:10F940004A4639462846FFF731FDA0F111035A42D5
:10F950005A412C4B044619782846FCF77BFD112CA4
:10F9600020D8072C02D80CBB26463DE0A4F10803A2
:10F97000092B1BD801A252F823F000BF69F902003D
:10F98000ADF90200ADF9020069F90200ADF902001B
:10F9900069F90200ADF90200ADF90200ADF902000B
:10F9A000CFF9020043F202039C42DDD02046FAF771
:10F9B000B5F8154E154902461548361AF6083604AC
:10F9C00046F001002B46F7F74CF803260CE0114BEC
:10F9D000324619782846FCF73DFD0F4B4A46197808
:10F9E0002846FCF737FD0026B8F1000FA3D03A46B1
:10F9F00021462846FFF7E6FE9DE700BF3C35002084
:10FA0000393500205E230020040903001D2B03006C
:10FA10005C0803005D2300205C23002013B50A4B23
:10FA200019780446FCF7FEFC084B01901978204633
:10FA3000FCF7F8FC019A01460123204602B0BDE81C
:10FA40001040FFF753BF00BF5C2300205D23002060
:10FA5000F7B507460C46002945D0FCF791FC054652
:10FA6000002842D03846FDF7BDFB06464FF6FF7032
:10FA7000301AA5F1020318BF01205D425D412378D1
:10FA800045EAC00523F009031D4325703846FCF7FD
:10FA900089FC237860F3410323703846FCF794FC1B
:10FAA000237860F3820323703846FCF79FFC0546F9
:10FAB000B8B93846FCF776FC50B16A4607213046A3
:10FAC000FEF76AFA58B9019B93F8440000F0010070
:10FAD000237860F304132370002003B0F0BD2846A0
:10FAE000F6E70120F4E70E20F7E743F20200F4E71F
:10FAF00013B5E0230C4601A98DF80430FFF7A8FFE9
:10FB00009DF80420237828B993430CBF01200020DE
:10FB100002B010BD0020FBE713B50378062B0446A6
:10FB200007D0132B0CD0204602B0BDE81040FFF7E1
:10FB30003DBE8168408802B0BDE81040FFF790BE2E
:10FB4000134B1A68FAB14088FCF72CFC0146E0B16F
:10FB5000227A6088C2F34003C2F300019B00C2F323
:10FB6000800243EAC10343EA021301A98DF804307D
:10FB7000FFF7BEFF80F00100C2B2002160880123C0
:10FB8000FFF7B4FECFE70121F8E70246F6E700BF32
:10FB90003C35002008B503780C2B0FD8082B0FD963
:10FBA000084B094918780022FCF778FC074B0849F4
:10FBB00018780022BDE80840FCF770BC142BEFD089
:10FBC00008BD00BF5F230020E5F802005E2300208F
:10FBD0001DFA020010B50F480F4CFFF7E9FD0F4862
:10FBE000FFF7E6FD0E48FFF7E3FD2046FFF7E0FDD7
:10FBF0002378182B0BD10B4B0B480C49C01AC008AB
:10FC0000000440F00100F6F71FFF032010BD0020A4
:10FC1000FCE700BF5E2300205F2300205C23002060
:10FC20005D2300205C08030004090300D2160300D2
:10FC300008B5FFF7D1FB074B074918780022FCF7FE
:10FC40002DFC064B064918780022BDE80840FCF759
:10FC500025BC00BF5F230020E5F802005E230020E2
:10FC60001DFA020010B5044630B90A4B18600A4B61
:10FC700001221A70002010BDFFF75AFD38B1074B62
:10FC800022681A6022791A71024A1360EFE707208E
:10FC9000F1E700BF3C350020393500203435002025
:10FCA00000230A461946FFF721BEA8DF7047ADDFE3
:10FCB0007047AEDF7047B0DF704762DF70473CDFF0
:10FCC00070473DDF704770472DE9F041044688B02A
:10FCD00038B10388512B27D006D8102B18D0112B00
:10FCE0001AD008B0BDE8F081532BFAD1304DC2884C
:10FCF000EB889A42F5D12B7E002BF2D000F0ACF9C4
:10FD00000028EED06B69022008B0BDE8F04118472A
:10FD10008288274B9A80E4E7254B81889A88914214
:10FD2000DFD14FF6FF72F5E7214DB0F80480AB88C4
:10FD30009845D6D18679022ED3D10289EB889A4292
:10FD4000CFD1837B043B022BCBD9102200210DEBBA
:10FD5000020000F0EEFC01AF69898DF8106002AA84
:10FD6000404602960397FFF7A2FF0646D0B93846F1
:10FD7000FCF7C9FBB0B19DF81630ADF8146043F044
:10FD800001038DF81630A88804A9FFF794FF112805
:10FD9000F9D0BDF81430002BA3D104F1080000F015
:10FDA000F7F89EE740F2FD13ADF81430EBE700BF23
:10FDB000403500207FB50023CDF80B308DF80F3093
:10FDC0000323ADF8023020238DF804300D4B8DF85D
:10FDD0000500DA88ADF8082002228DF80A206A446E
:10FDE0008DF806100492988801AA02A90592FFF7DF
:10FDF00060FF20B9BDF80230032B18BF0C2007B0FC
:10FE00005DF804FB4035002010B54FF0FF310020B5
:10FE1000FFF757FF044658B9B121FFF750FF0446DA
:10FE200030B9044B01205B6998470220F9F7B2FD15
:10FE3000204610BD40350020F0B51B4B87B002AC0A
:10FE4000024603F11007254618685968264603C67E
:10FE50000833BB423446F7D122B3144B12685A61BF
:10FE60004FF6FF719980002119760AB9104A5A613C
:10FE70000E4800F053F898B901204FF659630D4A27
:10FE80008DF8060001A9ADF80430FFF70EFF38B970
:10FE900006492846FFF711FF10B9044800F058F84A
:10FEA00007B0F0BD0E20FBE7822B03004035002099
:10FEB000C7FC0200423500204FF0030C00DF704702
:10FEC00014490B6810B51BB34B680BB30831984746
:10FED00008281DD0104C236858B9587601210220FB
:10FEE000FFF768FFA0B123685B690320BDE81040FD
:10FEF000184700225A7606210220FFF75BFF18B14F
:10FF0000236803205B699847236802205B69EDE75B
:10FF100010BD00BF7C3500207835002018B1034BA0
:10FF20001860002070470E20704700BF7835002011
:10FF300008B5FBF73DFB38B90448FFF7BDFF18B91A
:10FF4000BDE80840FBF768BB08BD00BF7C3500205A
:10FF500010B588B0044620220021684600F0E9FB75
:10FF600022460323ADF8003012F8063B8DF802302C
:10FF700042F60103ADF80C301723ADF80430608869
:10FF80004FF0013369460493FCF7C1FA08B010BD85
:10FF900070B50546007B2A4C01280ED0022824D0DB
:10FFA0000221287BFFF706FF18B1236803205B6955
:10FFB0009847236802205B6909E023685E7E4EB1A2
:10FFC0000621FFF7F7FE48B323685B690320BDE80D
:10FFD0007040184718760146FFF7ECFEF0B1236831
:10FFE00011281E7628D00421DBE76A7B531E132BD1
:10FFF00024D8144E05F10E01301D00F071FB6B7B0F
:020000023000CC
:10000000B36123685B7E002BEDD10F49304651F878
:10001000083B984718B9236801225A7670BD0F280B
:10002000E1D10A4B0A480B49C01AC008000440F04D
:100030000100F6F709FDD6E70621B2E70521B0E792
:10004000783500205C3500207C3500205C080300FA
:1000500084080300922B030008B5044B1B680020A2
:100060005B699847BDE80840FFF7CEBE78350020B1
:1000700010DF704711DF704713B504460949684621
:10008000F9F7F1FC019808B902B010BDD0E90021E0
:100090002046904718B16846F9F7EFFCF2E71120C7
:1000A000F2E700BF6C2C030013B50446074968460D
:1000B000F9F7D9FC019B0BB902B010BD2046D3E97A
:1000C000002190476846F9F7D8FCF3E7842C030039
:1000D000084B9A6822B11A6822F480021A607047AD
:1000E000054B4FF48002C3F88020BFF34F8FBFF35E
:1000F0006F8F7047EC29002000E100E00B4991F878
:1001000016335A09EC231341DB0706D5084B9A68CE
:100110003AB94FF480030B60704742F20200F7F7E0
:10012000A3B91A6842F480021A60704700E100E047
:10013000EC290020F7B5194F3C7864BB184E012517
:1001400020463570FFF798FF112821D02046FFF791
:10015000ABFF144B8DF80340186801900DF10300BC
:10016000F7F7DEFB104901A8FFF782FF0446B0FA5B
:1001700080F0400938709DF80300F7F7F5FB3CB9B3
:100180000A4B34701C70FFF7B9FF2846FFF78CFF4D
:10019000204603B0F0BD0824FAE700BF89350020EF
:1001A00088350020682C0300857402008A35002001
:1001B000F7B5154F3B781BB3144E01203070FFF795
:1001C0005BFF11284FF000051CD00220FFF76CFFE9
:1001D0000DF107008DF80750F7F7A2FBFFF74AFF74
:1001E00004469DF807003D70F7F7BEFB2CB90320CD
:1001F0003470FFF76DFFFFF757FF204603B0F0BDE7
:100200000824FAE72C46F8E78935002088350020D5
:10021000054B1B7833B1054B1B780BB1FFF7C8BFFB
:10022000FFF788BF082070478835002089350020F7
:10023000014B1878704700BF8935002007B5084981
:100240006846F9F710FC019B13B903B05DF804FB95
:10025000D3E9002090476846F9F70FFCF3E700BFA9
:10026000782C0300FFF7EABF60DF704769DF704753
:1002700061DF704730B5134B1B7891B0FBB1124D65
:1002800034240DF1020103A8ADF80240FFF7F0FF9E
:1002900070B9294601A8F9F7E6FB029B002BF0D0C4
:1002A00003A8D3E90021904701A8F9F7E6FBF4E79A
:1002B000052804D011B0BDE83040F7F7D5B811B02B
:1002C00030BD00BF8B350020C82E030030B50C4672
:1002D00085B0002900F08B800023CDE90133454A29
:1002E000039301230A608DF804008DF8063001A9FC
:1002F00006232020ADF80830FFF7B8FF60B1F9F70A
:100300000DFC3D4B3D4902463D481B1ADB081B04D2
:1003100043F00100F6F79CFB0023CDE90133039382
:100320002268012301A940208DF80530FFF79EFFC8
:1003300060B1F9F7F3FB304B3249024630481B1AE3
:10034000DB081B0443F00100F6F782FB00230120C9
:100350002268039301A9CDE901338DF80400FFF76A
:1003600085FF60B1F9F7DAFB234B274902462448A1
:100370001B1ADB081B0443F00100F6F769FB00239E
:10038000CDE9023322684FF4B06301A9A1200193A3
:10039000FFF76CFF60B1F9F7C1FB174B1B49024631
:1003A00017481B1ADB081B0443F00100F6F750FB4B
:1003B000012300252268039501A9A020CDE901555C
:1003C0008DF80430FFF752FF034668B1F9F7A6FB3A
:1003D000094B0F4902460A481B1ADB081B0443F06D
:1003E0000100F6F735FB2B46184605B030BD0E234D
:1003F000FAE700BF60220020BC080300902C030035
:100400005C080300D62C0300222D03006E2D030090
:10041000BF2D030073B505460668FFF725FF2B685F
:10042000B34204461DD91A481A4B1B491B1ADB0854
:100430001B0443F002000190F6F706FB2B681749F6
:1004400001983246F6F70DFB4FF080532A68D3F837
:100450000C31134901989B0203F100539A1AF6F7E5
:10046000F7FA2CB90F4B01221A70204602B070BD6A
:100470002046F9F753FB074B0B49024604481B1A69
:10048000DB081B0443F00100F6F7E2FAEDE700BFDA
:100490005C080300BC080300122E0300412E030079
:1004A000722E03008B3500209C2E03004BDF70471B
:1004B0001FB50E4C01A8FFF7F9FF70B9214602A83D
:1004C000F9F7D1FA039B002BF4D00198D3E900216E
:1004D000904702A8F9F7D1FAF4E7052804D004B050
:1004E000BDE81040F6F7C0BF04B010BDE02E030019
:1004F00053EA020C61D02DE9F04BB3FA83F51E00EC
:1005000007BFB2FA82F502FA05F403FA05F41646BB
:10051000C5F120051EBF22FA05F73C43203556EAF7
:10052000044C4FEA144418BF0134A3464FF00009AD
:10053000C846904271EB030C39D3094207BFB0FAA9
:1005400080F700FA07F6B1FA81F701FA07F6C7F16A
:1005500020071EBF20FA07FC46EA0C062037B6FB30
:10056000FBFC7F1B103F07F01F04C4F120060CFAB0
:1005700004F42CFA06F644BF34460026202FA4BF0C
:100580002646002454EA060C08BF012418EB040890
:1005900049EB0609A4FB027CC01B06FB02CC04FB52
:1005A00003CC71EB0C01904271EB030CC5D20B46EE
:1005B000024649464046BDE8F08BB2FBF3F200002C
:1005C0007F2805D8034A044B105C5B5C18407047D9
:1005D00000207047F82E0300782F0300A0F161037C
:1005E000192B98BF20387047A0F14103192B98BFF1
:1005F000203070477F299ABF017001206FF02E00D4
:10060000704700BF5AB10A787F2A0AD800B1026049
:100610000021501AC3E9001118BF0120704710468D
:1006200070476FF02E007047A0F16103192B98BF3F
:1006300020387047A0F14103192B98BF2030704734
:100640007F2805D8034A044B105C5B5C1840704758
:1006500000207047F82E0300782F0300024B5B68E0
:100660009B6809211B681847602300206AB30F2A82
:1006700070B511D8013A2FD0034600EB020C01E00F
:100680009C4524D08E461C4611F8012B13F8010B13
:100690009042F5D0801A70BD40EA010C1CF0030FA7
:1006A00004460B4606D0013AE6E7043A042A2046FF
:1006B0001946DFD9194620460E680568B54203F190
:1006C000040304F10404F0D0D4E7104670476078C6
:1006D0009EF80120801A70BD00780A78DAE700BF22
:1006E000844640EA010313F0030F18D18446202A00
:1006F0000BD32DE9F007B1E8F807A0E8F807A2F15D
:100700002002202AF7D2BDE8F007042A07D351F8C7
:10071000043B40F8043BA2F10402042AF7D2002A69
:1007200005D011F8013B00F8013B013AF9D16046D0
:1007300070478446002A2DD010F0030F04D000F833
:10074000011B013A26D0F7E7C9B241EA012141EA8B
:100750000141202A12D3A2F120022DE9F0030B4619
:100760000C460D460E460F4688468946A0E8FA0319
:10077000203AFBD2BDE8F00320320BD0042A05D387
:1007800040F8041B043A05D0042AF9D200F8011BF2
:10079000013AFBD16046704700F1010110F0030FF0
:1007A00011D010F8012B002A23D010F0030F0AD02B
:1007B00010F8012B002A1CD010F0030F03D010F802
:1007C000012B002A15D02DE970004FF001324FF0B7
:1007D000803350F8044BA4EB020525EA04051D40C4
:1007E00000D1F6E7A0F1040070BC10F8012B002A3C
:0807F000FBD1A0EB01007047F2
:1007F80039C2020000000000F9AF0200000000004A
:1008080099BE0200F42C00206DD50200283100208A
:1008180079C0020000000000C5E2020000000000EC
:100828007FD702003C310020C9FC0200403500207F
:08083800EDB002000000000019
:10084000A196020000000000719B02000000000061
:08085000C1FE020000000000DF
:040858005DB202008B
:10085C009A12030000000000A01203000000000028
:10086C00A712030000000000AB1203000000000000
:10087C00B012030000000000DA09030000000303BB
:10088C00CC0A030000000000F50A03000000000081
:10089C009412030000000000B71B030000000303C8
:1008AC00050D030000000303602C0300000003038C
:1008BC00B92E030000000303D42E03000000030331
:1008CC00DD200300000003034C18030000000303A9
:1008DC003C1A030000000303B026030000000303CE
:1008EC00681A030000000303001F03000000030349
:1008FC00E61C030000000303722B0300000003033B
:10090C00EC29030000000303780D03000000000035
:08091C00940D0300000000002F
:08092400E59402000000000050
:10092C00AD960200000000000D9C020000000000CB
:08093C0099B202000000000066
:100944007502030000000000B10403000000000071
:10095400AC09030000000000B8090300882200204D
:10096400B82300208024002088240020C0230020F5
:040974001800000067
:100978000000000000000000C18402000000000028
:04098800000000006B
:10098C00FFFFFFFFFFFFFFFFFFFFFFFFFFFFFFFF6B
:10099C0000000000000000000000D601060100006D
:1009AC00F164020055650200A16402007561727465
:1009BC005F6C6F675F6261636B656E64004261635D
:1009CC006B656E647320666C75736865640061702A
:1009DC0070000000A82800207F00000028290020BB
:1009EC001B5B313B33316D0025734C6F6773206497
:1009FC00726F70706564202825642925730D0A00B8
:100A0C001B5B306D003C25733E2025733A20002083
:100A1C002530327800202020007C002563001B5BF1
:100A2C00313B33306D001B5B313B33326D001B5B54
:100A3C00313B33336D001B5B313B33346D001B5B3F
:100A4C00313B33356D001B5B313B33366D001B5B2B
:100A5C00313B33376D007761726E696E6700696E7A
:100A6C00666F006465627567000000000C0A030085
:100A7C002A0A0300EC090300320A03003A0A0300B5
:100A8C00420A03004A0A0300520A03005A0A0300EE
:100A9C0000000000E20A0300620A03006A0A030075
:100AAC006F0A03000D0E0F10111213140000010138
:100ABC000100000001010000000001010000000025
:100ACC006170705F627574746F6E00009822002004
:100ADC00466174616C206572726F72005379737425
:100AEC00656D207265736574006170705F74696DFB
:100AFC00657200000100060000000000642900205F
:100B0C00F174020052544320696E7374616E636514
:100B1C0020616C726561647920696E697469616CBD
:100B2C00697A65642E005254433A20696E6974697F
:100B3C00616C697A65642E00000000000000000002
:100B4C00000000000338FDD8704700000000FFFFD4
:100B5C00DEC0ADDEFE011EF1DEC0ADDEFF011EF11A
:100B6C0030313233343536373839414243444546D7
:100B7C00705F667300257320636865636B20666124
:100B8C00696C656420696E20257328292077697447
:100B9C00682076616C756520307825782E00705F42
:100BAC0066732D3E705F61706900705F646573746D
:100BBC00006C656E00616464725F69735F616C697F
:100BCC00676E6564333228737263290061646472E2
:100BDC005F69735F77697468696E5F626F756E6465
:100BEC007328705F66732C207372632C206C656E97
:100BFC002900705F7372630021286C656E202520BC
:100C0C00705F66732D3E705F666C6173685F696EB2
:100C1C00666F2D3E70726F6772616D5F756E697471
:100C2C002900616464725F69735F616C69676E65EA
:100C3C0064333228646573742900616464725F697B
:100C4C00735F616C69676E65643332282875696EF1
:100C5C007433325F7429705F73726329006164644A
:100C6C00725F69735F77697468696E5F626F756EC6
:100C7C00647328705F66732C20646573742C206C0D
:100C8C00656E2900616464725F69735F706167658A
:100C9C005F616C69676E656428705F66732C207089
:100CAC006167655F616464722900616464725F6985
:100CBC00735F77697468696E5F626F756E647328B1
:100CCC00705F66732C20706167655F616464722C61
:100CDC0020286C656E202A20705F66732D3E705F35
:100CEC00666C6173685F696E666F2D3E65726173C9
:100CFC00655F756E69742929006E72665F66737420
:100D0C006F72616765006E72665F6673746F726195
:100D1C0067655F6572617365006E72665F6673749A
:100D2C006F726167655F7772697465006E72665F7A
:100D3C006673746F726167655F696E697400000039
:100D4C0000100000040000000100000029950200C2
:100D5C0009950200F99402003D970200ED960200FD
:100D6C00CD940200D1940200D59402007077725F8A
:100D7C006D676D7400000000C0220020580803004D
:100D8C005C08030004000000736F72746C69737468
:100D9C00004E52465F53554343455353004E524603
:100DAC005F4552524F525F5356435F48414E444C3D
:100DBC0045525F4D495353494E47004E52465F458D
:100DCC0052524F525F534F46544445564943455F28
:100DDC004E4F545F454E41424C4544004E52465F87
:100DEC004552524F525F494E5445524E414C004E63
:100DFC0052465F4552524F525F4E4F5F4D454D002C
:100E0C004E52465F4552524F525F4E4F545F464FC3
:100E1C00554E44004E52465F4552524F525F4E4F14
:100E2C00545F535550504F52544544004E52465FF8
:100E3C004552524F525F494E56414C49445F5041C6
:100E4C0052414D004E52465F4552524F525F494EF1
:100E5C0056414C49445F5354415445004E52465FF1
:100E6C004552524F525F494E56414C49445F4C4596
:100E7C004E475448004E52465F4552524F525F49BE
:100E8C004E56414C49445F464C414753004E5246E6
:100E9C005F4552524F525F494E56414C49445F4454
:100EAC00415441004E52465F4552524F525F4441AD
:100EBC0054415F53495A45004E52465F4552524F7A
:100ECC00525F54494D454F5554004E52465F455262
:100EDC00524F525F4E554C4C004E52465F4552524B
:100EEC004F525F464F5242494444454E004E524683
:100EFC005F4552524F525F494E56414C49445F41F7
:100F0C00444452004E52465F4552524F525F425536
:100F1C005359004E52465F4552524F525F434F4E0B
:100F2C004E5F434F554E54004E52465F4552524F02
:100F3C00525F5245534F5552434553004E52465FF4
:100F4C004552524F525F4D4F44554C455F4E4F5496
:100F5C005F494E495449414C495A4544004E52460A
:100F6C005F4552524F525F4D555445585F494E495B
:100F7C00545F4641494C4544004E52465F455252DF
:100F8C004F525F4D555445585F4C4F434B5F464154
:100F9C00494C4544004E52465F4552524F525F4DAC
:100FAC00555445585F554E4C4F434B5F4641494C49
:100FBC004544004E52465F4552524F525F4D555478
:100FCC0045585F434F4E445F494E49545F46414933
:100FDC004C4544004E52465F4552524F525F4D4F66
:100FEC0044554C455F414C52454144595F494E492B
:100FFC005449414C495A4544004E52465F45525261
:10100C004F525F53544F524147455F46554C4C002D
:10101C004E52465F4552524F525F4150495F4E4FC0
:10102C00545F494D504C454D454E544544004E522D
:10103C00465F4552524F525F464541545552455FAB
:10104C004E4F545F454E41424C4544004E52465F14
:10105C004552524F525F494F5F50454E44494E479F
:10106C00004E52465F4552524F525F4452565F54A7
:10107C0057495F4552525F4F56455252554E004E9E
:10108C0052465F4552524F525F4452565F54574935
:10109C005F4552525F414E41434B004E52465F45B5
:1010AC0052524F525F4452565F5457495F45525209
:1010BC005F444E41434B004E52465F4552524F5295
:1010CC005F424C455F495053505F52585F504B54F0
:1010DC005F5452554E4341544544004E52465F4571
:1010EC0052524F525F424C455F495053505F4348F8
:1010FC00414E4E454C5F414C52454144595F455819
:10110C0049535453004E52465F4552524F525F4220
:10111C004C455F495053505F4C494E4B5F444953CB
:10112C00434F4E4E4543544544004E52465F455244
:10113C00524F525F424C455F495053505F504545AA
:10114C00525F52454A454354454400556E6B6E6F91
:10115C00776E206572726F7220636F646500000099
:10116C00000000009D0D030001000000A90D03000C
:10117C0002000000C70D030003000000E80D03008F
:10118C0004000000FB0D0300050000000C0E030022
:10119C0006000000200E030007000000380E0300BC
:1011AC0008000000500E030009000000680E030048
:1011BC000A000000810E03000B000000990E0300D2
:1011CC000C000000B00E03000D000000C40E030064
:1011DC000E000000D60E03000F000000E50E030009
:1011EC0010000000F90E030011000000100F0300A6
:1011FC00120000001F0F030013000000340F030047
:10120C0080000000480F030081000000690F0300FC
:10121C0082000000850F030083000000A10F030073
:10122C0084000000BF0F030085000000E00F0300E6
:10123C008600000005100300900000001C10030045
:10124C00910000003A1003009200000058100300B7
:10125C00008200006D100300018200008B1003005F
:10126C0002820000A710030000840000C3100300DA
:10127C0001840000E7100300028400001111030038
:10128C000384000036110300636C6F636B00434CE6
:10129C004F434B004750494F544500505253005553
:1012AC004152540055415254450000000D000300BA
:1012BC008DAB02000E0003008DAB02000F0003008B
:1012CC008DAB0200100003008DAB0200E022002069
:1012DC000023002020230020446576696365206983
:1012EC007320707265706172696E6720746F20650F
:1012FC006E74657220626F6F746C6F6164657220BE
:10130C006D6F64652E00446973636F6E6E656374F4
:10131C006564202564206C696E6B732E00446576C1
:10132C006963652077696C6C20656E7465722062E8
:10133C006F6F746C6F61646572206D6F64652E00E5
:10134C005265717565737420746F20656E74657267
:10135C0020626F6F746C6F61646572206D6F646571
:10136C00206661696C6564206173796E6368726F65
:10137C006E656F75736C792E00526571756573743B
:10138C0020746F2073656E64206120726573706FBA
:10139C006E736520746F20636C69656E7420666172
:1013AC00696C65642E00556E6B6E6F776E2065767A
:1013BC00656E742066726F6D20626C655F64667515
:1013CC005F627574746F6E6C6573732E0046616921
:1013DC006C656420746F20646973636F6E6E6563F3
:1013EC007420636F6E6E656374696F6E2E20436F2D
:1013FC006E6E656374696F6E2068616E646C653ABD
:10140C00202564204572726F723A20256400506F5B
:10141C00776572206D616E6167656D656E7420779E
:10142C00616E747320746F20726573657420746FB1
:10143C0020444655206D6F64652E00506F776572A1
:10144C00206D616E6167656D656E7420616C6C6F8B
:10145C0077656420746F20726573657420746F20D7
:10146C00444655206D6F64652E004E425F444655D0
:10147C00313100427574746F6E6C65737320444621
:10148C0055204170706C69636174696F6E20737460
:10149C0061727465642E00457261736520626F6EB3
:1014AC006473210053657474696E67207665637488
:1014BC006F72207461626C6520746F20626F6F7440
:1014CC006C6F616465723A2030782530387800464C
:1014DC0061696C65642072756E6E696E67207364E9
:1014EC005F736F66746465766963655F7665637454
:1014FC006F725F7461626C655F626173655F736567
:10150C0074004E6F20626F6F746C6F616465722033
:10151C0077617320666F756E640053657474696EC1
:10152C006720766563746F72207461626C652074D9
:10153C006F206D61696E206170703A2030782530B3
:10154C00387800546865206C6F63616C206461743A
:10155C00616261736520686173206368616E6765A1
:10156C00642C20736F20736F6D65207375627363C9
:10157C0072697074696F6E7320746F206E6F74690A
:10158C006669636174696F6E7320616E6420696E45
:10159C006469636174696F6E7320636F756C64202A
:1015AC006E6F7420626520726573746F726564204F
:1015BC00666F7220636F6E6E5F68616E646C65201F
:1015CC002564006773636D5F6C6F63616C5F64624D
:1015DC005F63616368655F6170706C792829207244
:1015EC00657475726E65642025732077686963680D
:1015FC002073686F756C64206E6F742068617070F6
:10160C00656E2E20636F6E6E5F68616E646C653AFA
:10161C00202564006773636D5F736572766963651B
:10162C005F6368616E6765645F696E645F73656E46
:10163C006428292072657475726E65642025732088
:10164C00666F7220636F6E6E5F68616E646C653A74
:10165C0020256400466C6173682066756C6C2E20C6
:10166C00436F756C64206E6F742073746F72652099
:10167C006461746120666F7220636F6E6E5F686167
:10168C006E646C653A202564006773636D5F6C6FE4
:10169C0063616C5F64625F63616368655F757064EE
:1016AC0061746528292072657475726E65642025D5
:1016BC007320666F7220636F6E6E5F68616E646C10
:1016CC00653A20256400436F756C64206E6F74203E
:1016DC006163717569726520636F6E6E5F7374619F
:1016EC007465207573657220666C6167732E204972
:1016FC006E63726561736520424C455F434F4E4E7D
:10170C005F53544154455F555345525F464C4147D6
:10171C005F434F554E5420696E2074686520626C8F
:10172C00655F636F6E6E5F7374617465206D6F645B
:10173C00756C652E0043415220636861722076619E
:10174C006C756520636F756C646E27742062652000
:10175C0073746F72656420286572726F723A2025FB
:10176C0073292E205265617474656D7074207769CD
:10177C006C6C2068617070656E206F6E207468658B
:10178C00206E65787420636F6E6E656374696F6E1E
:10179C002E00556E657870656374656420474154FE
:1017AC005420737461747573207768696C65206755
:1017BC00657474696E6720434152206368617220BE
:1017CC0076616C75653A2030782578004D756C74AF
:1017DC0069706C6520282564292043415220636878
:1017EC006172616374657269737469637320666F87
:1017FC00756E642C207573696E672074686520663D
:10180C00697273742E00556E6578706563746564C7
:10181C00204341522063686172616374657269731D
:10182C007469632076616C7565206C656E6774688D
:10183C0020282564292C2073746F726520302E00AB
:10184C00706565725F6D616E616765725F67636D10
:10185C0000000100FFFF000000000000010000007C
:10186C007064735F706565725F646174615F7374DB
:10187C006F726528292072657475726E65642025F7
:10188C0073207768696C652073746F72696E67205A
:10189C0073657276696365206368616E67656473EE
:1018AC007461746520666F7220706565722069645E
:1018BC002025642E007064625F706565725F6461E0
:1018CC0074615F7074725F67657428292072657427
:1018DC0075726E656420257320666F7220636F6E5F
:1018EC006E5F68616E646C653A20256400446964BF
:1018FC0020616E6F74686572207468726561642013
:10190C006D616E6970756C61746520504D5F5045EA
:10191C0045525F444154415F49445F474154545FD1
:10192C004C4F43414C20666F7220706565725F6945
:10193C0064202564206174207468652073616D6572
:10194C002074696D653F207064625F77726974659D
:10195C005F6275665F72656C6561736528292072BC
:10196C00657475726E65642025732E0073645F62F6
:10197C006C655F67617474735F7379735F617474A2
:10198C00725F73657428292072657475726E656454
:10199C00204E52465F4552524F525F494E56414C73
:1019AC0049445F4441544120666F72204E554C4C63
:1019BC0020706F696E746572207768696368207334
:1019CC00686F756C64206E657665722068617070E6
:1019DC00656E2E20636F6E6E5F68616E646C653A27
:1019EC002025640073645F626C655F676174747357
:1019FC005F696E697469616C5F757365725F68614C
:101A0C006E646C655F6765742829207265747572E5
:101A1C006E65642025732077686963682073686F2E
:101A2C00756C64206E6F742068617070656E2E002A
:101A3C00706565725F6D616E616765725F67736318
:101A4C006D00000001000100601A0300010001009C
:101A5C00641A03000100000000000000706565724C
:101A6C005F6D616E616765725F696D0073645F6263
:101A7C006C655F6761705F646174615F6C656E67F4
:101A8C0074685F75706461746528292028726571AB
:101A9C007565737429206F6E20636F6E6E65637449
:101AAC00696F6E20307825782072657475726E655A
:101ABC00642025732E0054686520726571756573FA
:101ACC007465642054582F5258207061636B657490
:101ADC00206C656E67746820697320746F6F206C5E
:101AEC006F6E672062792025752F2575206F6374C2
:101AFC006574732E00546865207265717565737416
:101B0C00656420636F6D62696E6174696F6E206FBE
:101B1C006620545820616E64205258207061636BAB
:101B2C006574206C656E6774687320697320746FBC
:101B3C006F206C6F6E67206279202575206D69634C
:101B4C00726F7365636F6E64732E0073645F626C87
:101B5C00655F67617474635F65786368616E676500
:101B6C005F6D74755F726571756573742829207269
:101B7C00657475726E65642025732E0073645F62E4
:101B8C006C655F67617474735F65786368616E67B9
:101B9C00655F6D74755F7265706C7928292072654C
:101BAC007475726E65642025732E006E72665F62AA
:101BBC006C655F6761747400436F756C64206E6F45
:101BCC00742064656C657465207065657220646151
:101BDC0074612E206664735F66696C655F64656C06
:101BEC0065746528292072657475726E6564203081
:101BFC0078257820666F7220706565725F69643A2B
:101C0C0020256400436F756C64206E6F7420696EC0
:101C1C00697469616C697A6520666C61736820739C
:101C2C00746F726167652E206664735F7265676995
:101C3C007374657228292072657475726E656420E0
:101C4C00307825782E00436F756C64206E6F74208D
:101C5C00696E697469616C697A6520666C61736818
:101C6C002073746F726167652E206664735F696E92
:101C7C00697428292072657475726E6564203078D9
:101C8C0025782E00436F756C64206E6F742077720C
:101C9C00697465206461746120746F20666C617373
:101CAC00682E206664735F7265636F72645F7B7706
:101CBC00726974657C7570646174657D2829207205
:101CCC00657475726E656420307825782E20706589
:101CDC0065725F69643A20256400706565725F6D9A
:101CEC00616E616765725F70647300706D5F6275C1
:101CFC00666665725F7074725F676574282920630D
:101D0C006F756C64206E6F74207265747269657681
:101D1C00652052414D206275666665722E20626C9C
:101D2C006F636B5F69643A202564007064735F7045
:101D3C006565725F646174615F73746F7265282985
:101D4C002072657475726E65642025732E20706523
:101D5C0065725F69643A20256400536F6D6520706D
:101D6C00656572206461746120776173206E6F7495
:101D7C002070726F7065726C7920777269747465FB
:101D8C006E20746F20666C6173682E207772697494
:101D9C00655F6275665F73746F7265282920726562
:101DAC007475726E656420257320666F7220706581
:101DBC0065725F69643A20256400504D5F42554658
:101DCC004645525F494E49542829207265747572F4
:101DDC006E65642025732E0043616E6E6F742073E4
:101DEC00746F7265206461746120746F20666C611D
:101DFC007368206265636175736520706D5F6275D1
:101E0C00666665725F7074725F67657428292063FB
:101E1C006F756C64206E6F74207265747269657670
:101E2C00652052414D206275666665722E2049739D
:101E3C0020626C6F636B5F6964202564206E6F7425
:101E4C0020616C6C6F63617465643F007064625FE9
:101E5C0077726974655F6275665F72656C656173D4
:101E6C006528292072657475726E6564202573204F
:101E7C0077686963682073686F756C64206E6F7423
:101E8C002068617070656E2E20706565725F696484
:101E9C003A2025642C20646174615F69643A2025C2
:101EAC006400506565722049442025642077617375
:101EBC00206E6F742070726F7065726C7920726511
:101ECC006C65617365642E207064735F70656572F8
:101EDC005F69645F66726565282920726574757226
:101EEC006E65642025732E20706565725F69643A97
:101EFC0020256400706565725F6D616E6167657247
:101F0C005F706462002573206661696C6564206291
:101F1C00656361757365207064735F696E6974289D
:101F2C00292072657475726E65642025732E0025E8
:101F3C0073206661696C65642062656361757365A5
:101F4C00207064625F696E697428292072657475EB
:101F5C00726E65642025732E002573206661696C92
:101F6C006564206265636175736520736D5F696E6E
:101F7C00697428292072657475726E6564202573E6
:101F8C002E002573206661696C656420626563614F
:101F9C0075736520736D645F696E6974282920728E
:101FAC00657475726E65642025732E00257320662A
:101FBC0061696C6564206265636175736520676334
:101FCC006D5F696E697428292072657475726E650F
:101FDC00642025732E002573206661696C6564206E
:101FEC0062656361757365206773636D5F696E69A4
:101FFC007428292072657475726E65642025732EA1
:10200C000025732829206661696C6564206265630C
:10201C006175736520612063616C6C20746F207036
:10202C006D5F706565725F64656C657465282920E9
:10203C0072657475726E65642025732E20706565EB
:10204C00725F69643A20256400436F756C64206E7E
:10205C006F742072657472656976652072616E6B3F
:10206C00732E207064625F706565725F6461746169
:10207C005F6C6F616428292072657475726E65647B
:10208C002025732E20706565725F69643A20256483
:10209C0000436F756C64206E6F742075706461748E
:1020AC00652072616E6B2E207064625F7261775F67
:1020BC0073746F726528292072657475726E65640D
:1020CC002025732E20706565725F69643A20256443
:1020DC0000706565725F6D616E616765720000000E
:1020EC0001000600C8340020706D5F706565727366
:1020FC005F64656C65746500706D5F696E69740012
:10210C00706D5F636F6E6E5F7365637572652829A2
:10211C00206661696C656420626563617573652016
:10212C00616E20534D502074696D656F7574206914
:10213C00732070726576656E74696E672073656363
:10214C007572697479206F6E20746865206C696E85
:10215C006B2E20446973636F6E6E656374696E6772
:10216C0020636F6E6E5F68616E646C652025642EF3
:10217C000073645F626C655F6761705F6469736351
:10218C006F6E6E65637428292072657475726E6546
:10219C0064202573206F6E20636F6E6E5F68616EB6
:1021AC00646C652025642E00706D5F636F6E6E5FCE
:1021BC007365637572652829206661696C65642096
:1021CC0062656361757365207468652073746F72E2
:1021DC006564206461746120666F7220636F6E6E3B
:1021EC005F68616E646C6520256420646F65732084
:1021FC006E6F74206861766520612076616C69640D
:10220C00206B65792E00706D5F636F6E6E5F73650A
:10221C00637572652829206661696C656420626546
:10222C00636175736520636F6E6E5F68616E646C5D
:10223C0065202564206973206E6F7420612076619F
:10224C006C696420636F6E6E656374696F6E2E00CB
:10225C00417373657274696E672E20706D5F636F66
:10226C006E6E5F736563757265282920726574756F
:10227C00726E6564202573206F6E20636F6E6E5FC7
:10228C0068616E646C652025642E00417474656D04
:10229C007074696E6720746F20636C65616E206664
:1022AC006C6173682E0044656C6574696E67206C94
:1022BC006F776573742072616E6B656420706565F1
:1022CC00722028706565725F69643A202564290064
:1022DC00546865726520617265206E6F207065654B
:1022EC00727320746F2064656C6574652E00506584
:1022FC0065722072616E6B732066756E6374696FA4
:10230C006E616C6974792069732064697361626CA5
:10231C0065642C20736F206E6F207065657273205E
:10232C006172652064656C657465642E00436F6E24
:10233C006E656374696F6E20736563757265643A5C
:10234C0020726F6C653A2025732C20636F6E6E5F64
:10235C0068616E646C653A2025642C2070726F6322
:10236C0065647572653A20257300436F6E6E656304
:10237C0074696F6E20736563757269747920666118
:10238C00696C65643A20726F6C653A2025732C2059
:10239C00636F6E6E5F68616E646C653A2030782591
:1023AC00782C2070726F6365647572653A202573A2
:1023BC002C206572726F723A20256400466C617332
:1023CC00682073746F726167652069732066756C21
:1023DC006C00556E65787065637465642066617415
:1023EC00616C206572726F72206F636375727265B7
:1023FC00643A206572726F723A202573002C206E3D
:10240C006F206368616E676500506565722064615A
:10241C007461207570646174656420696E20666CEB
:10242C006173683A20706565725F69643A2025644F
:10243C002C20646174615F69643A2025732C2061DF
:10244C006374696F6E3A202573257300506565724D
:10245C0020646174612075706461746564206661C8
:10246C00696C65643A20706565725F69643A202511
:10247C00642C20646174615F69643A2025732C209C
:10248C00616374696F6E3A2025732C206572726FCC
:10249C00723A20257300506565722064656C657412
:1024AC006564207375636365737366756C6C793AD8
:1024BC0020706565725F69643A202564005065651B
:1024CC00722064656C6574696F6E206661696C65F9
:1024DC00643A20706565725F69643A2025642C202B
:1024EC006572726F723A20257300416C6C207065B6
:1024FC006572732064656C657465642E00416C6C48
:10250C0020706565722064656C6574696F6E2066F9
:10251C0061696C65643A206572726F723A2025733A
:10252C00004C6F63616C20444220636F756C6420B7
:10253C006E6F74206265206170706C6965643A20FE
:10254C00636F6E6E5F68616E646C653A2025642CF7
:10255C0020706565725F69643A20256400466C6181
:10256C007368206761726261676520636F6C6C656C
:10257C006374696F6E206661696C65642077697439
:10258C0068206572726F722025732E00556E657807
:10259C0070656374656420504D206576656E74209B
:1025AC0049443A20307825782E0041737365727453
:1025BC00696E672E005570646174650044656C65C6
:1025CC007465004F7574646174656420283029004B
:1025DC0053657276696365206368616E6765642014
:1025EC0070656E64696E6720666C6167004F757408
:1025FC00646174656420283229004F7574646174B9
:10260C00656420283329004170706C6963617469BA
:10261C006F6E20646174610052656D6F7465206427
:10262C006174616261736500506565722072616EE0
:10263C006B00426F6E64696E672064617461004C5C
:10264C006F63616C206461746162617365004365E2
:10265C006E7472616C206164647265737320726550
:10266C00736F6C7574696F6E00456E6372797074FC
:10267C00696F6E00426F6E64696E670050616972BB
:10268C00696E6700496E76616C696420526F6C6587
:10269C00005065726970686572616C0043656E7498
:1026AC0072616C00706565725F6D616E61676572F9
:1026BC005F68616E646C657200000000C1250300E8
:1026CC00C8250300CF250300DC250300F9250300F2
:1026DC0006260300132603002426030034260300D9
:1026EC003E2603004B2603005A26030090260300C7
:1026FC009D260300A82603007526030080260300F0
:10270C0088260300436F756C64206E6F7420636CB5
:10271C0065616E20757020616674657220666169F2
:10272C006C656420626F6E64696E672070726F6393
:10273C0065647572652E207064625F77726974656A
:10274C005F6275665F72656C6561736528292072BE
:10275C00657475726E65642025732E20636F6E6EC2
:10276C005F68616E646C653A2025642E00436F755A
:10277C006C64206E6F742072657472696576652066
:10278C0052414D2062756666657220666F722069D3
:10279C006E636F6D696E6720626F6E642E2070645D
:1027AC00625F77726974655F6275665F67657428CE
:1027BC00292072657475726E65642025732E2063F2
:1027CC006F6E6E5F68616E646C653A20256400699B
:1027DC006D5F626C655F616464725F676574282904
:1027EC002072657475726E65642025732E20636F7C
:1027FC006E6E5F68616E646C653A2025642E204CA9
:10280C00696E6B20776173206C696B656C792064E1
:10281C006973636F6E6E65637465642E0073645FB9
:10282C00626C655F6761705F7365635F696E666F2D
:10283C005F7265706C7928292072657475726E658B
:10284C0064204E52465F45524F525F494E56414CA2
:10285C0049445F53544154452C2077686963682080
:10286C00697320616E6572726F7220756E6C657320
:10287C007320746865206C696E6B206973206469C1
:10288C0073636F6E6E656374696E672E00436F754C
:10289C006C64206E6F7420636F6D706C6574652052
:1028AC00656E6372797074696F6E2070726F636598
:1028BC00647572652E2073645F626C655F6761700E
:1028CC005F7365635F696E666F5F7265706C7928A4
:1028DC00292072657475726E65642025732E2063D1
:1028EC006F6E6E5F68616E646C653A2025642C2097
:1028FC00706565725F69643A2025642E0052414D03
:10290C002062756666657220666F72206E65772030
:10291C00626F6E642077617320756E617661696C8D
:10292C0061626C652E207064625F77726974655F9A
:10293C006275665F67657428292072657475726E9E
:10294C0065642025732E20636F6E6E5F68616E6404
:10295C006C653A2025642E00436F756C64206E6F95
:10296C007420616C6C6F63617465206E6577207088
:10297C006565725F696420666F7220696E636F6D46
:10298C00696E6720626F6E642E00436F756C6420F5
:10299C006E6F742073746F726520626F6E642E207C
:1029AC007064625F77726974655F6275665F737479
:1029BC006F726528292072657475726E65642025A6
:1029CC00732E20636F6E6E5F68616E646C653A2067
:1029DC0025642C20706565725F69643A202564005B
:1029EC00706565725F6D616E616765725F736D6452
:1029FC000043616E6E6F7420736563757265206C35
:102A0C00696E6B20626563617573652061207072FD
:102A1C006576696F75732073656375726974792057
:102A2C0070726F63656475726520656E6465642091
:102A3C00696E2074696D656F75742E2044697363BB
:102A4C006F6E6E65637420616E642072657472794A
:102A5C002E20736D645F706172616D735F7265704F
:102A6C006C792829206F7220736D645F6C696E6BB2
:102A7C005F73656375726528292072657475726E53
:102A8C006564204E52465F4552524F525F54494D39
:102A9C00454F55542E20636F6E6E5F68616E646C8B
:102AAC00653A20256400436F756C64206E6F74204A
:102ABC00706572666F726D20736563757269747977
:102ACC002070726F6365647572652E20736D645F20
:102ADC00706172616D735F7265706C792829206FFB
:102AEC007220736D645F6C696E6B5F736563757276
:102AFC006528292072657475726E65642025732EA5
:102B0C0020636F6E6E5F68616E646C653A2025643D
:102B1C0000436F756C64206E6F7420706572666F05
:102B2C00726D2073656375726974792070726F634E
:102B3C0065647572652E20736D645F6C696E6B5F76
:102B4C0073656375726528292072657475726E657C
:102B5C00642025732E20636F6E6E5F68616E646CEB
:102B6C00653A20256400706565725F6D616E616702
:102B7C0065725F736D0050EADA308883B89F604FDE
:102B8C0015F30000C98E54686520626F6F746C6F0A
:102B9C006164657220686173207772697465207056
:102BAC00726F7465637465642069747320736574E3
:102BBC0074696E677320706167652E205468697341
:102BCC002070726F686962697473207365747469BC
:102BDC006E672074686520616476657274697369C8
:102BEC006E67206E616D652E2054686520626F6F74
:102BFC00746C6F61646572206D75737420626520EE
:102C0C00636F6D70696C65642077697468204E52CF
:102C1C00465F424C5F53455454494E47535F5041B5
:102C2C0047455F50524F544543543D3020746F20FC
:102C3C00616C6C6F772073657474696E672074684F
:102C4C0065206164766572746973696E67206E6164
:102C5C006D652E006E72665F73646800010000077C
:102C6C00240903002C090300080000004409030098
:102C7C0054090300080000002C0903004409030058
:102C8C000800000073645F626C655F6366675F7366
:102C9C00657428292072657475726E6564202573BD
:102CAC00207768656E20617474656D7074696E67E9
:102CBC0020746F2073657420424C455F434F4E4E19
:102CCC005F4346475F4741502E0073645F626C65FB
:102CDC005F6366675F73657428292072657475720B
:102CEC006E6564202573207768656E206174746549
:102CFC006D7074696E6720746F2073657420424C1C
:102D0C00455F4741505F4346475F524F4C455F43D9
:102D1C004F554E542E0073645F626C655F6366673B
:102D2C005F73657428292072657475726E656420F2
:102D3C002573207768656E20617474656D70746995
:102D4C006E6720746F2073657420424C455F434F4F
:102D5C004D4D4F4E5F4346475F56535F5555494463
:102D6C002E0073645F626C655F6366675F73657486
:102D7C0028292072657475726E656420257320771E
:102D8C0068656E20617474656D7074696E6720740B
:102D9C006F2073657420424C455F47415454535F18
:102DAC004346475F415454525F5441425F53495A22
:102DBC00452E0073645F626C655F6366675F736565
:102DCC007428292072657475726E656420257320D1
:102DDC007768656E20617474656D7074696E6720B8
:102DEC00746F2073657420424C455F4741545453B3
:102DFC005F4346475F534552564943455F434841FD
:102E0C004E4745442E00496E737566666963696565
:102E1C006E742052414D20616C6C6F6361746564FB
:102E2C0020666F722074686520536F6674446576F3
:102E3C006963652E004368616E6765207468652060
:102E4C0052414D207374617274206C6F63617469AC
:102E5C006F6E2066726F6D203078257820746F202D
:102E6C00307825782E004D6178696D756D20524152
:102E7C004D2073697A6520666F72206170706C6981
:102E8C00636174696F6E20697320307825782E0029
:102E9C0073645F626C655F656E61626C6528292086
:102EAC0072657475726E65642025732E006E726681
:102EBC005F7364685F626C6500000000F8070300D4
:102ECC0040080300080000006E72665F7364685F60
:102EDC00736F6300400803005808030008000000EB
:102EEC0043000000504F5349580000002020202080
:102EFC00202020202068282828282020202020205E
:102F0C0020202020202020202020202048101010BD
:102F1C0010101010101010101010101084848484D5
:102F2C00848484848484101010101010108181818A
:102F3C0081818101010101010101010101010101F5
:102F4C000101010101010110101010101082828288
:102F5C0082828202020202020202020202020202C5
:102F6C0002020202020202101010102000070320BD
:102F7C00041702010857104080000000EC2E0300DB
:102F8C00F02F03000431030053756E004D6F6E007B
:102F9C005475650057656400546875004672690085
:102FAC0053617400000000004A616E0046656200C7
:102FBC004D617200417072004D6179004A756E006E
:102FCC004A756C0041756700536570004F6374005F
:102FDC004E6F76004465630000000000414D0050C8
:102FEC004D0000002831030024310300243103007C
:102FFC002431030024310300243103002431030065
:10300C00243103002431030024310300FFFFFFFFB0
:10301C00FFFFFFFFFFFFFFFFFFFF00006430030017
:10302C00942F0300A0300300B42F0300E82F0300FB
:10303C0048300300F830030054300300256D2F2571
:10304C00642F25790000000025612025622025656C
:10305C00202554202559000053756E646179004D6C
:10306C006F6E64617900547565736461790057659E
:10307C00646E657364617900546875727364617908
:10308C000046726964617900536174757264617988
:10309C00000000004A616E756172790046656272CB
:1030AC0075617279004D6172636800417072696C70
:1030BC00004D6179004A756E65004A756C79004166
:1030CC0075677573740053657074656D6265720015
:1030DC004F63746F626572004E6F76656D626572D8
:1030EC0000446563656D62657200000025483A25F1
:1030FC004D3A255300000000C1050300DD05030017
:10310C00E905030041060300290603003506030008
:10311C00F505030005060300000000002E0000006A
:10312C0000000000002000400000000000200040D3
:10313C000000000000000000FF0000000090D00321
:10314C00000000000000000000000000FFFFFFFF77
:10315C00FFFFFFFF00000000000000000000000067
:10316C0000000000001001401100040000000000ED
:10317C0000000000FFFFFFFFFFFFFFFF000000004B
:10318C000000000000000000000000000000000033
:10319C0000000000FFFFFFFFFFFFFFFF000000002B
:1031AC000000000000000000000000000000000013
:1031BC0000000000FFFFFFFFFFFFFFFF000000000B
:1031CC0000000000000000000000000000000000F3
:1031DC0000000000FFFFFFFFFFFFFFFF00000000EB
:1031EC000000000000000000000000000A180100B0
:1031FC00FFFF1801FFFFFFFFFFFFFFFFFFFFFFFFB8
:10320C00FFFFFFFF1818181818181818882F03003C
:10321C00882F0300882F0300882F0300882F0300BA
:040000032000637501
:00000001FF
